:020000040000FA
:040000006FD00400B9
:101000006F00907E00000000000000009020002093
:10101000AA220020A9BDF9F56C23002000000000E1
:10102000000000006C230020902000200000000041
:101030000000000090200020000000009020002010
:101040000000000090200020902000209020002030
:101050009020002090200020582F00209424002071
:101060000000000090200020902000201E2400207E
:1010700090200020D22300209020002090200020EB
:101080009020002090200020902000209020002020
:101090009020002001A04111B7170040985F3AC688
:1010A000945F3247E39CE6FE3245410182800111A4
:1010B00013078008F337078093F787083EC20100C3
:1010C0000100B7170040930570052380B70413068D
:1010D00080FA2380C7040100010083C6B70493F699
:1010E000F60DA385D704238007049246F3A6068055
:1010F0000100010093760502D5CEF336078093F602
:10110000860836C4010001002380B7042380C70489
:1011100001000100B70614007D89558D88C70100C4
:1011200001000100010023800704A246F3A6068007
:101130000100010073370780137787083AC6010062
:1011400001002380B7042380C704010001000100CF
:1011500001003727004093061005A303D7802380A2
:101160000704B247F3A70780010001009307800836
:10117000F3B7078093F787083ECE01000100B71749
:101180000040130770052380E704130780FA2380CB
:10119000E7040100010003C7B70413670708A3852C
:1011A000E70423800704F247F3A70780010001004A
:1011B0000561828093760504BDC6F336078093F6F9
:1011C000860836C8010001002380B7042380C704C5
:1011D00001000100B7061400938606047D89558D31
:1011E00088C7010001000100010023800704C246F6
:1011F000F3A6068001000100733707801377870884
:101200003ACA010001002380B7042380C70401000B
:1012100001003727004093062005A303D7802380D1
:101220000704D24781B773370780137787083ACC12
:10123000010001002380B7042380C70401000100DE
:1012400098471367070C98C723800704E24719BF24
:101250000111814601468145114506CE97000000E7
:10126000E780605893078008F3B7078093F78708F3
:101270003EC601000100B717004013077005238028
:10128000E704130780FA2380E7040100010003C785
:101290006704136717002383E70423800704B2471A
:1012A000F3A7078001000100F2400561828041112F
:1012B000814601468145114597000000E780A05214
:1012C00013078008F337078093F787083EC40100AF
:1012D0000100B7170040130670052380C70493066A
:1012E00080FA2380D70401000100FD552396B70240
:1012F00023800704A245F3A5058001000100733790
:101300000780137787083AC6010001002380C704CD
:101310002380D7040100010003C767041367170087
:101320002383E70423800704B247F3A70780010063
:10133000010001A0BD473305F50201007D1575FDD3
:101340008280411122C426C206C6AA8401446317C2
:101350009400B24022449244410182800504130566
:10136000803E420497000000E78000FD4180C5B741
:101370009305000273A04580824573901534924016
:101380002242B2424243D2436244F2440255925551
:101390002256B2564257D2576258F25806499649D9
:1013A000264AB64A464BD64B664CF64C065D965DD1
:1013B000265EB65E465FD65F09617300203041113C
:1013C000B7170040985F3AC6945F3247E39CE6FE49
:1013D000324541018280B71700401307000323887C
:1013E000E702854717170000232EF74673002030C9
:1013F000411122C42D6426C24AC006C637190040D6
:101400001304A4AAB704002023208900977000E0E9
:10141000E780000D9C408297977000E0E780400CC9
:10142000E5B737370040834747009146BD8B639E41
:10143000D702B73600401306F00F973500009385AA
:10144000651E9737000083D7E72D03C7A6001377E3
:10145000F70F1DE3B7E70400BC4F09468945171590
:1014600000000345A5F7829731A099466394D70001
:10147000834757007300203003C786001377F70FA8
:10148000E365F6FC13851700AE9717380000231BA1
:10149000A8282380E70075B7B787004003C7670017
:1014A000098B6309071003C77700930600031377BE
:1014B0000703630DD708173800000348F87C173678
:1014C0000000130666790547B30606012380E6008F
:1014D00083C57700173700001307077A429793F503
:1014E000F50F2300B70003C58700973500009385EB
:1014F000A577C2951375F50F2380A5000347070054
:1015000089451377F703630CB70C63E7E50A6306B5
:10151000071A8545630CB7129737000083C7D77643
:101520003307F600034707001377F70F19CB85073A
:1015300093F7F70F3D476363F71A17370000A305CA
:10154000F774B787004009472383E700B787004057
:1015500083C77700E207E18763DE0704973700005F
:1015600083C79772173700001307076F3E978546AA
:101570002300D70017370000130707703E97930624
:1015800000032300D700173700001307E76D3E97CD
:10159000A14685072300D70093F7F70F3D47636403
:1015A000F71417370000A301F76EB787004009470B
:1015B0002383E70073002030930610026300D70EE8
:1015C000930620026305D70693060002E316D7F4BC
:1015D00003C727021377C70F13672700D5A803C7D0
:1015E00067001377070465CB03C7A702173800000D
:1015F00013080848173500001305453F134707082F
:101600002385E70203C7A7021377370F1367870005
:101610002385E702814713070004B305F5008C41D9
:10162000B306F80091078CC2E399E7FEF5B503C74E
:10163000A702134707042385E70203C7A70213770E
:10164000C70F136727002385E702F9B503C76700B3
:101650001377070449C303C767021738000013084C
:10166000E834173500001305252C1347070823839A
:10167000E70203C767021377370F136787002383D7
:10168000E702814713070004B305F5008C41B30658
:10169000F80091078CC2E399E7FEBDBD03C767025E
:1016A000134707042383E70203C767021377C70FB3
:1016B000136727002383E70285B503C76700137705
:1016C000070411CB03C727021377370F136787006F
:1016D0002381E70291B5238006003DBD97370000C6
:1016E000A384075AB9BD97370000A38F075875BD6B
:1016F0002303048015472303E48001002302A48010
:10170000828083076480E3CE07FE23030480828007
:1017100083076480E3CE07FE03454480828083070D
:101720006480E3CE07FE2302A4808280411126C498
:101730004AC24EC006C61377F50BAD47AA892E895B
:101740009544630CF700194597000000E78080FA84
:1017500097000000E78020FB8D444E859700000035
:10176000E78040F9FD59FD1463983401B240A2446A
:101770001249824941018280135509011375F50F01
:1017800097000000E780E0F92209F1BF011126CCA3
:1017900006CEB704080097000000E780C0F61545A4
:1017A00097000000E78000F597000000E78080F6D2
:1017B00097000000E78000F62AC697000000E78047
:1017C00080F432459377150089EB13651500137586
:1017D000F50FF240E24405618280FD14E9F0014515
:1017E000CDBF397126DC4ADA4ED852D656D45AD2F9
:1017F0005ED006DE62CE66CCB7E700E07D5783AAF6
:10180000070022C603AA470023A0E71823A2E7186F
:10181000B7170040130770052380E704130780FA09
:101820002380E70483C74704930B75FFB684E20760
:1018300093FBFB0F8546AA892E8B32893724004003
:10184000E187015763FA76016308D50089461307DB
:1018500000026313D5000157D98F93F7F70FB71C18
:1018600000402382FC0411472303E4801305F00F9A
:1018700097000000E78000E8094C97000000E7802F
:1018800080E863657C15B7050700DA9537870700A0
:10189000795563FEE504B3879500636AF704370B57
:1018A0000800A94733EB65016395F90881E8814495
:1018B00097000000E78020E5268515A8DA85094510
:1018C00097000000E780C0E605090345F9FFFD1415
:1018D000050B97000000E780C0E481C49377FB0FFD
:1018E000E5F797000000E780A0EA69F17D55B7179A
:1018F0000040130770052380E704130780FA238054
:10190000E70403C74704418B2382E704F250B7E79B
:1019100000E023A0571123A24711E2543244525948
:10192000C259325AA25A125B825B724CE24C21615C
:101930008280A547639BF90685691309F00FB306FA
:101940009900B3742B01B6941349F9FFB37499004D
:10195000856B33796901416B9387F9FFB3F72701F1
:1019600099E363FC340193D94900C147E3E637FFAB
:101970003DBF0569C1697D19D9B71305800D63881D
:101980006901130500026384790113051008CA85F3
:1019900097000000E780C0D997000000E78040DF93
:1019A00031D54E99B38434416DBFDA852D4597000A
:1019B0000000E780E0D7CA94E30B99EE0509970091
:1019C0000000E78020D5A30FA9FEFDB79387F9FF9C
:1019D00093F7F70F636DFC0C83C71C0413073008E3
:1019E0006315F706370708006361EB06B3079B0032
:1019F000B706100063FBD704334BEB0089476399AC
:101A0000F9068980D549E38404EADA850945970017
:101A10000000E780E0D111090327C9FF9147232087
:101A2000E48003076480E34E07FE23033481FD173F
:101A3000EDFBFD14110B81C49377FB0FE9FF9700B9
:101A40000000E780E0D461F155B5B717004003C747
:101A50005704B70708001377070219E3B787070091
:101A60007955E376FBE833079B00E3F9E7F841B5E6
:101A70008547E380F9F0DA852D4597000000E7807F
:101A800020CB9389F4FFE38404E297000000E78011
:101A900060C893F7390091EB83260480032709007F
:101AA00093074900E396E6E03E89CE84D9BFB54767
:101AB0006399F9001305900B97000000E78080C33D
:101AC000FDB3B1471305B00AE388F9FE9947639760
:101AD000F904B7050800B365BB002D459700000069
:101AE000E78000C581448D4BA14997000000E78045
:101AF00060C263967401832704802320F900850463
:101B0000E39534FF8327048013172B0163550700E7
:101B10002312F90069BB2322F90051BB9D47639F43
:101B2000F90281451305B00497000000E78040C02A
:101B3000BD442320090023220900FD59970000001D
:101B4000E78040BD93F77400CA9703C70700FD14F0
:101B5000398D2380A700E39334FF91BBA14763979E
:101B6000F90697000000E780A0C28144630D0B00D6
:101B70008D479304C0036308FB00930400056304CE
:101B80008B01930440041375C507E30295D21945F0
:101B900097000000E78000B697000000E780A0B63D
:101BA000054597000000E780E0B426859700000017
:101BB000E78020B7094597000000E78080B69700CE
:101BC0000000E780E0BCE31405CE0DB39147639FAE
:101BD000F9001305600697000000E780A0B19700A8
:101BE0000000E78040B213059009F9B5E38109CC04
:101BF000F1547DB9BD66014717360000130606355E
:101C0000938606A685458347060093F7F70F91C391
:101C100082800507E3F9E6FE973700002388B73294
:101C2000DDB77D166206618693178601E18763D46E
:101C3000070001458280931726003307F500AE9711
:101C400018439C4363E7E7007D16E37FF7FC7D556F
:101C5000828005458280FD15E205E18513978501A7
:101C6000618793F7F50F63480700FD15139725006B
:101C70002A97584365D713851700620561858280CE
:101C80003308B5021C4283A80600B335B502C297DB
:101C900033B50701AE98469585486367B5006394F0
:101CA000A50063E3070181480C43C6950CC388C2B5
:101CB0001CC2828081471397870161876343B70005
:101CC0008280139727002A97232007008507E5B70E
:101CD0008147014793968701E18663C5B6001335B6
:101CE0001700828093962700AA9694428507558F05
:101CF000D5B793D755408A07AA979C430545331516
:101D0000B5007D8D828017F3FFDFE702833D2A84D3
:101D100097000000E78060F405C5931725003E9406
:101D20000327C4FF814711EB7D1516053E9542053B
:101D3000418517F3FFDF6700033D05838507E5B79E
:101D40000145C5BF81471397870161876343C7007A
:101D5000828013972700B386E50094422A9785076F
:101D600014C3D5B77D1662066186014793178601B5
:101D7000E18763D50700133517008280931726008B
:101D8000B306F500AE9794429C437D16B58F5D8FE8
:101D9000F1BF8A05AA9501476363B500828083A6D7
:101DA000C5FFF11593D71600D98F9CC11397F60183
:101DB000E5B72A830148014701456343D700828084
:101DC000B387050183A80700B30706019C43C697A4
:101DD000AA976384F80033B517010507B308030118
:101DE000620723A0F80061871108C1BF2A83014759
:101DF0008147014563C3D70082803388E50083288B
:101E00000800330EE600032E0E003388A840330886
:101E1000C8416384080133B508018507B308E300AE
:101E2000E20723A00801E1871107E9B717F3FFDFF5
:101E3000E702232B0111B286B2842E86AA850A8579
:101E400097000000E780C0FA2A84A6850A859700DB
:101E50000000E78020E833348000060413351500C5
:101E6000018D056117F3FFDF6700E32917F3FFDF3B
:101E7000E702A3244111AA89AE8A328BB68402C23A
:101E800002C402C60144131C8401135C8C416349E3
:101E90009C02939B1400FD1B0549138CF4FFF15C1D
:101EA00033048901620461846340740792478E049D
:101EB000CE9423AEF4FE410117F3FFDF67006323E6
:101EC00013192400B30B2B01014A93172A00D6974C
:101ED00083A50B0088437800340050009700000071
:101EE000E78040DA050A93178A01E187F11BE35E78
:101EF000FCFC92474E9905042320F900A2473EC2FC
:101F0000B24702C63EC441B7131A8901135A8A4127
:101F1000131D240093178A01E18763CF970092472E
:101F20000A044E941CC0A24705091379F90F3EC25A
:101F3000B24702C63EC4ADB7B3079A0313152A00D1
:101F400056950841780034005000050AEA97DA9760
:101F50008C4397000000E780E0D26DBF197106C284
:101F600012C416C61AC81ECA22CC26CE2AD02ED219
:101F700032D436D63AD83EDA42DC46DECAC0CEC2C9
:101F8000D2C4D6C6DAC8DECAE2CCE6CEEAD0EED2F9
:101F9000F2D4F6D6FAD8FEDA971500009385058CB0
:101FA0008841E700050092402242B2424243D243B8
:101FB0006244F244025592552256B2564257D257C5
:101FC0006258F25806499649264AB64A464BD64BBD
:101FD000664CF64C065D965D265EB65E465FD65F45
:101FE0000961730020300000972100209381810156
:101FF000175100201301018117F5FFFF1305C500DC
:102000009705002093850500171600201306C6FDCE
:1020100063FAC5008322050023A055001105910530
:10202000E3EAC5FE17150200130545F097150020D9
:102030009385C5FB171600201306C66563FAC50015
:102040008322050023A0550011059105E3EAC5FE92
:102050001715002013050564974500209385053B5F
:102060006377B500232005001105E36DB5FEFD4241
:10207000739002BC8D4273904280B722000093821D
:10208000828873900230970200209382A2F793E235
:1020900032007390523097520000938282B873904E
:1020A00012346FB0F47573002030397101436EC67D
:1020B00019A0397141536AC866CA62CC5ECE19A0B4
:1020C000397101535AD056D252D44ED64AD826DA54
:1020D00022DC06DE33016140828241114AC026C201
:1020E00022C406C68282B24D4101024D924C224C5E
:1020F000B24B4101024B924A224AB2494101024984
:1021000092442244B240410182803D432A87637356
:10211000C3029377F700BDEFADE5937606FF3D8AE6
:10212000BA960CC34CC30CC74CC74107E36BD7FE30
:1021300011E28280B306C3408A0697020000969699
:102140006780A6002307B700A306B7002306B700E1
:10215000A305B7002305B700A304B7002304B70005
:10216000A303B7002303B700A302B7002302B700FD
:10217000A301B7002301B700A300B7002300B700F5
:10218000828093F5F50F93968500D58D9396050182
:10219000D58D61B7939627009702000096968682A8
:1021A000E78086FA9680C1171D8F3E96E374C3F8C8
:1021B000A5B73367B500FD530D8B79E7B7877F7FF0
:1021C0009387F7F710419441B372F6003363F6003A
:1021D000BE92B3E262006397720C6318D606504158
:1021E000D441B372F6003363F600BE92B3E26200EC
:1021F0006398720A631BD60410459445B372F600C7
:102200003363F600BE92B3E262006391720A631E0A
:10221000D6025045D445B372F6003363F600BE9241
:10222000B3E26200639A72086311D60210499449BE
:10223000B372F6003363F600BE92B3E262006393BA
:1022400072085105D105E30FD6F6131706019397CF
:102250000601631CF7001357060193D706013305E7
:10226000F7409375F50F91E982804183C18333056F
:10227000F7409375F50F91E182801377F70F93F78D
:10228000F70F3305F74082800346050083C605003B
:10229000050585056313D60065FA3305D6408280AF
:1022A00011059105E312D6FE014582802105A105A5
:1022B000E31CD6FC014582803105B105E316D6FC4E
:1022C000014582804105C105E310D6FC01458280AD
:1022D000B717004003C777051377E70FA38BE70411
:1022E000130700F8A38DE7043D47238CE704130789
:1022F0005003A38CE70403C7A7051377D70F238DDB
:10230000E7048280B717004003C7E7020D89411137
:102310001377C70F498F93068008F3B6068093F6AC
:10232000860836C601000100930670052380D70495
:10233000930680FA2380D704010001002387E70277
:1023400023800704B247F3A7078001000100410181
:10235000828041112A83014E930E407E130F001993
:10236000930F400663E56E129308001913034006AD
:10237000B3781503854E0D4FA14F337365020D8958
:102380001335150063EFBE121308F6FF79467298F5
:102390004208135808013307C70213D61700BE07B7
:1023A00032976146B3F6C60213068070B386C60242
:1023B0003697A166F58F42075D8FB716004083C739
:1023C000F60293F70708A303F1000346710083C7E1
:1023D000F60293F70708E394C7FE83477100B71628
:1023E000004093F7F70F6388071293078008F3B74D
:1023F000078093F787083EC401000100B71700402B
:10240000930670052380D704930680FA2380D704AF
:102410000100010023AA070383C6170393E60608F9
:10242000A388D70223800704A247F3A707800100EF
:1024300001001166B71700407D16D45BC85F938515
:102440004703A98EF18EF5FA93068008F3B606804D
:1024500093F6860836C601000100930670052380B6
:10246000D704930680FA2380D7040100010098C1A5
:1024700003C7170313670704A388E7022380070431
:10248000B247F3A7078001000100410182807D135C
:102490003368E3039308E016630E08003368F30320
:1024A0009308D016630808009378330093B8180097
:1024B0009388D81633081E01131E0801135E0E01FF
:1024C00055B56393E5030548638608000148630337
:1024D00003002A8871087298FD15131E0801C205B1
:1024E000135E0E01C18179BD13F8150063F4BF00BE
:1024F0007908D5B713381800E5BF83C7F60293F7FC
:102500000708A303F1000346710083C7F60293F79F
:102510000708E394C7FE8347710093F7F70FF1DFD5
:10252000E9B531714AD966CB06DF22DD26DB4ED70D
:1025300052D556D35AD15ECF62CD6AC96EC7AA8C26
:1025400002D897100000E78020B12A8993078008FD
:10255000F3B7078093F787083EDA01000100B71749
:102560000040130770052380E704130780FA2380D7
:10257000E7040100010003C7F7021377770FA38771
:10258000E70203C7F70213678700A387E7022380E8
:102590000704D257F3A70780010001000545970003
:1025A0000000E78060D6130780C13347E902116A53
:1025B00093070AE893065002BD69930BA004814A71
:1025C000014B13048008930470057D1AB347F90288
:1025D0003307D7023EC0FD873ECC938709A69309F7
:1025E000803E3347F7023AC27D873AC43347390306
:1025F0008549B399990193D93940B306D702B30BF2
:102600007703B3C6F602B3CBFB0236C6FD8636C8E7
:1026100093D6FB4136CEB7460F0093860624334946
:10262000D9028566938606FAB3969601B389E902C4
:10263000130760553309D90293060010B389E902E4
:102640003349D902B3C9F9029316390036CA37198A
:102650000040FD8636D0930D090493D7F9413ED250
:10266000F336048093F6860836DC010001009307F8
:1026700070052380FD00930680FA2380DD000100B1
:1026800001008346390593F6860FA309D9048346D2
:10269000390593E61600A309D90423800D00E256FC
:1026A000F3A6068001000100130C80FA116DF336C9
:1026B000048093F6860836DE01000100930770055A
:1026C0002380FD0023808D01010001008346390530
:1026D000216693E60602A309D90483560905B3E6E9
:1026E000A6012318D90483560905D18E2318D904CD
:1026F00023800D00F256F3A60680010001008346F8
:10270000390593F606026381061A03463905218AC4
:102710006DDE081897100000E7800098733604807B
:1027200013768608B2C20100010023809D00238039
:102730008D0101000100B717004003C6370513766D
:10274000F60DA389C70403C6370513660602A389DD
:10275000C704835609052166B3E6A6012318D904E8
:1027600083560905D18E2318D90423800D0096467F
:10277000F3A60680010001008346390593F60602A0
:10278000638B061483463905A18AEDFE970000206D
:10279000E7806090AA8636D497000020E780A08F5B
:1027A000A256E30AD5FE835609054255B3E6A601B3
:1027B0002318D90497100000E780C08F834639059D
:1027C000A18AEDDE03560905834629058247337643
:1027D000CA00B306DA0293D5F641B296B388F64042
:1027E000E24733B8C6002E983308F840A247B3B684
:1027F00016013308D84063C70701631DF8009247EC
:1028000063FA1701C247634FF80E63950701B24799
:1028100063EAF80E894663E9660FF24693151800DD
:1028200013D3F8015E8613951800B365B30042D642
:1028300046D497D00100E780C0B83258050B137B0F
:10284000FB0F63470001631A0838A25863870838F2
:1028500013081500B336A800B69513D6F5013298C3
:10286000B336C800AE9613581800FE06B3E606014C
:102870007336048013768608B2C6010001002380F7
:102880009D0023808D01010001000356C902B2960C
:10289000C206C1822316D90223800D00B646F3A6D4
:1028A00006800100010021B5F336048093F6860806
:1028B000B6C00100010023809D0023808D0101002E
:1028C00001008346390593E60602A309D904238053
:1028D0000D0086460DB5F336048093F68608B6C41F
:1028E0000100010023809D0023808D010100010073
:1028F0008346390593E60602A309D90423800D0017
:10290000A646BDB5E30B0BF0F336048093F68608BC
:10291000B6C801000100930680FA23809D00238041
:10292000DD00010001008346390593F5FC0F93F6A5
:10293000860FA309D90483463905CD8EA309D9048E
:1029400023800D00C646F3A6068001000100130592
:1029500080FA03463905930639051D8A631C9629BA
:102960007336048013768608B2CC0100010013068A
:1029700080FA23809D002380CD000100010003C662
:1029800006001376F60D2380C60003C60600136604
:1029900006022380C600835609051166D18E2318CE
:1029A000D904835609052166D18E2318D9042380C2
:1029B0000D00E646F3A6068001000100130680FA2A
:1029C0008346390593F60602638006268346390559
:1029D000130C3905A18AFDDA081897000000E7807A
:1029E000A06BF336048093F68608B6D00100010090
:1029F000930680FA23809D002380DD000100010002
:102A000083460C00116693F6F60D2300DC00834626
:102A10000C0093E606022300DC0083560905D18EE4
:102A20002318D904835609052166D18E2318D904A9
:102A300023800D008656F3A60680010001001306D0
:102A400080FA8346390593F60602638A0620834698
:102A50003905A18AEDFE97F0FF1FE780C0632A8C3D
:102A600097F0FF1FE7802063E30C85FF835609057D
:102A700011664255D18E2318D90497000000E780D3
:102A800060638346390513063905A18AFDDAF336FA
:102A9000048093F68608B6D401000100930680FAFC
:102AA00023809D002380DD00010001008346060095
:102AB00093F6F60D2300D60023800D00A656F3A64C
:102AC0000680010001008356090503462905D24707
:102AD000B376DA003306CA021305800C9355F6412B
:102AE0003696330DF6408257333CD6002E9C333653
:102AF000A601330CFC40330CCC40330885039256BE
:102B00004E86B335A5033305A503C29597D00100C2
:102B1000E780208B63468001631E0C16630C0D1644
:102B2000130615003335A6002E959356F5013696FB
:102B3000B335D600AA959396F50105828585D18E89
:102B40006346B000639D051A638B061A0356C902DB
:102B500015823305D6003336C500B2956348B00000
:102B6000639105241306F00F637DA622894663F363
:102B7000561593078008F3B7078093F78708BED6EA
:102B80000100010037170040930770052300F70488
:102B9000930780FA2300F704010001008356C7025F
:102BA00089678117D58FC207C1832316F7022300D7
:102BB0000704B657F3A7078001000100FA506A54D2
:102BC000DA544A59BA592A5A9A5A0A5BFA4B6A4C49
:102BD000DA4C4A4DBA4D296182801308F5FF33352E
:102BE000A800FD152E951356F5013298B336C8008E
:102BF000AA9695B9F336048093F68608B6CA010002
:102C0000010023809D002380AD0001000100834668
:102C10003905CD8EA309D90423800D00D646F3A62D
:102C200006800100010035B3F336048093F6860870
:102C3000B6CE0100010023809D002380CD0001005D
:102C400001008346390593E60602A309D9042380CF
:102C50000D00F646F3A606800100010095B3F33699
:102C6000048093F68608B6D20100010023809D00FF
:102C70002380CD00010001008346390593E606025A
:102C8000A309D90423800D009656F3A606800100FF
:102C9000010045BB9306F5FF33B5A600FD152E9543
:102CA0009355F501AE96B3B5B600AA951396F50106
:102CB000858269B5F336048093F68608B6D801009C
:102CC0000100930680FA23809D002380DD0001002F
:102CD00001008356C9020566011693F6F60FD18EE0
:102CE000C206C1822316D90223800D00C656F3A660
:102CF000068001000100850A93FAFA0F95B233E6C7
:102D0000B60045C20356C9023305D0403338A0008F
:102D1000B305B040B385054115826345B000D1E1EC
:102D20006371A608894663F0560593078008F3B7D8
:102D3000078093F78708BEDA01000100B71700404B
:102D4000130770052380E704130780FA2380E70444
:102D50000100010003D7C7027D8B2396E702238081
:102D60000704D65781BDF336048093F68608B6DC97
:102D700001000100930680FA23809D002380DD007E
:102D8000010001008356C9020566011693F6F60F8D
:102D9000D18EC206C1822316D90223800D00E656C9
:102DA000B9B793078008F3B7078093F78708BEDEAB
:102DB0000100010037170040930770052300F70456
:102DC000930780FA2300F704010001000356C702AD
:102DD00093975600B297C207C1832316F7022300C8
:102DE0000704F657C1BB914763EEB70217E701002E
:102DF000130787FB8A05BA959C41BA978287B71754
:102E0000004003A7470B1345F5FF698F23AAE70A84
:102E100003A7070B698F23A8E70A03A7070A798D81
:102E200023A0A70A8280B717004083A6470B134749
:102E3000F5FFF98E23AAD70A83A6070B558D23A881
:102E4000A70A83A6070A758F23A0E70A8280B7170F
:102E5000004003A7470B498F23AAE70A03A7070BE4
:102E60001345F5FF45BFB717004083A6470B13472F
:102E7000F5FF758F23AAE70A03A7070A598D4DB7F7
:102E8000B717004003A7470B498FEDB7914763EE93
:102E9000B70217E70100130767F28A05BA959C414C
:102EA000BA978287B717004003A7470D1345F5FF70
:102EB000698F23AAE70C03A7070D698F23A8E70CE6
:102EC00003A7070C798D23A0A70C8280B7170040B9
:102ED00083A6470D1347F5FFF98E23AAD70C83A6C7
:102EE000070D558D23A8A70C83A6070C758F23A06B
:102EF000E70C8280B717004003A7470D498F23AA2C
:102F0000E70C03A7070D1345F5FF45BFB7170040B2
:102F100083A6470D1347F5FF758F23AAE70C03A778
:102F2000070C598D4DB7B717004003A7470D498FC0
:102F3000EDB7797122D43714004026D24AD0035914
:102F400024028354040206D64209C2044ECE52CC57
:102F500056CA13590901C1802DE11379F9F793F489
:102F6000F49F4209C20413590901C18093078008E4
:102F7000F3B7078093F787083EC401000100930769
:102F800070052300F404930780FA2300F404010081
:102F90000100231124032310940223000404A247F8
:102FA000F3A7078001000100B25022549254025945
:102FB000F249624AD24A45618280B7F507008146EC
:102FC0003000B105194597000020E7808081A247B5
:102FD00013972701E34A07FC1369090893E40440A7
:102FE00093098008F3B7098093F787083EC0010072
:102FF0000100930A700523005405130A80FA230088
:10300000440501000100231124032310940223002E
:1030100004048247F3A7078001000100294597F0C7
:10302000FF1FE7802031F3B9098093F989084EC268
:1030300001000100230054052300440501000100A4
:103040008357040293E707202310F40223000404AB
:103050009247B9B7B7170040884742054181937737
:10306000050491EB9377F5013755E80113050580C9
:103070003345F50282809377050C130700046397AC
:10308000E7009377F50137459C1CCDB72165130503
:1030900005D0828037E700E01C435443A183E20659
:1030A000D58F1CC1FD572320F7182322F7188280E3
:1030B00013178500B7E700E023A0E710618123A282
:1030C000A7108280B7F700E08847CC47828081470D
:1030D00037370040A14663C4C7003285828003456C
:1030E000B740E38EA6FE3385F5000345050085074E
:1030F0002304A740CDB797070020938727EF9C4371
:1031000017370020130787303E95636EE5001737A9
:1031100000201307273F6368A70017070020232715
:10312000A7EC3E858280FD57EDBF8280411122C40D
:1031300006C62A8497000000E78000F22947B307FB
:10314000E502B2408D83B3D7870222449507B3D7F7
:10315000E70237370040C207C1832316F700410159
:103160008280411137150E0006C697000000E780E7
:1031700020FCB7370040130770F82381E7000D47A4
:10318000A381E70013070004A380E7000547238716
:10319000E700B24041018280373700408347270073
:1031A0001A0593F7F703C98F93F7F70F2301F70079
:1031B0008280B737004003C7170019C9D98DA38093
:1031C000B70003C70700136787002380E7008280EA
:1031D00093C5F5FFF98DA380B7008280AE872A875B
:1031E000B736004021463738004089E71703000012
:1031F0006700E3F383C8B600E30916FF05078348B9
:10320000F7FFFD17C20723041801C183F9BF41115D
:1032100022C406C62A8497000000E780E0E329471D
:10322000B307E502B2408D83B3D7870222449507E6
:10323000B3D7E70237370040C207C1832316F740F0
:1032400041018280716541111305052006C6970072
:103250000000E78000FCB7370040130770F82381B7
:10326000E7400D47A381E74013070004A380E74030
:1032700005472387E740B24041018280CC4141119C
:1032800006C6328503C6150083C5050022064D8E8D
:1032900042068D654186138875A2630C0611634B47
:1032A000C804138845A26300060D634AC8009385CD
:1032B00035A26301B6082390060029464DA0138865
:1032C00055A26305060D938565A2E316B6FE8D45EE
:1032D0001D4663E6E5081146198E63F3C7003E8676
:1032E000B7E704002390C600FC4797E501009385EB
:1032F00025AF9DA0138895A263030611634E060DAA
:103300001388A5A263000613938505A5E315B6FAF5
:1033100099451D4663E5E504198E63F3C7003E86B3
:10332000B7E704002390C600FC479705002093856B
:1033300025D61DA09D451D4663E3E5022146198E55
:1033400063F3C7003E86B7E70400FC472390C6003E
:103350009705002093858534BA9582970146B2403F
:10336000328541018280AD451D46E3EAE5FE3146E6
:10337000198E63F3C7003E86B7E704002390C600AA
:10338000FC4797E50100938525A8F9B7B1451D468F
:10339000E3E7E5FC3546198E63F3C7003E86B7E7E1
:1033A00004002390C600FC4797E501009385C5A65D
:1033B00065B78D451D46E3E4E5FA1146198E63F3C2
:1033C000C7003E86B7E704002390C600FC4797E598
:1033D00001009385A5A149B78D451D46E3E1E5F8B8
:1033E0001146198E63F3C7003E86B7E704002390A9
:1033F000C600FC4797E501009385C5A3B1BFA5456D
:103400001D46E3EEE5F42946198E63F3C7003E86B8
:10341000B7E704002390C600FC4797E501009385B9
:10342000A59D1DBFB5451D46E3EBE5F23946198E56
:1034300063F3C7003E86B7E704002390C600FC474D
:1034400097E501009385C59801BFB7E7040003A382
:103450000713970600209386A6C24146A545170587
:1034600000201305E5B802832D455DE703C505007F
:103470000947631FE50803A84500411106C6034735
:10348000180032850346080022074168518F9308CF
:1034900028FE6307170563E9E800051863030703BF
:1034A00023900600294591A8130648FE630AC70425
:1034B0001518E31707FF15463E87637BF60015478F
:1034C00001A8130600023E876374F600130700028A
:1034D000B7E704002390E600FC471316070111A884
:1034E0003E8691C30546B7E70400FC472390C6001B
:1034F0004206CC45418282970145B240410182801B
:10350000130600083E87E375F6FC13070008C9B7E9
:103510002390060005458280828041677917630405
:10352000E504411122C406C685472A84639FF5003D
:10353000B7E7040022852244B24003A3871397050E
:1035400000209385E52F4101028389476399F500A7
:10355000B7E7040083A7070B8545829771D9B2406E
:103560002244410182808280797126D252CCAE847D
:103570002A8A97E501009385E58D17E5010013057B
:10358000E58F06D63AC622D44AD0368432894ECE4A
:1035900097C00100E780202EA28517E501001305E2
:1035A000E58E97C00100E780002D294597C00100F6
:1035B000E780403183C7840093F70702F9E383C9AA
:1035C00004008947054532476396F908D44083C70C
:1035D000160083C60600A207D58FC166138616FEA5
:1035E000638CC7028D16638FD7068D6693862690EF
:1035F00029456391D706B7E70400A286225403A3A6
:103600004714B250F2494A86A6850259925452850F
:10361000624A8547456102832D450DEF93070002FD
:10362000354563E98702B7E70400FC47C844130641
:103630000002CA8582978149970700209387072156
:103640009C43014581CB9C4391C74E852286CA8508
:1036500082970145B250225492540259F249624A6B
:10366000456182802D457DF79307700F3545E3E373
:1036700087FEB7E70400FC47C8442286CA858297C4
:1036800065BF2145C1BF411122C437E4040083272F
:10369000841326C2AA84416506C697050020938537
:1036A000251A7D1582978327C40A17050000130584
:1036B00005E78588829795C0032304132244B2400E
:1036C000924497060020938626AE4146C5451705CD
:1036D00000201305659C41010283B24022449244BC
:1036E00001454101828019C59707002023A0A71634
:1036F00001458280454582801147636AA70A97D6B3
:1037000001009386E6730A0536951841411106C6F5
:103710003697AE87B2850287130700026145639D25
:10372000E700B7E70400FC47130600021705002076
:10373000130545F782970145B24041018280054754
:103740006145E39BE7FEB7E70400FC470546170524
:103750000020130525F7F9BF1307700F6145E39D9E
:10376000E7FCB7E70400FC471306700F17050020BD
:10377000130585F5C1B7130700086145E39EE7FA15
:10378000B7E70400FC4713060008170500201305DF
:1037900025034DB715476145E390E7FAB7E7040005
:1037A000FC471546170500201305C50961B70945F3
:1037B0008280411126C2B7E4040083A7C41322C447
:1037C0004AC006C62E8497050020938565072A897E
:1037D0008297058905C5970700209387E78B83D7D4
:1037E000A70BA28503A3440D2310F4002244B2408A
:1037F00092444A850249014641010283B240224473
:103800009244024949454101828097070020238163
:1038100007049707002023AF0702B717004003A74C
:10382000070CB706C0FFFD16758F23A0E70C03A792
:10383000070DB7064000558F23A8E70C03A7070C18
:103840003D9B23A0E70C03A7070D1367070123A8DF
:10385000E70C8280B717004003A5470C83A7470CED
:10386000598113451500C18B058999E3136525001E
:103870009707002083C7C7FD6380A7029707002032
:103880002388A7FC11C9970700209387A7FC03A3EF
:1038900007006303030002838280114517F3FFFFD3
:1038A000670063C8011122CC06CE3714004026CA37
:1038B0004AC84EC652C483447405034AB4058349BA
:1038C00084050349940597F0FFFFE780A0A0834794
:1038D000A40593F4F40F137AFA0F93E71700230D5E
:1038E000F40493F9F90F1379F90FB717004003C7E0
:1038F000A705058B6DFF03D5C705A38D4705238C51
:103900003705A38C2705A38B9704F2406244D24469
:103910004249B249224A05618280411193970501CB
:1039200022C406C626C2C1872E8463DC0700B7E422
:103930000400FC54829719C1BC5482972165218DE3
:1039400015A893F7150013C515008DE793F725000B
:103950009DC797000000E78020F0B7E70400BC4F48
:103960001306000A894517050020034525EF8297B5
:1039700013452400B240224492444101828093972F
:10398000250163D80702B7E4040083A7C41E829709
:1039900097000000E780A0F0BC4C375607001306E4
:1039A0000630896517050020034545EB82970965B8
:1039B00079B7939715010145E3DE07FA17D50100A2
:1039C0001305C55497C00100E780C002B7E70400A3
:1039D000BC4F13060064916517050020034505E8F8
:1039E00082971165A9BF1D71A2CC37E404005C5C0D
:1039F000485886CE494697D501009385A54C8297B5
:103A000011E917D501001305254D97C00100E78086
:103A100060FE01A0B7F600E0795798CAFD57DCCAEE
:103A20000567B7E700E023A0E7101306F00290C295
:103A300023A0E718010001003707002018471306EC
:103A4000000481459706002023A8E6E04157A38A99
:103A5000E7403C4408088297970700209387077C3B
:103A60003EC8856713870740938757D1231AE10023
:103A70002312F1021307B00F97F7FFFF9387C76474
:103A80002310E1023ED81547970700009387C7E14E
:103A9000B7F50700A30FE1003EDC054797070000DC
:103AA0009387E7DF81463000E10519452301E102F4
:103AB0003EDE97F0FF1FE780C0D218088147994685
:103AC00030003E960346060085070507A30BC70096
:103AD000E398D7FEC24791C70357410185676373D7
:103AE000F70001A0B7E7040083A7470A08088297F8
:103AF000AA8511C917D501001305453F97C00100DC
:103B0000E78060D701A0F6406644256182804111BC
:103B100026C2B7E4040083A7040806C622C417051A
:103B200000001305C5DF829717040020130404D397
:103B30002300A40097000000E780800297000000A7
:103B4000E780E0CC03450400224403A38405B2408F
:103B5000924413060032896541010283797106D6C9
:103B600022D413078008F337078093F787083EC2F3
:103B700001000100B7170040930570052380B704CA
:103B8000130680FA2380C7040100010083C6F702F0
:103B900093F6A60FA387D702238007049246F3A6C5
:103BA00006800100010073370780137787083AC445
:103BB000010001002380B7042380C7040100010035
:103BC00003C7F70213672700A387E70223800704D0
:103BD000A247F3A7078001000100054597E0FFFF1A
:103BE000E780807297000000E78060CB0147814644
:103BF0008147054685451305407E97E0FFFFE78036
:103C0000807537E404003C44680051468145829742
:103C1000B707C0A83EC8B787E803938707D03ECA56
:103C200097E7FF1F9387A7793EC67C586800829765
:103C3000B250225445618280411197E5010093857D
:103C4000E59117D501001305652306C697C001004D
:103C5000E78060C217E50100130545A997C0010080
:103C6000E78060C1B2402945410117C301006700E8
:103C700063C5411197E501009385858F17D5010034
:103C80001305C51F06C697C00100E780C0BE17E533
:103C90000100130565A497C00100E780C0BDB240D4
:103CA0002945410117C301006700C3C1411122C466
:103CB00006C6834705002A849DC797E501009385C2
:103CC000E59017D501001305651B97C00100E7803B
:103CD00080BA4C4017E50100130505B697C00100F6
:103CE000E78060B93DA058410DEF97E5010093854D
:103CF000E58D17D501001305651897C00100E78011
:103D000080B717E501001305A5B497C00100E7804F
:103D100080B62244B2402945410117C30100670023
:103D200063BAA1679386D7036313D70297E50100AF
:103D30009385C58917D501001305451497C0010067
:103D4000E78060B317E50100130585B17DBFED077E
:103D500097E501009385858717D5010013050512A6
:103D6000631BF70097C00100E780E0B017E5010092
:103D7000130545B059BF97C00100E780C0AF4C4064
:103D800017E50100130505B191BF411197D5010059
:103D90009385457F17D501001305450E06C697C0CC
:103DA0000100E78040ADB2402945410117C3010041
:103DB000670043B1397122DC26DA4AD82E842A8979
:103DC0008145B2844808714636C606DE97E0FFFF9B
:103DD000E780E03397F7FF1F9387075EDC4783D7C1
:103DE0000700231C2101231BF10097600000E780DE
:103DF00040B8B246230DA10091E285469307001911
:103E00003ECE2686FD57A2854808A30DD100230289
:103E1000F10297600000E780A0B8F2506254D254DB
:103E20004259216182808546170300006700C3F86C
:103E30004111972700202396078E97170020238F84
:103E4000077C06C6170700200347C72D9307F00A13
:103E50006315F7029307F0F889451705002013054D
:103E6000652C17070020230FF72A97070020A38B44
:103E7000072A97600000E780C07897700000E7800D
:103E800080A597700000E780C0A681453705040033
:103E90009707002023AE07269707002023890726CF
:103EA000970700202398071E970700202396071CDA
:103EB00097070020239B072497070020239C0724B3
:103EC00097400000E780C002014597600000E7804E
:103ED000407C97D501009385656D17D501001305CA
:103EE000E5F9970700202393072297C00100E78098
:103EF000809817E50100130525A097C00100E78011
:103F00008097B2402945410117C301006700839B98
:103F10004111814617F6FF1F1306464785451705D1
:103F200000200355251506C697D00000E7806006DF
:103F300015C997D501009385256817D5010013058C
:103F4000E5F397C00100E780009317E50100130532
:103F5000A58A97C00100E7800092294597C001001B
:103F6000E780409697D501009385056517D5010038
:103F70001305C5F097C00100E780E08F17E5010049
:103F80001305C58897C00100E780E08E294597C0DA
:103F90000100E780209397F7FF1F9387E741DC47F5
:103FA000054797D50100938525612390E70017D534
:103FB00001001305A5EC97C00100E780C08B17E551
:103FC00001001305E58597C00100E780C08AB24073
:103FD0002945410117C301006700C38E411122C466
:103FE00097D501009385C55F2A8417D50100130575
:103FF000E5E806C697C00100E780E0874C4017D58A
:1040000001001305E57C97C00100E780C0862945C3
:1040100097C00100E780008B034704009307F00F6F
:10402000631FF70297D501009385855B17D50100C3
:104030001305C5E497C00100E780E0834C4017D525
:1040400001001305E57997C00100E780C082224492
:10405000B2402945410117C301006700A386B24061
:10406000224441018280411122C426C22A84AE84A6
:1040700017D50100130585E097D5010093850552FA
:1040800006C697B00100E780007F17E50100130521
:10409000258597B00100E780007E294597C0010083
:1040A000E780408297D501009385454F9707002010
:1040B000239287FC17D50100130545DC05449707BB
:1040C0000020239797FA97070020239487FA9717E1
:1040D00000202398976497B00100E780C079971576
:1040E000002083D5056417D501001305E57F97B03F
:1040F0000100E7804078294597B00100E780807C87
:1041000097170020238C875097F7FF1F9387C72AA4
:10411000DC4717F5FF1F0345E57403D70700C167A8
:10412000FD17631EF700B7E7040003A38705130616
:10413000000A85452244B240924441010283B7E718
:10414000040003A387051306001493050010DDB7D0
:10415000B1C1411122C417D50100130525D22E8407
:1041600097D501009385C54206C697B00100E78048
:104170008070A28517D501001305C57597B00100A1
:10418000E780606F2244B2402945410117B3010026
:10419000670043738280B7E70400FC471171A2DD1A
:1041A000CAD986DFA6DBCED72E8432892E86AA8591
:1041B00017050020130505F782971707002013073E
:1041C00067F683470700930680029387E70793F714
:1041D000F70FE3ECF610BA898A0717D70100130727
:1041E00027D3BA979C43BA9782878D4797D501000A
:1041F0009385854417D50100130545C8630FF40066
:1042000097B00100E780206717D5010013058501ED
:1042100097B00100E7802066BDA497B00100E78059
:10422000806517D501001305650197B00100E7808F
:104230008064294597B00100E780C068930720F8A3
:104240001146970500209385E5ED4A851707002064
:10425000230AF7EC97070020A38707EC97000000DC
:10426000E780A0BC2A841DC997D501009385C53C71
:1042700017D50100130585C097B00100E780A05F46
:10428000A28517D50100130525FF97B00100E7802F
:10429000805E294597B00100E780C06297D5010094
:1042A0009385853917D50100130545BD97B00100E9
:1042B000E780605C17D50100130545FD97B001004C
:1042C000E780605B294597B00100E780A05F41650A
:1042D000930730FA0546970500209385A5E47D15E0
:1042E000170700202300F7E497000000E780E0B301
:1042F0002A841DC997D501009385053417D501007F
:104300001305C5B797B00100E780E056A28517D521
:104310000100130565F697B00100E780C0552945F7
:1043200097B00100E780005AB7E70400BC4F05666C
:10433000130606C8A14517F5FF1F0345A55282972E
:10434000FE506E54DE544E59BE5911618280914721
:104350006303F40297D501009385052E17D501005C
:104360001305C5B197B00100E780E05017D50100F3
:10437000130505F571BDB7E70400FC4F914517F52E
:10438000FF1F0345254E829797D501009385C52AC7
:1043900017D50100130585AE97B00100E780A04D49
:1043A00017D50100130585F397B00100E780A04CF5
:1043B000294597B00100E780E05097500000E78062
:1043C0004072914535A485476303F40297D50100F7
:1043D0009385852617D50100130545AA97B00100DE
:1043E000E780604917D501001305C5F015B597079B
:1043F0000020239127CBB7E704000566BC4F1306C6
:1044000006C8C1450DBF8D476303F40297D501006F
:104410009385852217D50100130545A697B00100A5
:10442000E780604517D50100130585EED5B39307E6
:1044300040F81146970500209385C5CE4A85170799
:1044400000202301F7CE97070020A38E07CC97000A
:104450000000E780809D2A84E30405EE97D50100E3
:104460009385851D17D50100130545A197B001005F
:10447000E7806040A28517D501001305E5DF97B0FE
:104480000100E780403F294597B00100E780804365
:1044900045BD9147E31CF4F6B7E70400FC4F9305D4
:1044A000000217F5FF1F0345E53B829797D50100F2
:1044B0009385851817D501001305459C97B0010019
:1044C000E780603B17D50100130505E6F1BD89477C
:1044D00063E3870297D501009385051617D5010080
:1044E0001305C59997B00100E780E03817D50100A2
:1044F0001305C5E431BB9704002083C4C4C29707E9
:10450000002083C737C297D501009385E512A20426
:1045100017D5010013058596DD8C97B00100E78063
:104520008035A28517D50100130585E297B00100FB
:10453000E7806034C204294597B00100E7808038E5
:10454000C1849305D4FF93960401C1824A8693F5F2
:10455000F50F17050020130515BD97400000E780F3
:10456000E09CE35F90DC930750F817070020230BD3
:10457000F7BA83C73900228697050020938585BA4C
:1045800085074A8517070020A30FF7B8970000009A
:10459000E780A0892A84E30505DA97D50100938591
:1045A000A50917D501001305658D97B00100E780B7
:1045B000802CA28517D501001305C530C9B58947E0
:1045C00063E3870297D501009385050717D501009E
:1045D0001305C58A97B00100E780E02917D50100CF
:1045E0001305C5D835B197500000E780804FA285EC
:1045F00017050020130505B397600000E7806000F1
:1046000081B38D476303F40297D501009385C502FA
:1046100017D501001305858697B00100E780A02516
:1046200017D50100130545D6E5B6B7660200014669
:10463000B7750200054597E0FF1FE780801A9307D2
:1046400060F817070020230FF7AC97070020A38C12
:1046500007AC93070006170700202307F7AC89472C
:1046600017070020A302F7AC97070020238F07AAA3
:1046700097070020A38B07AAC1471707002023072D
:10468000F7AA930720F917070020A301F7AA3146DC
:1046900097070020A38DA7A897050020938585A8DC
:1046A0004A8597070020238407A897F0FFFFE7803B
:1046B000C0772A84E30605C897D501009385C5F71E
:1046C00017C501001305857B97B00100E780A01A8C
:1046D000A28517D501001305A5CC55B3B1476303D7
:1046E000F40297D50100938525F517C50100130540
:1046F000E57897B00100E780001817D50100130591
:10470000E5CB39B6B7E70400FC4F9305000417F575
:10471000FF1F03452515829797500000E780603CF6
:10472000B145F9B5914763E3870297D501009385B9
:10473000A5F017C501001305657497B00100E78067
:10474000801317D50100130525C9D9B4970400209B
:1047500083C4849D9707002083C7F79CA204DD8C47
:104760008E04B77702006D14BE942286A68517D5F5
:1047700001001305A5C797B00100E780C00FB7E798
:104780000400FC472286970500209385F5992800B0
:10479000829793160401C1823000A685094597E0EF
:1047A000FF1FE78000042A8409C917D501001305FB
:1047B000A5C597B00100E780E023930770F819467C
:1047C00097050020938505964A8517070020230B3F
:1047D000F79497070020A389879497F0FFFFE7805D
:1047E000C0642A84E30E05B497D501009385C5E41F
:1047F00017C501001305856897B00100E780A00781
:10480000A28517D50100130525C195B99947630BFA
:10481000F41297D50100938525E217C50100130511
:10482000E56597B00100E780000517D50100130585
:1048300025C0F9BA914763E3870297D501009385B4
:10484000A5DF17C501001305656397B00100E78078
:10485000800217D50100130525BF5DBA970400201B
:1048600083C4848C9707002083C7F78BA204DD8C58
:104870008E04B77702006D14BE942286A68517D5E4
:1048800001001305A5BD97B00100E780C0FEB7E7A2
:104890000400FC472286970500209385F5882800B0
:1048A000829793160401C1823000A6850D4597E0DA
:1048B000FF1FE78000F32A8409C917D501001305FB
:1048C000A5BB97B00100E780E012930780F8194676
:1048D00097050020938505854A8517070020230347
:1048E000F78497070020A381878497F0FFFFE78074
:1048F000C0532A84E30605A497D501009385C5D348
:1049000017C501001305855797B00100E780A0F691
:10491000A28517D50100130565B795B699476303BE
:10492000F40297D50100938525D117C50100130521
:10493000E55497B00100E78000F417D50100130596
:1049400065B6F9B0B7E70400FC4F9305000417F50E
:10495000FF1F034525F1829797500000E7806018FC
:10496000994579B18D476303F40297D5010093858A
:10497000A5CC17C501001305655097B00100E7806D
:1049800080EF17D50100130565B359B017D50100A5
:104990001305C5B397B00100E780C0051305C01229
:1049A00097E0FF1FE780E099014597E0FFFFE78070
:1049B000A06E0D4597100000E7806040294597E004
:1049C000FF1FE780009897E0FF1FE78060888DBA9F
:1049D00099476303F40297D501009385E5C517C590
:1049E00001001305A54997B00100E780C0E817D57D
:1049F0000100130565AE29B817F7FF1F0347D772EB
:104A000097F7FF1F83C7477222075D8F9166BA969B
:104A1000C2061166C1821306F6EF8D476365D602A2
:104A200097F7FF1F938747999C4B17F6FF1F034685
:104A3000966F9386C7002DC203D6070069CA8907FF
:104A4000E39CD7FE89471307A0F8114697F5FF1F8F
:104A50009385456D4A8597F6FF1F2385E66C17F70A
:104A6000FF1FA302F76C97F0FFFFE780003C2A844A
:104A7000E308058C97D50100938505BC17C5010097
:104A80001305C53F97B00100E780E0DEA28517D58A
:104A900001001305A5A5E5B203D60700630EE60ADB
:104AA0008907E39BF6FE8D4779BF91476304F402C3
:104AB00097D50100938545B817C501001305053C3E
:104AC00097B00100E78020DB17D50100130585A30F
:104AD0006FF00FF4B7E70400FC4F9305000817F5DB
:104AE000FF1F034525D88297C9B897D50100938544
:104AF000A5B417C501001305653897B00100E7801C
:104B000080D717D50100130565A16FF06FF02390D2
:104B1000E70017F5FF1F1305258A97400100E7807E
:104B2000000297D50100938525B117C50100130533
:104B3000E53497B00100E78000D417D501001305D4
:104B4000E59E97B00100E78000D3294597B00100AA
:104B5000E78040D78147C5BD2390070017F5FF1FA9
:104B60001305858597400100E78060FD97D501001A
:104B7000938585AC17C501001305453097B001003A
:104B8000E78060CF17D501001305C59B5DBF0111FC
:104B900022CC06CE26CA4AC8834705002A849DC770
:104BA00097D50100938505A517C501001305052DAF
:104BB00097B00100E78020CC4C4017D501001305C9
:104BC000A5D797B00100E78000CB21A25841B707D5
:104BD000CF009387777D631DF70A0359C50085478A
:104BE00004450356E50063FA270903C7040083C59B
:104BF0001400F17693178700CD8FC207C187938683
:104C0000C6556393D70297300000E78020EE630417
:104C100005106244F240CA8526854249D2440561A6
:104C200017330000670023ED954763F827059307C6
:104C300030056314F704930750046390F50483C6AA
:104C4000240093071004639AF60283C73400639626
:104C5000E70203C744009307B0046310F70203C7D9
:104C6000540093079005631AF700CA85268532C65B
:104C700097300000E78020E832466244F240CA855F
:104C800026854249D244056117F3FFFF6700E350D0
:104C9000B707CC009387777D6317F70497D501009A
:104CA0009385459517C501001305451D97B0010073
:104CB000E78060BC1C448356E4008355C40003C6EF
:104CC000070017D501001305A5C897B00100E780BC
:104CD00080BA6244F240D24442492945056117B383
:104CE0000100670023BEB707CE009387777D63047A
:104CF000F70297D501009385E58F17C501001305CD
:104D0000E51797B00100E78000B74C4017D50100C8
:104D1000130545B87DB5F2406244D244424905616D
:104D20008280B7E70400FC4741112E8606C622C4E4
:104D300026C24AC02E842A89AA8517F5FF1F1305AB
:104D4000653E829797D501009385C59017C50100F0
:104D50001305C51297B00100E780E0B197F5FF1F7A
:104D600083C5453C17C501001305C53697B0010042
:104D7000E78060B0294597B00100E780A0B497F4C0
:104D8000FF1F9384243A83C7040041479387070693
:104D900093F7F70F6369F75A17C7010013078721C5
:104DA0008A07BA979C43BA9782879D476307F402A4
:104DB00097D501009385058A17C501001305050CD9
:104DC00097B00100E78020AB17C50100130505313E
:104DD00097B00100E78020AAA1AC97F7FF1F83C717
:104DE0007734DDCB17F7FF1F0347F73397F7FF1F24
:104DF00083C7673322075D8F97F7FF1F83C7C732CB
:104E0000C2075D8F97F7FF1F83C71732E207D98F5D
:104E100017F7FF1F232EF72E83C7640097D50100D5
:104E20009385458317C501001305450517F7FF1F37
:104E3000230FF72C97B00100E780E0A397F7FF1F3F
:104E40009387072D8C4317F6FF1F0346462C17C583
:104E500001001305652A97B00100E780C0A129452C
:104E600097B00100E78000A697F7FF1FA38C072AE1
:104E70002244B24092440249930700F817F7FF1FFB
:104E80002302F72A9D4517F5FF1F1305A5294101A8
:104E9000175300006700E37697700000E780A04694
:104EA00097F7FF1F2381A7289357850017F7FF1F48
:104EB000A30BF726935705012A8417F7FF1F230535
:104EC000F72693578501014517F7FF1FA30EF72417
:104ED00097700000E780804797F7FF1F2387A7247C
:104EE00097C501009385057717C50100130505F9DE
:104EF00097B00100E780209817F6FF1F0346E622CF
:104F0000A28517C501001305A520B1B7CD476303DE
:104F1000F40297C501009385E57317C501001305D9
:104F2000E5F597B00100E780009517C5010013056E
:104F3000A51F79BD97F7FF1F83C7E71FA20717F7C4
:104F4000FF1F0347371FD98FC207C1876357F0027E
:104F500017F7FF1F231CF71AB7E7040003A3870501
:104F60001306000A89452244B2409244024917F5CB
:104F7000FF1F0345258F41010283D147D1BF8D47D4
:104F80006303F40297C501009385C56C17C5010042
:104F90001305C5EE97B00100E780E08D17C501004D
:104FA0001305452835B517F4FF1F0344C41797F7B9
:104FB000FF1F83C7371797C501009385A569220492
:104FC00017C50100130585EB5D8C97B00100E780E4
:104FD000808AA28517C501001305851697B00100C8
:104FE000E7806089294597B00100E780A08D0D46D4
:104FF00097F5FF1F93850513228597F0FFFFE78044
:10500000C0E2AA8421C197C501009385A56417C594
:1050100001001305A5E697B00100E780C085A685CD
:1050200017C501001305051397B00100E780A084A0
:105030002244B240924402492945410117B301007C
:105040006700438897F7FF1F23968704B7E704009C
:10505000116603A38705130606E8914529B78D4716
:105060006303F40297C501009385C55E17C501006F
:105070001305C5E097A00100E780E07F17C5010098
:1050800013050529B1B317F4FF1F0344C40997F7AB
:10509000FF1F83C7370997C501009385A55B2204CD
:1050A00017C50100130585DD5D8C97A00100E78021
:1050B000807CA28517C501001305050B97A0010090
:1050C000E780607B294597A00100E780A07F0D461F
:1050D00097F5FF1F93850505228597F0FFFFE78071
:1050E000C0D4AA841DC197C501009385A55617C5D4
:1050F00001001305A5D897A00100E780C077A68519
:1051000017C501001305850705B797F7FF1F2395FE
:1051100087F6B7E70400116603A38705130606E8C0
:105120009305000289B5894763E3870297C50100AB
:105130009385455217C50100130545D497A001007A
:10514000E780607317C501001305451F51B197F43F
:10515000FF1F83C444FD97F7FF1F83C7B7FC97C5A4
:1051600001009385254FA20417C50100130505D141
:10517000DD8C97A00100E7800070A68517C50100AF
:105180001305450197A00100E780E06E294597A02F
:105190000100E7802073228697F5FF1F938585F82D
:1051A000268597F0FFFFE78040C82A84630E051A22
:1051B00097C501009385054A17C50100130505CC65
:1051C00097A00100E780206BA28517C50100130599
:1051D000A5FD99BD854763F98718834519002244C9
:1051E000B24092440249B335B00097F7FF1F238DB8
:1051F000B7EA17C50100130565FC410117A30100BB
:1052000067006367A2852244B24092444A850249FE
:105210004101171300006700C3C099476303F402FC
:1052200097C501009385054317C50100130505C502
:1052300097A00100E780206417C501001305C52968
:1052400041BE17F4FF1F034404EE97F7FF1F83C707
:1052500077ED97C501009385E53F220417C501004E
:105260001305C5C15D8C97A00100E780C060A285D1
:1052700017C50100130505F697A00100E780A05FA0
:10528000294597A00100E780E063194697F5FF1FC5
:10529000938545E9228597F0FFFFE78000B9AA844E
:1052A0001DC197C501009385E53A17C50100130597
:1052B000E5BC97A00100E780005CA68517C501004A
:1052C000130545F295B397F7FF1F239587E4B7E7DA
:1052D0000400116603A38705130606E8930500087A
:1052E00059B1854797C501009385C53617C501009B
:1052F0001305C5B8630BF40097A00100E780A05721
:1053000017C50100130545EFE1B497A00100E78040
:10531000805617C501001305A5EF97A00100E7808F
:105320008055294597A00100E780C0592244B2402A
:105330009244024997F7FF1F239A07DC4101177334
:1053400000006700C3EC97C501009385A53017C521
:1053500001001305A5B297A00100E780C05117C551
:1053600001001305A51BADB4B2402244924402498A
:1053700041018280411106C622C426C239C12A8455
:1053800097F00000E7806075AA8411EDB7E704008C
:10539000BC474146814522858297B24022442685FA
:1053A00092444101828041657D1597F00000E780BD
:1053B000A073B7E7040001E9BC4741468145228557
:1053C00082978144D9BF0347E501FC4793059008C4
:1053D00019E393050003AA954146228582978544E7
:1053E0006DBF411106C622C426C24AC097F0000014
:1053F000E780A06E55CD97700000E78080F12A8489
:1054000097100000E7806050AA842285637394009F
:105410002685B7D7B0009387F75E63F3A702B7E797
:10542000B000130514009387F74F63E3A7082244E5
:10543000B24092440249410117730000670023EE15
:105440008567938707F13E956364A4003305F400F4
:1054500097700000E780A0EC97700000E78060EB99
:105460002A8963F6A40097100000E780C04C97C516
:1054700001009385A51F17C50100130525A097A05E
:105480000100E780403FA6864A86A28517C5010035
:10549000130585B697A00100E780E03D2244B240A5
:1054A000924402492945410117A301006700834145
:1054B000B24022449244024941018280011122CC2F
:1054C00037E404005C5C06CE354697C50100938541
:1054D000252317D501001305250B829711E917C560
:1054E00001001305659F97A00100E780A05001A06F
:1054F00097E7FF1F9387C7373EC4B7F50700856757
:1055000093870780814617E6FF1F1306E635E105FE
:1055100019453EC697D0FF1FE780A02C7C44194652
:1055200097E5FF1F9385453417F5FF1F1305C5B693
:105530008297340017E6FF1F1306063397C5010054
:105540009385856417C50100130585659770000074
:10555000E78000912A841DCD97C501009385850BB6
:1055600017C501001305859197A00100E780A030C1
:10557000A28517C501001305A51997A00100E780B2
:10558000802F294597A00100E780C033F240624494
:105590000561828097E00000E780E0FA17C501000E
:1055A0001305050E97600000E780408597A0000076
:1055B000E780204F97600100E780A0B317E5FF1F49
:1055C000130505DC97600100E780409C17C50100CA
:1055D0001305050C97600100E78020B42A849760CA
:1055E0000000E78080EB97100100E780808B9780B8
:1055F0000100E780A02497700000E780404B97608F
:105600000000E780806197300100E780E04C97C59B
:1056100001009385250017C501001305258619C8CB
:1056200097A00100E7802025A28517C5010013057A
:105630006510A1B797A00100E780E02317C501001E
:105640001305851197A00100E780E022294597A066
:105650000100E780202797300100E780C02897F0FD
:105660000000E780804769CD97E7FF1F938747C415
:1056700083D707008545370504001707002023124C
:10568000F70A97300000E780A08697C50100938550
:1056900065F817B501001305657E97A00100E78046
:1056A000801D17C501001305A50C97A00100E78018
:1056B000801C294597A00100E780C0208547170777
:1056C0000020230DF7F497E7FF1F9387E7CEDC4711
:1056D00003D70700C167FD176316F70097F0FFFFB8
:1056E000E780408397000000E780E0CF971000003C
:1056F000E780C0F5170500200355A502975000006C
:10570000E780A0C5054597500000E78080F89750D6
:105710000000E780001E97C501009385A5EF17B52F
:1057200001001305A57597A00100E780C01417C5F7
:1057300001001305A50897A00100E780C01391B5EB
:1057400097C50100938505ED17B501001305057395
:1057500097F7FF1F239C079A97A00100E780A011ED
:1057600097C501009385055E17C5010013058502E5
:1057700097A00100E7802010294597A00100E7804D
:105780006014014597500000E780A0F069B741110F
:1057900022C437E404008327041A06C68297975070
:1057A0000000E78040BF83270408170500001305A9
:1057B0000503829797E7FF1F2386A70A17E5FF1FB8
:1057C000130585BF97400000E78060682244B2401F
:1057D0004101170300006700A3CE011122CC06CEC1
:1057E00026CA4AC84EC693F715002E84B5CB97E05B
:1057F000FFFFE7802072930710F817F7FF1F2303BE
:10580000F79297F7FF1F83D7A78617F7FF1FA30B02
:10581000F7909145A18317F5FF1F1305A59017F782
:10582000FF1F2302F79097F7FF1FA38E078E975055
:105830000000E78000DDB7E70400BC4F130600144A
:105840009305001017E5FF1F0345C5018297134517
:105850001400F2406244D2444249B2490561828058
:1058600093F70510B1C7054597500000E78060E247
:10587000170500200355E5EA97500000E780E0ADEA
:1058800097000000E78020B697100000E78000DC5A
:1058900097F7FF1F83C7579889E797500000E78065
:1058A000800397500000E780C0041345041055B7EB
:1058B00093F72500E9CF17F7FF1F0357278569C71F
:1058C000AD64B71900409384A4AA23A0990097F669
:1058D000FF1F9386E683944297C701009387C7030F
:1058E00017F6FF1F0346A682814517C50100130561
:1058F000A50397700000E780A08123A0990097E797
:10590000FF1F239FA79A2A8941C197C5010093854C
:1059100065D117B501001305655697A00100E78012
:1059200080F5CA8517B501001305C56F97A0010062
:10593000E78060F4294597A00100E780A0F897E789
:10594000FF1F2395077C930710F817E7FF1F230B12
:10595000F77C97E7FF1F83D7A77117E7FF1FA30304
:10596000F77CA18317E7FF1F230FF77A91458D4737
:1059700017E5FF1F1305057B17E7FF1FA305F77A40
:1059800097500000E780E0C713452400D9B593F78E
:105990004500D1C397C501009385C5C817B501005F
:1059A0001305C54D97A00100E780E0EC17B5010095
:1059B0001305056997A00100E780E0EB294597A052
:1059C0000100E78020F0930720F817E7FF1F230B63
:1059D000F77497E7FF1F83D7E76B17E7FF1FA30352
:1059E000F774A18317E7FF1F230FF772854717E7A7
:1059F000FF1FA30AF77297400000E780800E17E5AB
:105A0000FF1F13052572914597500000E78060BF86
:105A1000134544003DBD93F78500A9C797C5010014
:105A2000938545C017B501001305454597A00100B2
:105A3000E78060E417B501001305C56197A0010078
:105A4000E78060E3294597A00100E780A0E797E79A
:105A5000FF1F239D076A97600000E780407B134586
:105A60008400C5BB93F70501D1C3854517E5FF1F2A
:105A70000355456297500100E780E03497C5010067
:105A8000938545BA17B501001305453F97A001005E
:105A9000E78060DE17B501001305055D97A00100E2
:105AA000E78060DD294597A00100E780A0E193072A
:105AB00030F817E7FF1F2307F76697E7FF1F83D725
:105AC000675D17E7FF1FA30FF76417E5FF1F1305B7
:105AD0006565A1838D4517E7FF1F2306F76497507F
:105AE0000000E78000B213450401A5B393F7050257
:105AF000D1C797C501009385E5B217B5010013051D
:105B0000E53797A00100E78000D717B5010013051E
:105B1000E55797A00100E78000D6294597A001002E
:105B2000E78040DA930740F817E7FF1F230CF75E82
:105B300097E7FF1F83D7475417E7FF1FA304F75EBC
:105B4000A18317E7FF1F2300F75E854717E7FF1FB5
:105B5000A30BF75C97E7FF1F2390075297400000C5
:105B6000E78020F817E5FF1F1305C55B91459750A7
:105B70000000E78000A913450402E1B993F705048A
:105B8000FDC397C501009385E5A917B5010013056D
:105B9000E52E97A00100E78000CE17B501001305A0
:105BA000655097A00100E78000CD294597A001002E
:105BB000E78040D197E7FF1F83C7C7561307700AD6
:105BC0006386E7061307800A638CE7081307600AF9
:105BD0006393E704930760F817E7FF1F2304F75464
:105BE00097E7FF1F83D7675217E7FF1FA30CF752F2
:105BF000A18317E7FF1F2308F752854717E7FF1F09
:105C0000A307F752B14517E5FF1F1305A55197509C
:105C10000000E780009F97400000E78080EC13457C
:105C2000040497E7FF1F2392074E25B1930770F8EE
:105C300017E7FF1F2308F74E97E7FF1F83D7E74CAF
:105C400017E7FF1FA300F74EA18317E7FF1F230CE1
:105C5000F74C854717E7FF1FA308F74C994565B731
:105C6000930780F8F1B793F705080145E38307BE72
:105C700097C501009385059B17B501001305052005
:105C800097A00100E78020BF17B501001305054369
:105C900097A00100E78020BE294597A00100E7807A
:105CA00060C29307A0F817E7FF1F230DF74697E799
:105CB000FF1F83D7274617E7FF1FA305F746A183DA
:105CC00017E7FF1F2301F746854717E7FF1FA30CC0
:105CD000F74497E7FF1F239F074297400000E780A4
:105CE00040E017E5FF1F1305E5439145975000007D
:105CF000E780209113450408A9BE1307F5FF7571CD
:105D00004207C16706C722C526C34AC14183F517AA
:105D100063EFE700854597500100E780C00A85449E
:105D2000BA402A4426850A499A4449618280B7E7E5
:105D30000400BC471306000881450A8582970A853E
:105D400097600000E78080620A841309010881449B
:105D50000355040009C98545850497500100E78073
:105D6000800693F4F40F2104E31489FE55BF41111A
:105D700006C697E0FFFFE78020040DC197E7FF1FED
:105D800083D7A732850717E7FF1F2310F73297E75E
:105D9000FF1F239DA730B2404101828097E7FF1F7C
:105DA00083D7E730850717E7FF1F2312F730E5B7E2
:105DB0008546170300006700C3FB411122C49146CA
:105DC0002A8417E6FF1F1306E6439D652D4506C688
:105DD00097D0FF1FE780E0A0B7F7070003C70701D0
:105DE000A5476313F70001A09306001001469D65C7
:105DF000254597D0FF1FE780C09E97E7FF1F2383AD
:105E000087402244B240914617E6FF1F1306863FA3
:105E10009D652945410117D3FF1F6700839C1171C0
:105E2000CED7B7E9040083A7C904CAD917E9FF1F71
:105E30001309492FA2DD2E8686DFA6DB2E84AA85D4
:105E40004A85829797E7FF1F83C7C72D1307700AFC
:105E50006385E710636DF7001307600A6385E70445
:105E6000FE506E54DE544E59BE59116182801307A4
:105E7000800A6385E7161307900AE393E7FE8D47D0
:105E80006306F41C97C50100938505B817B501009A
:105E90001305C5FE97A00100E780E09D17C501002E
:105EA0001305C5B325A08D47630CF40297C5010007
:105EB000938585B517B50100130545FC97A0010032
:105EC000E780609B17C50100130585AA97A0010014
:105ED000E780609A294597A00100E780A09E49B716
:105EE000854717C50100130565AA17E7FF1F230D96
:105EF000F71A97A00100E780E0AFB7750200B76618
:105F000002000146054597D0FF1FE780808D93076B
:105F100060F817E7FF1F2307F72097E7FF1FA38409
:105F200007209307002617E7FF1F232FF71EE577AB
:105F30009387072117E7FF1F231AF71EB14597E73D
:105F4000FF1F2386071E97E7FF1FA382A71E4A8510
:105F500097000000E780E01621B7914763E38702CE
:105F600097C50100938545AA17B50100130505F1F2
:105F700097A00100E780209017C50100130505A335
:105F8000B1B797E4FF1F83C4241A97E7FF1F83C7A5
:105F90009719A204DD8C83A7C9046D14228697E5A6
:105FA000FF1F93857518280082978E0493160401AD
:105FB000B7750200C1823000A695094597D0FF1F32
:105FC000E7802082930770F817E7FF1F230CF71470
:105FD000994597E7FF1FA389A71495BF914763E3EE
:105FE000870297C50100938525A217B50100130507
:105FF000E5E897A00100E780008817C501001305B8
:10600000659CE9B597E4FF1F83C4041297E7FF1F5F
:1060100083C77711A204DD8C83A7C9046D1422867F
:1060200097E5FF1F93855510280082978E049316DD
:106030000401B7750200C1823000A6950D4597C0D6
:10604000FF1FE780007A930780F8BDBF17C50100E6
:106050001305059A97A00100E780C099930790F86F
:106060002304F100834719008D452800A304F100A3
:10607000834729002305F10097000000E7806004B2
:106080001305C01297C0FF1FE780A02B014597D0D2
:10609000FFFFE78060000D4597000000E78020D2F9
:1060A000294597C0FF1FE780C02997C0FF1FE780E1
:1060B000201A7DB397E7FF1F23AEA714828097E7CE
:1060C000FF1F9387271503A30700630303000283C1
:1060D000174300006700E35241114AC097F6FF1FC3
:1060E00083D62664328917D6FF1F0356062F22C493
:1060F00026C206C62A84AE8497000000E780406C62
:1061000029C921C8994763F69704834714000347B8
:106110000400A207D98F13978700A183D98FC207E4
:106120003167C1831307C7556395E70297D7FF1FF0
:1061300083D7A72AA301F400A1832302F40097F7D1
:10614000FF1F83D7075E91C7A302F400A183230337
:10615000F400630D090297F7FF1F83C7274C9DE7E3
:1061600097E7FF1F83C7470B95C38DC097E7FF1FB6
:1061700083C787F381EF22852244B2400249A68576
:1061800092444101174300006700A347B2402244F4
:1061900092440249410182801DCD95472A870145DD
:1061A00063FDB70297F7FF1F83C747479DC7834724
:1061B000570083464700A207D58F85C341112E861D
:1061C0003E85BA8506C697000000E780A0BEB240B3
:1061D00005454101828001458280828097B7010098
:1061E000938747BA9C4301116800914506CE3EC68D
:1061F00097000000E780E0ECF240056182808D4767
:1062000063F6B708011126CA06CE22CC0344350036
:1062100097E4FF1F83C4540097C5010093858580D0
:10622000B337800017E7FF1FA308F7FE09C497B52F
:1062300001009385E57F17B501001305E57F979071
:106240000100E780406397E7FF1F83C7F7FC638681
:10625000970097000000E780C04697400000E78065
:1062600040699967938757EE2316F10068008547C8
:106270009145A30781002307F10097000000E78004
:1062800040E4F2406244D2440561828082808947C2
:1062900063F7B708011122CC06CE26CA8344250035
:1062A00085472A84639DF404914763F5B704034549
:1062B00045008347340022055D8D97D7FF1F239E3D
:1062C000A71097000000E78080589967938767EED2
:1062D0002314F1008347340023059100A305F10046
:1062E00083474400954528002306F10097000000ED
:1062F000E78020DDF2406244D24405618280FDF8EF
:106300009967938767EE2314F10097D7FF1F83D710
:10631000C70CA305F10023050100A183E1B782802A
:106320000111996722CCD51717F4FF1F1304042F0E
:106330002314F1008347040026CA97F4FF1F9384B7
:10634000443E2305F10083D7040028009545A305AA
:10635000F100A18306CE2306F10097000000E7803C
:1063600040D603D604008345040017B50100130589
:10637000A56D97900100E7800050F2406244D2443E
:10638000056182809D677971D9172316F10097F70F
:10639000FF1F9387A72883C707001305F10006D6C0
:1063A0002307F10097F0FFFFE78000FD09E9B7E759
:1063B0000400BC47414681451305F10082976800FF
:1063C000CD4597000000E780C0CF97F5FF1F83C53C
:1063D000E52417B501001305256A97900100E780B1
:1063E0008049B25045618280630C0516011126CAAE
:1063F00006CE22CC4AC84EC697E7FF1F83C7D7E117
:1064000097F4FF1F83C4842199C393E424002A8452
:1064100097100000E780806D93E9C40119E193E9CA
:10642000C40037E90400832789042285130620036A
:1064300081458297930750FA2300F4009307A00543
:10644000A300F4008D472301F4009147A301F40059
:106450009307F005A302F40097F7FF1F83D7672C7B
:106460002304F400A183A304F40097D7FF1F83D76C
:10647000C7F62305F4009304C400A183230204009B
:1064800023033401A305F400268597F0FFFFE7807E
:10649000A0EE19E583278904414681452685829728
:1064A00097D7FF1F83D707F1230EF400A183A30E14
:1064B000F40093070002230FF400930710FAA30FD0
:1064C000F4009D472300F402A3000402B7E7040090
:1064D000FC4713052402194697D5FF1F9385C5383D
:1064E000829797E7FF1F83D787BC2304F402A18319
:1064F000A304F40297E7FF1F83D727BB2305F40209
:10650000A183A305F40297E7FF1F938727BA839718
:1065100007002285930500032306F402C207C18306
:10652000A183A306F40297D7FF1F938767D98397A8
:1065300007002307F402C207C183A183A307F40263
:1065400097000000E780C0232308A4022181A3084C
:10655000A402F2406244D2444249B24905618280B9
:1065600082805D71E17793C777FF1305E10086C6EE
:106570002316F10097000000E78040E768009305CC
:10658000400397000000E780C0B3B640616182809D
:106590005DC9411122C426C206C6930750FA2300E2
:1065A000F5009307A005A300F50089472301F50036
:1065B0009147A301F5009307F005A302F50097F7B3
:1065C000FF1F9387A70583C707009304C5002A848C
:1065D0002303F50097E7FF1F938717C483C70700BE
:1065E00023020500A303F50097F7FF1F83D7671366
:1065F0002304F500A183A304F50097D7FF1F83D7D9
:10660000C7DD2305F500A183A305F500268597F0D6
:10661000FFFFE78060D601E9B7E70400BC474146C9
:106620008145268582972285F14597000000E78005
:106630002015230EA4002181A30EA400B240224401
:1066400092444101828082805D710A8586C6A2C41F
:1066500097000000E78000F437E404007C448A855A
:106660000810794682973C441305E10309468145A9
:106670008297101093050002014597D0FFFFE78035
:10668000E007B640264461618280411122C426C2DF
:106690002A84AE848566AA850146254506C697C02C
:1066A000FF1FE7800014A2852244B2402686924450
:1066B000A1462945410117C3FF1F6700831201113D
:1066C000B7C7A55A22CC9387C73317E4FF1F13041B
:1066D000B4B43EC4834704002C00196506CE3EC600
:1066E00097000000E780A0FA8345040017B5010079
:1066F0001305054397900100E780E017F2406244DC
:10670000056182800111A146300099652D4522CC9A
:1067100006CE97C0FF1FE780C00CA24737C4A55A1A
:106720001304C43363958702B24517B501001305FE
:10673000E536B335B00097E7FF1FA38FB7AC97904E
:106740000100E7804013F240624405618280916558
:10675000A1463000938505F02D4597C0FF1FE780C7
:106760004008A247E38287FC97E7FF1FA38607AA9A
:10677000814517B501001305A534D1B7C167697606
:106780008146FD1705061397060141836364B70030
:106790003E8582803307D50003470700B98F214724
:1067A00013F81700858363050800B18FC207C18302
:1067B0007D171377F70F6DF78506F1B741C5A5472C
:1067C000054763F2B70883471500034705003168A2
:1067D000A207D98F13978700A183D98FC207C183DE
:1067E0001308C855054763900707411106C622C420
:1067F00026C203442500914763F0870493075400A1
:1068000063ECF502A301C50021822302C5009304B5
:10681000340091C6A302D500A1822303D5002A84A7
:10682000A68597000000E780A0F526942300A40029
:106830002181A300A4000147B240224492443A853A
:106840004101828005473A8582800111B7C7A55A68
:1068500022CC9387E7342A842AC62C00156506CEFD
:106860003EC497000000E78080E2A28517B50100D2
:106870001305052D97900100E780E0FF97000000C9
:10688000E780C0DCF2406244056182800111A146CC
:10689000300095652D4522CC06CE97C0FF1FE780BE
:1068A00040F4A24737C4A55A1304E4346395870221
:1068B000B24517B501001305A52297D7FF1F239EE8
:1068C000B7B0C205C18197900100E780C0FAF240DD
:1068D0006244056182809165A1463000938505EE92
:1068E0002D4597C0FF1FE780C0EFA247E38287FCDA
:1068F000D14717D7FF1F2312F7AED14517B50100B7
:1069000013050520C9B70111A146300091652D4539
:1069100006CE97C0FF1FE780C0EC2247B7C7A55A35
:106920009387073501456313F7003245F24005614F
:1069300082800111B7C7A55A2AC6938707352C0054
:10694000116506CE3EC497000000E78040D4F240B7
:106950000561828021C1411126C206C622C4AE84CF
:106960008DC52A8497100000E780E01897E7FF1F85
:1069700083C7878A99CB22852244B240A685924458
:106980004101174300006700C3C7B240224492444C
:1069900041018280828001114EC606CE22CC26CAD9
:1069A0004AC893F71500AE899DCBAD6737170040F5
:1069B0009387A7AA1CC3B7E70400BC4F13060019AE
:1069C000854517D5FF1F034525A1829713C51900DB
:1069D000F2406244D2444249B2490561828093F751
:1069E00025000145F5D717F7FF1F035767D39547D4
:1069F00063F9E70C014417F6FF1F130666C29306FE
:106A0000300513055004130810049308B004130351
:106A10009005930764006374F7043A847D5997F4F2
:106A2000FF1F83C4E4BF97F7FF1F83C777BFA2048C
:106A3000DD8CAD679387B755638BF41463E3970AD6
:106A4000A9679387A755638EF414A28517F5FF1FD6
:106A5000130505BD97000000E78000F0E9A0B3072B
:106A6000860083C50700639AD50483C51700639623
:106A7000A50483C527006392050583C53700639E7F
:106A8000D50283C54700639A150383C757006396F1
:106A9000670222890DE897F5FF1F83D565C8B38586
:106AA0002541C20517F5FF1F130585B7C1814A951A
:106AB00097000000E78040EAE1A00504420441801D
:106AC00089BF3A847D598547E3EB87F45DC48545EA
:106AD00017F5FF1F1305C5B497000000E780C0E756
:106AE00069A8B1679387C7556389F404B56793872D
:106AF000D755E39CF4F4A28517F5FF1F130545B2A3
:106B000097400000E780E0AF8947630EF4009305EB
:106B1000E4FFC205C18117F5FF1F130585B097106B
:106B20000000E78040FDA68517B5010013050503A9
:106B300097900100E78020D489A097300000E7807B
:106B4000E09997100000E78060FA11C9A28517F557
:106B5000FF1F1305E5AC97100000E780C0F905465C
:106B6000A28517F5FF1F1305A5AB97F0FFFFE78080
:106B7000E05697300000E7806096FD57E31DF9F07E
:106B800097F7FF1F239E07B813C5290091B5A2856B
:106B900017F5FF1F1305C5A897F0FFFFE7800060FA
:106BA00059B7A28517F5FF1F130585A797F0FFFFBB
:106BB000E78000638DBF411122C437E404005C5CB0
:106BC00006C6354697B50100938585B317C5010004
:106BD0001305859B829711E917B50100130545F947
:106BE00097900100E78000E101A08327041C8297B1
:106BF0002A84054597D00000E780409497700100F3
:106C0000E780601997700100E78060EE97C0000090
:106C1000E780C0A52285B240224441018280411113
:106C2000054506C622C426C297C0FFFFE780A030F4
:106C30001305A00497B0FF1FE78060477575854571
:106C40007D1597C0FFFFE780401A7D7585451305C8
:106C5000F53697C0FFFFE780A02337140040832755
:106C6000840A8D451305002093E707202324F40AA6
:106C700097C0FFFFE7806017B7E4040097C0FFFFED
:106C8000E780805CC85897900100E780A0D617C5C0
:106C900001001305658F97900100E780A0D5832739
:106CA000840C8545414593E707082324F40C97C0DD
:106CB000FFFFE780E01D8D451305000897C0FFFF2B
:106CC000E780001D97C0FFFFE780E04937A5070078
:106CD0001305051297C0FFFFE7808045014597C067
:106CE000FFFFE780A04B95450545894717F7FF1F34
:106CF000230AF7A297C0FFFFE780E04BB7E700E069
:106D000013070006238DE7403707000423A0E71090
:106D100097D0FFFFE78060CD97D0FFFFE78060DF6F
:106D200097000000E78060E997000000E780C09DC1
:106D300097000000E780C0B597F0FFFFE78060A5EF
:106D400097100000E78060DC97000000E78080106B
:106D500083A7040817050000130525C4829797C769
:106D6000FF1F238BA766BC4C1306006485458297E2
:106D700097B0FF1FE780C06701458280AD67371776
:106D800000409387A7AA1CC3B7E700E0370740007D
:106D900023A0E71801000100B7F7070003C70701A8
:106DA000A5476316F7009397450191C301A04111D0
:106DB000AE860146AA85254506C697C0FF1FE78017
:106DC00040A2B240B7E700E03707400023A0E71039
:106DD000410182804111B2862E86AA852D4506C6C4
:106DE00097C0FF1FE780E09FB240014541018280CC
:106DF0009307000463ECC7041D71A2CC2A84080821
:106E0000A6CACAC886CE32C697900100E780409BCA
:106E1000AD67371700409387A7AA1CC3B7E400E00B
:106E20003709400023A0241901000100B2461008D0
:106E3000A285294597C0FF1FE780A09AF6406644C7
:106E400023A02411D6444649256182803955828089
:106E500041110D658D4506C697C0FFFFE780E0F83C
:106E6000B71700408D6623A6D70A17F5FF1F130535
:106E7000A58B1387C70A9387870A1CC15CC58566E3
:106E800089675CC958C114C518C9B7E70400B24086
:106E900003A3871E410102830387060009E763E01D
:106EA000C5022E85828093871500C207C183E3F84F
:106EB000C7FEAA952380E5008506BE85F1BF2E9505
:106EC00023000500F9BF01111C08BA9706CE238ADA
:106ED00007FE5C003E9797B801009388A80613F858
:106EE000F6004698034808007D17918223000701A9
:106EF000E397E7FEBE8697000000E78020FAF240A5
:106F0000056182808146E548B307D50003C70700C5
:106F1000B387D50083C70700A1C31308F7F9137817
:106F2000F80F63E5080101171377F70F1388F7F9D6
:106F30001378F80F63E50801811793F7F70F631FC4
:106F4000F700850693970601C183E3EFC7FAB29570
:106F50008387050093B717003E8582808147EDBF88
:106F60008547814663F1B702034705009307000395
:106F7000631BF700834715001307800593F7F70D90
:106F80006393E700894601470148254E1543914E1A
:106F900089A0B307D50083C70700938807FD93F83E
:106FA000F80F637C1E019388F7FB93F8F80F636872
:106FB0001303938797FC93F8F70F120833681801AF
:106FC000050742081377F70F135808018506630F6A
:106FD000D70193970601C183E3EDB7FA39A09388EF
:106FE000F7F993F8F80F6378130101C7231006012E
:106FF00005473A858280938797FA75BF8145B30725
:10700000B5008387070089E7172300006700A353B3
:107010008505C205C181E5B7411106C6B94763EED2
:10702000B70017B501001305A5BE97000000E78063
:1070300020FDB2400545410182808347E5001307EA
:1070400010036394E702854717F7FF1F2308F782B1
:1070500017B50100130505BE97F7FF1F239F078093
:1070600097E7FF1F23960772C9B713070003E39A38
:10707000E7FA97F7FF1F2383078097E7FF1F239EF9
:10708000077E97E7FF1F2395077017B501001305CB
:10709000E5BB61BF411126C2E97797E4FF1F9384E6
:1070A000247E22C49387A7552E842381B4002E8684
:1070B000AA8517E5FF1F1305E57C06C62390F4009B
:1070C000A381040097800100E780806F930524006E
:1070D000C205C18117E5FF1F1305A57A97F0FFFFD1
:1070E000E780006AB38784002382A7002181A382FE
:1070F000A700930564002244B24026859244C2054D
:10710000C1814101172300006700E34309C99307C8
:10711000000463E6B700170300006700E3F782800E
:10712000011106CE2307010081EE97B60100938678
:1071300026E197000000E78060D6F240056182807A
:1071400058002A88AE883283A9473A85A945254E3A
:1071500033F6B602FD1793F7F70F13060603A304E1
:10716000C70033D6B6026375DE007D17B286EDF335
:10717000B306F5001A86C685428565BF397197B694
:1071800001009386A6D41306001006DE22DC26DA60
:107190002A844AD84ED697000000E78020D0AA85DE
:1071A00097E6FF1F83D6E657114713060010228586
:1071B00097000000E78060D197E7FF1F83C707466D
:1071C000AA8597B601009386E6CD89C797B60100D8
:1071D0009386C6CC13060010228597000000E78036
:1071E000E0CBAA8597B60100938686CE13060010E1
:1071F000228597000000E78060CAAA8597B6010043
:10720000938686CD13060010228597000000E78044
:10721000E0C8AA8591461306001022859700000059
:10722000E78040F0AA8597B601009386E629130609
:107230000010228597000000E78040C6AA8597B617
:1072400001009386E6CF1306001022859700000008
:10725000E780C0C4AA8597B601009386E626130688
:107260000010228597000000E78040C3AA8593069E
:10727000F00513060010228597000000E78080EAE1
:1072800097D7FF1F83C757F9AA8597B60100938642
:10729000E6C189E797B601009386C6C113060010C0
:1072A000228597000000E78060BFAA8597B601009D
:1072B000938606C313060010228597000000E7801E
:1072C000E0BDB7A60700AA85938606121306001034
:1072D000228597000000E780E0E4AA8597B60100C8
:1072E000938686C013060010228597000000E78071
:1072F000E0BA97C7FF1F83C7670EAA8597B601003C
:107300009386C6BB89E797B601009386A6BB130692
:107310000010228597000000E78040B8AA8597B644
:107320000100938626BD13060010228597000000F9
:10733000E780C0B6AA8597B60100938626BC1306DF
:107340000010228597000000E78040B5AA8597B617
:107350000100938626BB13060010228597000000CB
:10736000E780C0B31147AA8597C6FF1F83D686045E
:1073700013060010228597000000E78000B52AC69A
:1073800097500000E780E0F8B245AA8497B6010064
:10739000938686B713060010228597000000E780C9
:1073A000E0AF93D60401AA85094793F6F60F1306BA
:1073B0000010228597000000E78020B19396040119
:1073C0001147AA85C182130600102285970000008C
:1073D000E780A0AFAA8597B60100938666B313062F
:1073E0000010228597000000E78040AB1147AA8576
:1073F00097C6FF1F83D666FE1306001022859700EE
:107400000000E78080ACAA8597B601009386C6B0DD
:1074100013060010228597000000E78020A811477E
:10742000AA8597D6FF1F83D686C81306001022852B
:1074300097000000E78060A9AA8597B601009386AF
:1074400026AE13060010228597000000E78000A5F5
:107450001147AA8597D6FF1F83D626C513060010AD
:10746000228597000000E78040A6AA8597B6010014
:10747000938686AB13060010228597000000E780F4
:10748000E0A11147AA8597D6FF1F83D626C213060F
:107490000010228597000000E78020A3AA8597B6F8
:1074A00001009386A6A8130600102285970000000D
:1074B000E780C09EAA85114797C6FF1F83D646E086
:1074C00013060010228597000000E78000A0AA851F
:1074D00097B60100938606A6130600102285970032
:1074E0000000E780A09BAA85814497C9FF1F93896C
:1074F000A9371949B387340183C607000947130622
:107500000010228597000000E780209C8504AA8552
:10751000E39224FF97B60100938646A2130600105B
:10752000228597000000E78060972AC6080897E048
:10753000FFFFE78060E4B24504081309010283C736
:10754000040083C614001147A207DD8E1306001045
:10755000228597000000E78040978904AA85E31000
:1075600099FEF2506254D2544259B259216182803C
:10757000297137074000232C811223282113232E41
:107580001112232A9112232631132324411323227B
:10759000511317E9FF1F1309A91A0144594625077A
:1075A0006302A45483470900D91793F7F70F63695F
:1075B000F600B357F700858B930619006390071602
:1075C0003304854042044180BD4763EE8714014780
:1075D000630AF416B70640005946A506B307E9004A
:1075E00083C70700131507014181D91793F7F70FD8
:1075F000636FF600B3D7F600858B91CB05070505C1
:10760000931707014205C1834181E3E987FCB30970
:10761000A440C20993D90901A14763FF3727B304E6
:10762000A900254697A501009385456F268597807B
:107630000100E780801663110526A547638EF900D7
:1076400083C7940035476389E70029476386E700CD
:1076500093F7F70D6392072497A601009386C66CF3
:10766000130600048145081097000000E78000839E
:10767000AA8597A601009386666C1306000408107D
:1076800097000000E7808081AA8597A60100938675
:10769000A66B13060004081097000000E780008026
:1076A000AA85914613060004081097000000E780A1
:1076B00060A7AA8597B60100938606E11306000429
:1076C000081097F0FFFFE780607DAA8597B601005C
:1076D0009386068713060004081097F0FFFFE780E3
:1076E000E07BAA8597B60100938606DE13060004A8
:1076F000081097F0FFFFE780607A9306F005130605
:107700000004AA85081097000000E780A0A197A6B2
:107710000100938626D61306000485A805044204BA
:1077200041803689B5BD414697A5010093858554B2
:107730004A8597800100E780400697A6010093865E
:10774000A65405C13D4697A50100938525554A8558
:1077500097800100E78060043DE597A601009386CD
:10776000E654130600108145081097F0FFFFE780EC
:10777000E072AA85081097000000E78060A097A635
:107780000100938626CF13060010AA85081097F0F3
:10779000FFFFE780A070AA85081097200000E7800F
:1077A00080DA85448320C1130324811326850329AD
:1077B0000113832441138329C112032A8112832ACE
:1077C000411231618280C14763F6870C454697A517
:1077D00001009385E54E4A8597800100E780E0FB34
:1077E0000147E31905DEFD572314F100C54497AAAC
:1077F0000100938A2A4E9389540093970901139AA2
:107800000401C183135A0A0163FA870233852401F4
:107810001546D68597F0FFFFE780006F850461DD90
:107820009305B4FFB3854541C2053000C1813305DE
:10783000390197F0FFFFE780E07221C50355810011
:1078400097E0FFFFE780A04B2A8497A6010093866C
:10785000E648130680028145081097F0FFFFE78095
:10786000E063AA85A2861306800208109700000034
:10787000E780408B97A601009386C6BF130680025F
:1078800029B717A501001305E54697F0FFFFE7802C
:10789000207701BF01473DBBB5478144E3F487F042
:1078A000394697A501009385A54A4A85978001002E
:1078B000E780A0EE09E9A2854A8597F0FFFFE780FF
:1078C000E075AA84C5B5394697A501009385454959
:1078D0004A8597800100E78040EC6315051A9307FD
:1078E00024FFC20723130100C1830D476373F70A06
:1078F0009304E900114697A501009385A5362685D6
:1079000097F0FFFFE78040602DC139144204490918
:10791000418097A901009389E934814497AA010025
:10792000938A4A3B138A5400637C8A021546D685A3
:107930003305990097F0FFFFE780005D2DC56D14BA
:10794000B3059440C20513066100C18133054901A6
:1079500097F0FFFFE780006131C183576100B1EB11
:1079600017A50100130505430DB7114697A50100A2
:107970009385C52F268597F0FFFFE780E05811C952
:10798000391442044909418097A901009389092EBD
:1079900069B717A501001305A53DC5BD17A50100D1
:1079A00013054541DDB59385140093940501C1800D
:1079B00095BF2167B98F7917E374F7FA97E7FF1F2F
:1079C00083C7C7C517A5010013050541E38F07EA63
:1079D00097A601009386C63861468145280097F036
:1079E000FFFFE780A04BAA85CE866146280097F06E
:1079F000FFFFE780A04AAA8597A60100938686A785
:107A00006146280097F0FFFFE78040492A8603552A
:107A1000610095462C0097E0FFFFE780803511C597
:107A200017A501001305453D8DB597A60100938666
:107A3000A63E130680028145081097F0FFFFE780FD
:107A4000E045CE86AA8513068002081097F0FFFF56
:107A5000E780C044AA8597A601009386263D1306B9
:107A60008002081097F0FFFFE780404383566100D3
:107A7000AA85114713068002081097F0FFFFE780E0
:107A8000C044CDBBC147E3FF87D0414697A5010065
:107A90009385453A4A8597800100E78000D0E3133B
:107AA00005D08347090113071003639CE70085474E
:107AB00017C7FF1F2304F79217A501001305C53848
:107AC000E9B31307000317A501001305E53AE39E88
:107AD000E7DA97C7FF1F2383079017A50100130557
:107AE000253865B381447DB917C5FF1F0345058F50
:107AF000828097E7FF1F83C767D889E717230000B5
:107B0000670063A4828097E7FF1F83C7C7DB99EFF5
:107B1000411106C697200000E780C09AB240854711
:107B200017E7FF1F2301F7DA410182808280630E8D
:107B3000053A638C053A1D71B706400086CEA2CC8B
:107B4000A6CACAC8CEC6D2C4D6C2DAC05EDE62DC5D
:107B500066DA6AD86ED601475948A5061319070197
:107B6000135909016371B902B307E50083C7070020
:107B7000D91793F7F70F6368F800B3D7F600858B32
:107B800013061700B9EF338925414209135909013A
:107B9000B947AE89AA8463F827053304E50039465E
:107BA00097A501009385C51A228597800100E7807B
:107BB000C0BE15E9CA85228597F0FFFFE780004621
:107BC000630E0530F6406644D6444649B649264A17
:107BD000964A064BF25B625CD25C425DB25D256107
:107BE00082803287A5BF97E7FF1F83C727C96384B9
:107BF0000722BD6A396C014A17EBFF1F130B8BB9C3
:107C0000938BFA55938CFA66130DEC5505A8B38740
:107C1000440183C6070097E7FF1F83D707C68DE798
:107C20009307A005639BF600854717E7FF1F231600
:107C3000F7C497E7FF1F238FD7B4050A93170A01EC
:107C4000C183E3E637FDBDBF854D639BB703930753
:107C5000500A639EF600894717E7FF1F231FF7C0EE
:107C6000930750FA17E7FF1FA306F7B2F9B7930778
:107C7000A005E384F6FC97E7FF1F239007C075BFBC
:107C8000138717004207DA9741832380D70017E64E
:107C9000FF1F2314E6BE8D47E3F1E7FA17E4FF1F49
:107CA000034474AF97E7FF1F83C7E7AE22045D8CE0
:107CB0009307F4FFC207C1839306F00DE3EDF6FAD4
:107CC00093076400C207C183E319F7F69305240004
:107CD000C205C18117E5FF1F1305E5AB97F0FFFF54
:107CE000E78000AA33078B0083475700034747000C
:107CF000A207D98F17E7FF1F231107B86312F510EA
:107D00000149630DB40117E9FF1F0349E9A82209DE
:107D100097E7FF1F83C757A83369F90017F5FFFFDF
:107D20001305053F97E0FFFFE780003963057909F8
:107D300063EF2B036308A9059307EC656303F9065A
:107D400097E7FF1F83C747A505476380E70881CBF7
:107D50001387A7051377F70F8D4663F9E608130716
:107D6000F0072300E100A300F100894595A863090D
:107D700099059387FA77E315F9FC97E0FFFFE78011
:107D8000807E11A8A28517E5FF1F1305E5A097E0E7
:107D9000FFFFE7800047014597E0FFFFE780C03124
:107DA00069BDA28517E5FF1F1305059F97E0FFFF3B
:107DB000E780204ECDB797E0FFFFE780A056E1BFF8
:107DC00097E0FFFFE780405CF9B7930710F81305D1
:107DD00011002300F10097E0FFFFE780A07BFD4545
:107DE0000A8597F0FFFFE780202B75B7A28517E57E
:107DF000FF1F1305659A97E0FFFFE780800261BFD0
:107E00009307F00789450A852310F10097F0FFFFDB
:107E1000E78080281DB5954763F8370B03C704003A
:107E20009307500B6312F70A03C714009307B005BA
:107E30000144631CF708CE85268597E0FFFFE780A5
:107E4000E03511C917A50100130545D997F0FFFFCB
:107E5000E780001B85BB17A50100130565D9FDB799
:107E6000B387840083C7070063842701639C4701AD
:107E70000DC597F0FFFFE780E06F97E7FF1F23999D
:107E8000079021A8E3EBAAFE130715005A9597E681
:107E9000FF1F239FE68E2300F500050493170401BE
:107EA000C18317E5FF1F0355A58EE3EB37FBE30BFB
:107EB00005D097F0FFFFE780E06BE30505D097E77B
:107EC000FF1F2397078CFDB901443549294A930ABE
:107ED000E00417EBFF1F130BAB86C9B7CE852685D1
:107EE00097B0FFFFE780C02FF1B98280411126C211
:107EF000AE848D4522C406C62A8497B0FFFFE78072
:107F000020F9B717004099C803A5C70C418D23A6D7
:107F1000A70CB240224492444101828003A5870C01
:107F2000418D23A4A70CF5B783470500034715002F
:107F3000A207D98FC2076177C18713072720639AE9
:107F4000E70083452500370504001703000067009C
:107F500023FA828017E6FF1F130646978147B286F1
:107F60001303F00FA9483308F6000348080013F77D
:107F7000F70F6307A80C630668008507E39517FFF2
:107F80002947B387E6002380A70097E7FF1F938761
:107F9000A7945DA8411113D765001347170006C6C3
:107FA00093F63500058B954791CA05469947638737
:107FB000C60009469D476383C600A14713F64500E6
:107FC0003336C00093F68503050685C2A145638B51
:107FD000B604E145638AB604930580026388B6045B
:107FE000930580036393B600914697E5FF1F238AAC
:107FF000F5B497E5FF1F2385C5B497E5FF1FA3815F
:10800000D5B4BE8517A501001305C5F797800100FB
:10801000E7806086B240854717E7FF1FA303F7B2EA
:10802000410182808546D1B78946C1B78D4675BF6B
:1080300017A50100130585F7178301006700A383C7
:1080400017E7FF1F13074789BA972380B700E14757
:10805000E302F5F493077002E30CF5FC82802A87B3
:1080600023800500814717E5FF1F130525861308A8
:10807000F00F2946B306F50083C606006396E602B4
:1080800097E6FF1F93864685B69783C70700054589
:108090002380F5009947636EF7029D4763FDE70073
:1080A000E147630DF7008280638506018507E3934E
:1080B000C7FC0145C5B7238005008280B737004063
:1080C00003C7370083C7050093F70704D98F2380C0
:1080D000F50082805D7152DC56DA5ED6716A97EBEC
:1080E000FF1F938B2BB78D6AA6C24EDE62D486C665
:1080F000A2C4CAC05AD866D26AD06ECEC1495E8CBC
:1081000097D4FF1F9384047E130A0A20938A7ADC93
:1081100017E9FF1F034909B7B3872B0183C707007E
:1081200093F7F70FC9EFB787004003C76700058BC8
:10813000E310077C03C76700118BE30D077E83C73D
:108140005700918B99E36F10200317E7FF1F034738
:1081500087B385476304F7006F10400197E7FF1F5F
:10816000A381E79E97E7FF1F238E078297E7FF1FF4
:10817000238C078E97E7FF1F238A079A97E7FF1F35
:108180002387079A97E7FF1FA38E078097E7FF1FB4
:10819000A38C078C97E7FF1FA38A079897E7FF1F19
:1081A000A387079897E7FF1FA38E079897E7FF1FFE
:1081B000A38B07ACB787004011476F007077930718
:1081C000190093F7F70F3D476364F70617E7FF1FA2
:1081D000230AF7AA97E7FF1F9387C7A9CA9783C700
:1081E00007001307100293F7F703638EE71E636619
:1081F000F70405446385871CE38C07620947638E97
:10820000E71013070002E384E74EB7E700E0370703
:10821000400023A0E7180100010062992300090033
:10822000FD1923A0E71093F9F90FE39309EEE5BDDB
:1082300097E7FF1F238807A471BF130730026388E5
:10824000E70C63E8E71613074002638CE70A13079D
:108250000003E39CE7FA97E7FF1F9387A7A0CA975D
:1082600003C70700A1471377F70FE31BF71483C772
:10827000640097E6FF1F238DF68A97D7FF1F83C7F9
:10828000D76691C7FD5797E6FF1F2383F68A97D5D8
:10829000FF1F83C5356597E7FF1FA38BB78897D767
:1082A000FF1F83C7276413FB07089306000493F797
:1082B0000706639FD74C9307A009638DF51663EA01
:1082C000B7129307F0056386F54A93075009638454
:1082D000F52A014497E7FF1F83C797851547E39267
:1082E000E736B7E700E03707400023A0E7180100B2
:1082F0000100B786004023808602130680FC6F00D1
:10830000500EFD5717E7FF1F2303F782FDBDFD57F2
:1083100017E7FF1F230CF780CDBD17A5010013053C
:1083200065DA97700100E780E06C97E7FF1F93879D
:108330006793CA9703C40700014B97DCFF1F938C18
:10834000EC721374F40F17AD0100130D2DD86347B1
:108350008B04294597700100E780C056854717D7E1
:10836000FF1FA303F77017D7FF1F2300877017D7CE
:10837000FF1F2309F77C37E700E0B7064000232002
:10838000D71801000100378600408347A60293F703
:10839000370F2305F6022320D71085BDB3876C0164
:1083A00083C507006A85050B97700100E780A04C24
:1083B00079BF854717D7FF1F2308F76AB9B517E7B5
:1083C000FF1F1307278A4A970347070097D6FF1F07
:1083D000A38AF65C97D6FF1F2387E65C17D7FF1F9B
:1083E0002302F7761DB5854717D7FF1F230CF75AD1
:1083F00029BD9307400A6389F5349307200B6384F2
:10840000F5369307100AE396F5EC838724000144C0
:10841000E3D207EC97D7FF1F83C7F74C93F63700DB
:10842000638A061A0546638AC62209466395C61AF8
:108430001D4755A217D5FF1F0345E54AC94797DCDD
:10844000FF1F83CC5C4A97D5FF1F83C5E54917D42E
:10845000FF1F034474496315F510CD476392FC1068
:1084600093077008639CF5021307300FB7170E00CF
:108470006308E4001307900DB7B704006314E40821
:1084800017D7FF1F232CF76ABE8517A50100130518
:1084900065C497700100E780003E25BD9307800802
:1084A000639DF500B307804013F4F70FB7774600DC
:1084B000938787CDB3D78702E1B793079008639A74
:1084C000F500B307804013F4F70F91679387C766F1
:1084D000D5B79307A008639BF500B307804013F45A
:1084E000F70FB7173D0093870790E9B79307B008D8
:1084F000639AF500B307804013F4F70F91679387F1
:1085000097D04DBF93F5F5078D47639BF500B307F3
:10851000804013F4F70FB7975B00938707D859BFD4
:108520008947639BF500B307804013F4F70FB777D3
:108530000B009387071BBDBF8547639AF500B30700
:10854000804013F4F70FDD67938767E3A5B7D28701
:1085500085F9B307804093F7F70FB3D7FA020DB749
:1085600097000000E780409FA28566859700000085
:10857000E780809EB9BB9305610017D5FF1F0345B7
:10858000853617D4FF1F0344143697000000E78098
:1085900040AD93057100228597000000E78060AC34
:1085A0003C0017D7FF1F2325F76A83476100230488
:1085B000F10083477100A304F100894717D7FF1F1B
:1085C0002308F7568357810017D7FF1F231CF73066
:1085D000094409B3154793F64700B336D00093F723
:1085E0008703850685C32146638BC7066146638A78
:1085F000C706130680026388C706130680036393C9
:10860000C700914717D6FF1F230CD65297D6FF1FDE
:10861000A388F65297D7FF1F2385E75217D7FF1F6E
:108620000347872C9376070497D7FF1F83C7D72B61
:108630008DEE1377770C93067008630CD7021377CF
:10864000F7078D466312D70CB307F040B7955B0070
:1086500093F7F70F938505D849A81947ADBF85470C
:1086600055B7894745B78D4771BF930670086311A9
:10867000D7021307300FB7150E006389E7021307FF
:10868000900DB7B504006383E7021307700845BF78
:108690009306800C6311D702B307F040B77546000C
:1086A00013F7F70F938785CDB3D5E70297D7FF1F51
:1086B00023A6B748D9BB9306900C631CD700B30719
:1086C000F04093F5F70F91679387C766B3D5B7026C
:1086D000F1BF9306A00C631DD700B307F040B71598
:1086E0003D0093F7F70F93850590B3D5F5027DBF55
:1086F0009306B00CE315D7F4B307F04093F5F70FEA
:108700009167938797D0D9B78946631BD700B30782
:10871000F040B7750B0093F7F70F9385051BF1B782
:108720008546631AD700B307F040DD6593F7F70F6E
:10873000938565E35DBFD28535FBB305F04093F5C6
:10874000F50FB3D5BA029DB783C72400C18B99C773
:10875000854717D7FF1F2300F73EA5BE97D7FF1FFA
:10876000238B073CBDB6854717D7FF1FA30BF73CEC
:108770008DB63C0017D7FF1F232CF74C09479307F2
:1087800000032314F10097D6FF1F2383E63A2DBD83
:1087900063940756A94763E5B7421797010013078B
:1087A000A77B8A05BA959C41BA97828717D4FF1F89
:1087B00003447413894C6306940D63E68C06854765
:1087C0006303F4089307F00F17D7FF1F03474736DB
:1087D00063F6E70017D7FF1F230CF73497DCFF1F62
:1087E00083CC0C359307000413F4FC0F63F497015A
:1087F0001304000497D7FF1F9387874503AD070035
:1088000022862685EA85B38C8C40229D97700100D4
:10881000E78000FB97D7FF1F238C973197D7FF1F67
:1088200023A8A74345BC8D47630CF40A9947E31B73
:10883000F4F8979701009387A77817D7FF1F23298C
:10884000F740A94751B717D7FF1F0347C74397D72B
:10885000FF1F9387E72F4946979501009385457F32
:1088600063068700979501009385857A3E8597700A
:108870000100E780E0F417D7FF1F232BA73CC9476F
:10888000A1B797D6FF1F83C60640054797D7FF1F9E
:108890009387072C6394E6023E8513067002979532
:1088A00001009385657897700100E78060F117D724
:1088B000FF1F232FA7389307700239B73E85130691
:1088C0003004979501009385657097700100E780EB
:1088D00020EF17D7FF1F232DA73693073004EDB5E0
:1088E00097D5FF1F83C52500179501001305C57F88
:1088F00097700100E78020F8054D97DDFF1F83CDBD
:108900008D3897D5FF1F83C505FE17950100130508
:10891000A57D6398AD0B97700100E780C0F597D7F0
:10892000FF1F83C747FCB5CBE36EF4E81794010043
:1089300013044476638CB701179401001304047682
:1089400063869701179401001304C47622859770FB
:108950000100E780600B1375F50F9307150086077C
:1089600017D7FF1F2306F71E8D4717D7FF1FA30139
:10897000F71E97D7FF1F9387A71D0147BE86137663
:10898000F70F89076365A60297D7FF1F23A2D72C8D
:1089900097D7FF1F83C7C71B05BD97970100938714
:1089A000676817D7FF1F2325F72A914731BD330684
:1089B000E40003460600A380070005072380C700E4
:1089C0007DBF97700100E78000EB97D7FF1F83C73B
:1089D00087F1E1D7E368F4DE17940100130484689B
:1089E000638CA70117940100130444686386970100
:1089F0001794010013040469228597700100E78031
:108A0000A0001375F50F93071500860717D7FF1FF2
:108A10002300F7148D4717D7FF1FA30BF71297D723
:108A2000FF1F9387E7120147BE861376F70F89076A
:108A3000E37CA6F43306E40003460600A3800700A7
:108A400005072380C700D5B797D5FF1F83C5A5E9C4
:108A5000179501001305056A97700100E780A0E1F2
:108A600097D7FF1F83C7970E93E7470017D7FF1FBE
:108A7000A30EF70C83C7240017D7FF1FA306F70C1C
:108A800089B8179501001305256897700100E780E4
:108A900060F697D7FF1F9387270B83C7070017D769
:108AA000FF1F2301F7E417D4FF1F03446408333486
:108AB00080000DB017950100130545669770010001
:108AC000E78040F397D7FF1F83C7570893E7070155
:108AD00017D7FF1FA30CF70683C7240017D7FF1F64
:108AE0002304F7066FF0EFFE1795010013054564A8
:108AF00097700100E78000F003C704007D8B51EF01
:108B0000B787004003C767021377C70B13672700B7
:108B10002383E70203C7A7021377C70B1367270056
:108B20002385E70203C7E7021377C70B1367270004
:108B30002387E70203C727031377C70B13672700B1
:108B40002389E702854717D7FF1F230DF7E417D7BF
:108B5000FF1F230BF7F017D7FF1F2309F7FC17D7C9
:108B6000FF1F2306F7FC97D7FF1FA38D07E297D7B8
:108B7000FF1FA38B07EE97D7FF1FA38907FA97D78D
:108B8000FF1FA38607FA97D7FF1FA38D07FA97D772
:108B9000FF1FA38A070E6FF0CFF389476312F70216
:108BA00097D7FF1F83C747D49146638CD70863E0EC
:108BB000F604638EE70C6369F70A05476380E70EE6
:108BC000FD5717D7FF1FA305F7F637074000B7E794
:108BD00000E023A0E71801000100B786004013065B
:108BE000F0FC2381C60223A0E7106FF00FE2130709
:108BF00020086382E7086362F70213071008E39115
:108C0000E7FC378700408347670293F7C70B93E77A
:108C100027002303F7026FF0CFEB130730086389B7
:108C2000E70213074008E39DE7F8378700408347D2
:108C3000270393F7C70B93E727002309F7026FF089
:108C40004FE9378700408347270393F73707F5B786
:108C5000378700408347E70293F7C70B93E7270066
:108C60002307F7026FF0EFE6378700408347E702FC
:108C700093F73707F5B7378700408347A70293F785
:108C8000C70B93E727002305F7026FF08FE43787C0
:108C900000408347A70293F73707F5B737870040AF
:108CA0008347670293F73707ADB7179501001305A0
:108CB000254997700100E780E0D397D7FF1F2383F2
:108CC00007C2D5B3179501001305854897700100B9
:108CD000E78040D297D7FF1F239607C097D7FF1F83
:108CE000938707E503C40700894763F387000944B6
:108CF0001374F40F6FF00FDE13070002E392E7EC3A
:108D0000631B0B0A638FF500930720026383F5084A
:108D1000179501001305454797700100E780A0B53E
:108D200045B5179501001305654397700100E7806D
:108D300060CC0144179D0100130D8D43A14CB387F6
:108D4000840083C507006A85050497700100E780E9
:108D500080B2E31694FF178501001305A57797707D
:108D60000100E78020C917D4FF1F0344E4B701E8DE
:108D700097D7FF1F238A07B4014B6FF0AFD5894700
:108D8000E310F4E4854717D7FF1F230FF7B26FF006
:108D90004FD417D6FF1F034616B597D5FF1F83C5BF
:108DA00085B4179501001305253D97700100E780F4
:108DB00080AC6FF00FD26380F50693071002E39941
:108DC000F5F497D5FF1F83C525B21795010013054C
:108DD000A53C97700100E78000AA97D7FF1F23A941
:108DE00097E697D7FF1F938767D5944383D74700AC
:108DF00017D7FF1F0347E7D417D6FF1F2324D6AE8C
:108E00001D4497D6FF1F2391F6AE97D7FF1F238EE1
:108E1000E7AC6FF02FCC97D5FF1F83C5E5AC179556
:108E200001001305E53897700100E780C0A497D7CB
:108E3000FF1F238B07A897D7FF1F239507AA6FF063
:108E40002FF92547638FE7C8994637870040639419
:108E5000D70223008702B7E700E0B706400023A04F
:108E6000D71801000100130600FC2301C70223A04C
:108E7000D7106FF08FB99306100A639FD7002300B5
:108E80008702B7E700E0B706400023A0D71801002B
:108E90000100130680FCD1BF9306A009E381D7FE31
:108EA0009306400AE38DD7FC93062002639DD7000A
:108EB000B7E700E0B706400023A0D7180100010083
:108EC00023008702F9B78546E384D7FE930700089D
:108ED000E300FBFEB7E700E0B706400023A0D71889
:108EE00001000100130620FC23008702BDBF17D735
:108EF000FF1F0347F7C36302F71E63E7E7029547C7
:108F00006300F7109947630AF704B786004023808F
:108F10000602B7E700E03707400023A0E71801008A
:108F200001001306A0FC75B99307F005630AF7006A
:108F3000930750096306F70093071002E317F7FC45
:108F4000B7E700E03707400023A0E7180100010061
:108F5000B7860040130620FC69B117DBFF1F034BE7
:108F60002BBD930700045A8D63F46701130D0004B1
:108F700097D7FF1F9387C7CD83AC07001374FD0FEE
:108F80002286E685268597700100E7806083B30717
:108F90008B40669417D7FF1F230CF7B897D7FF1F96
:108FA00023A887CAB7870040630C0B022380A7035E
:108FB000B7E600E03706400023A0C6180100010014
:108FC00003C72702134707042381E70203C72702C9
:108FD0001377C70F2381E70223A0C6106FF0EFA21B
:108FE0002380070237E700E0B70640002320D718A8
:108FF00001000100130620FC2381C7026FF0AFB906
:10900000378700408347370097D6FF1F83C6D6B304
:1090100093F70708D58FA301F700B7064000B7E71D
:1090200000E023A0D718010001001306A0FC35BD05
:1090300097D7FF1F938707C3CA9783C7070093F784
:10904000F70FC1CF97D7FF1F83C7E7C3D9E717D75C
:10905000FF1F0347F7AD930700026310F70883ADC6
:10906000040017DDFF1F034D2D8897DCFF1F83CC05
:10907000BC8717DBFF1F034B4B87E6876A87DA86BF
:109080006E8697D5FF1F83C52584179501001305AC
:10909000A51397600100E780007E97D7FF1F23AFDD
:1090A000B7A997D7FF1F238DA7A997D7FF1FA3891C
:1090B00097A997D7FF1F238667A997D7FF1FA38478
:1090C0008780B7E700E03707400023A0E7180100DA
:1090D0000100B78600406FF04FA2B7E700E0370706
:1090E000400023A0E71801000100B786004015BD2D
:1090F00097D6FF1F83C626B90547639CE604294718
:109100002381E70209472383E7022385E70297D7F4
:10911000FF1FA38907A297D7FF1FA38607B6B787AC
:109120000040A381070017D7FF1FA30F07A0054723
:109130002383E700B640264496440649F259625A12
:10914000D25A425BB25B225C925C025DF24D61617D
:10915000828029472381E70209472383E702238589
:10916000E7022387E7022389E70255B717C7FF1FE6
:10917000A30BF7746FE01FFF854717D7FF1F23036B
:10918000F78217D7FF1F2301F78E17D7FF1F230F73
:10919000F79817D7FF1F230CF7986FE0BFFE85479E
:1091A00017D7FF1F2300F78017D7FF1F230EF78A5B
:1091B00017D7FF1F230CF79617D7FF1F2309F79622
:1091C00017C7FF1FA300077E17D7FF1FA30E07882F
:1091D00017D7FF1FA30C079497D7FF1FA3890794E6
:1091E0008280411106C697000000E78080FBB787A8
:1091F000004023800700130740FC2386E700130785
:10920000C004A386E70017C7FF1F1307A76D2398A5
:10921000E70017C7FF1F1307E770239AE70017C778
:10922000FF1F1307677C239CE70017D7FF1F130757
:10923000E787239EE70029472381E7020947238325
:10924000E7022385E7022387E7022389E702A38158
:109250000700930600F8A380D700930690022380AE
:10926000D700FD562383D7002381E700930600052E
:1092700037E700E0230BD740B70640002320D71084
:1092800003C7170013671700A380E700B24097D702
:10929000FF1F239B078A41018280411106C6970068
:1092A0000000E78000F0B787004023800700130725
:1092B00000FC2386E7003147A386E70017C7FF1F9E
:1092C000130747622398E70017C7FF1F1307876537
:1092D000239AE70017C7FF1F13070771239CE700B6
:1092E00029472381E70209472383E7022385E70211
:1092F000A3810700930600F8A380D700930690028D
:109300002380D700FD562383D7002381E7009306EF
:10931000000537E700E0230BD740B70640002320C5
:10932000D71003C7170013671700A380E700B240E8
:1093300097D7FF1F239A078041018280F1679387A7
:10934000072017C7FF1F232BF77E854717C7FF1F6F
:109350002318F77EA14717C7FF1F2304F77E97C77F
:10936000FF1FA380077E97C7FF1F238D077C97C72A
:10937000FF1F238B075497C7FF1FA38607548147FE
:1093800017C5FF1F13058554FD5517C6FF1F13068C
:10939000A6542947B306F5002380B600B306F600AD
:1093A000238006008507E397E7FE97C7FF1FA38288
:1093B000077897C7FF1FA380077897C7FF1F238BE6
:1093C000077697C7FF1F2386077697C7FF1F23855A
:1093D000077697C7FF1FA38F077497C7FF1F238CBC
:1093E0000774814717D6FF1F1306C6864147B30689
:1093F000F600238006008507E39BE7FE828017D7EF
:10940000FF1F0347478885476316F70017030000CF
:109410006700E3E8170300006700E3DC411122C4A2
:1094200006C617D7FF1F0347078685472E8613F406
:10943000F50FAA856317F70417C5FF1F1305C55E4F
:1094400097600100E780C03797C7FF1F238E076032
:10945000B787004023848702B7E600E03706400064
:1094600023A0C6180100010003C7A7021377C70F86
:109470002385E702B240224423A0C61001454101E2
:10948000828017C5FF1F1305E54D97600100E78037
:10949000203397C7FF1F23870750B78700402382D9
:1094A0008702B7E600E03706400023A0C618010097
:1094B000010003C767021377C70F2383E7025DBF6D
:1094C000411106C697000000E78080E7B2404101E5
:1094D000170300006700E3F2411106C697F0FFFF93
:1094E000E78080BF97C7FF1F83C7D74BA1CB97C526
:1094F000FF1F83C5454B89C917C5FF1F1305C54A03
:1095000097E0FFFFE780E06297C7FF1FA38C074843
:1095100097C7FF1F2388076237E700E0B7064000C0
:109520002320D718010001003786004083476602D8
:1095300093F7370F2303F6022320D710B2404101DF
:10954000828041C9D9C597C7FF1F83C7E75FD1C3D1
:10955000011122CC4AC84EC656C25AC006CE26CAEF
:1095600052C42E89AA890144930A0004371B0300C0
:1095700063772403B3078940C207C183BE8463F4C1
:10958000FA0093040004C204C180130A1BD497C7D5
:10959000FF1F83C727419DE37D1A631C0A00F24029
:1095A0006244D2444249B249224A924A024B05617E
:1095B000828097F0FFFFE78020B2D1BF338589001A
:1095C0002694A685420497000000E78060E541806C
:1095D00045B7828097C7FF1F9387477D18429C43FA
:1095E00083D645000345070083C5C70003564600E0
:1095F0006396A50083D5E700638DD502011106CEE1
:109600002386A7002397D700B705CF00DC4B9385AF
:10961000757D05077D162EC2230001003AC423166E
:10962000C1002317D10099C30A858297F2400561D2
:1096300082808280411122C417A4FF1F130484DC9E
:109640005C4C06C691CBC84B01C9B7E70400BC57B8
:1096500082975C4C23AA0700B240224441018280D9
:10966000DC4DDC4B81CFB7E70400904503A38705B1
:10967000914517C5FF1F0345A57302838280B7E795
:10968000040003A30705A14517C5FF1F0345457245
:1096900002836D713C083EC6B707E5002322911096
:1096A0003EC8AA843C083285232611103ECA2324D2
:1096B0008110232021112E8997300000E780006659
:1096C0002A84979501009385A5B3177501001305AA
:1096D000E57A97600100E780001AA28517950100DE
:1096E0001305C5BE97600100E780E0182945976023
:1096F0000100E780201DB705CB009385757D6800CC
:1097000097100000E780A067A285680097300000EE
:10971000E7802053014781467000CA85268597203F
:109720000000E780208B05CD2A8497950100938562
:1097300025AD177501001305657497600100E7807A
:109740008013A28517950100130505B997600100E4
:10975000E7806012294597600100E780A01683200A
:10976000C110032481108324411003290110516189
:10977000828097C7FF1F9387676318429C43797164
:1097800022D406D60348070083C807012A8483D65B
:109790004500035546006396080183D82701638D71
:1097A000D8022388070105072399D7003708CC0082
:1097B000DC4B1308787D3ACC1307F5FF42CA230827
:1097C0000100231EE100231FD10099C7080832C6FB
:1097D0002EC482973246A245228597000000E7807A
:1097E00080EBB25022544561828079713146977581
:1097F000010093856559280006D697600100E7802F
:1098000020FC97A7FF1F83D7E7BF231B0100231C62
:109810000100231D0100231E0100231F010099E305
:10982000C167FD17231AF10097A7FF1F83D7A7BDB4
:1098300091EB97C7FF1F938767579C439C43DC4777
:1098400083D7070097A6FF1F9386C6BB231BF10093
:10985000D84E83D74600231CF1005C4B91CB97A7D1
:10986000FF1F83C797BA81EB97000000E780C0DC39
:10987000B25045618280FD1717A6FF1FA307F6B8F7
:109880000356070183C706014C472800230FF10048
:1098900097300000E780003897C7FF1F9387075174
:1098A0009C430147979601009386069F88433000AA
:1098B0004C0897100000E780E0715DD975B799C931
:1098C000B7E7040003A30705A14517C5FF1F03451C
:1098D000254E028382805C4EDC4BB9CFB1CD411165
:1098E00022C417750100130565592E849795010050
:1098F0009385459606C697600100E780C0F7A2856C
:10990000179501001305459797600100E780A0F6C1
:10991000294597600100E780E0FAB7E70400224498
:10992000B24003A3870517C5FF1F0345654813060B
:1099300040069145410102838280411122C417A44F
:10994000FF1F1304E4A91C4C06C689C7DC4399C356
:109950004C488297584CB7E70400BC57484B829755
:109960005C4CB240224423AA07004101828017A721
:10997000FF1F1307E7A8834707009306F00B85072F
:1099800093F7F70F63E9F60097A6FF1F238AF6A661
:10999000034507008280930700F8FDB78357450011
:1099A00099E37D558280011122CC17A4FF1F130477
:1099B00064A55C4C4AC84EC6DC4B52C406CE26CACF
:1099C00056C2B2892E8A2A898DC7B7E70400FC5F88
:1099D000829797C7FF1F9387673B9C431307301FEE
:1099E000B307F54071556375F70697000000E780EF
:1099F000A0C49307D00D7D5563EC3705B7E4040090
:109A000093878900B858832AC401139507014181BF
:109A1000029723AAAA00484C584921E797950100CC
:109A20009385458117750100130545459760010031
:109A3000E78060E4179501001305C58C976001006D
:109A4000E78060E3294597600100E780A0E75D5566
:109A5000F2406244D2444249B249224A924A0561E4
:109A6000828013874900B705CF002319E50093854D
:109A7000757D310597100000E7806030484C8345C4
:109A80006900310597300000E780A01B484C4E86E6
:109A9000D285310597300000E780C0177146CA852E
:109AA00017A5FF1F1305059697600100E78040D1B9
:109AB000FC5C82970326C90097C7FF1F23A8A72C29
:109AC00011CABC4C854517C5FF1F0345652E8297FB
:109AD0000145BDBF97000000E78060D1D5BF4111AF
:109AE00006C622C426C217C4FF1F1304642C9700A5
:109AF0000000E78060B4B7E40400FC4C03450400B8
:109B00008545829703450400224403A3C405B2405F
:109B10009244A14541010283411126C297C4FF1F0F
:109B20009384C4289C4006C622C44AC0D5C3DC43E3
:109B3000C5C35CC12300B5002A84978501009385C5
:109B4000A56A177501001305653397600100E7806A
:109B500080D2294597600100E780C0D69C4023A4AD
:109B6000070023A2070097A7FF1F93876787DC4F93
:109B7000DC4B91C7295597000000E78040DC97A790
:109B8000FF1F93872788DC4FDC4B89C797000000B5
:109B9000E78020F537E904008327C905894517C503
:109BA000FF1F0345E52082978327C905914517C507
:109BB000FF1F0345E51F82979C4003A347016309EC
:109BC000030022852244B2409244024941010283AB
:109BD000B2402244924402494101828001113285FF
:109BE00006CE22CC26CA2E8497300000E7800013D0
:109BF000AA84978501009385656217750100130596
:109C0000E52797600100E78000C70307840003563B
:109C1000640083554400A686178501001305456836
:109C200097600100E78020C5294597600100E78023
:109C300060C99797FF1F83C7077B639D9700014506
:109C400097000000E780A0CF81450A8597000000BB
:109C5000E780C0ECF2406244D244056182806D71BD
:109C600023248110232611102322911093F74500FD
:109C70002E84638707143C083EC0B707E5003EC248
:109C80003C083EC4231701002318010023190100DA
:109C9000231A0100231B01009797FF1F83D74774E6
:109CA00099E3C167FD172316F1009797FF1F83D72C
:109CB000477391EB97C7FF1F9387470F9C439C43C4
:109CC000DC4783D707001797FF1F13076771231718
:109CD000F100544F835747002318F100DC4AA1E7F5
:109CE000978501009385C557177501001305051960
:109CF00097600100E78020B817850100130505670C
:109D000097600100E78020B7294597600100E78050
:109D100060BB134544008320C110032481108324B9
:109D20004110516182809797FF1F83C7D76B2555DC
:109D3000D9C3FD171796FF1FA307F66A03D60601BE
:109D400083470701CC460A85230BF10097300000BA
:109D5000E78040EC97C7FF1F938747059C43179701
:109D6000FF1F1307E76797860100938666508843B5
:109D70000A866C0097100000E780C025AA8451D99C
:109D8000978501009385C54D177501001305050FD3
:109D900097600100E78020AEA685178501001305B6
:109DA000A55D97600100E78000AD2945976001003F
:109DB000E78040B1268597000000E78040B891BF5A
:109DC00093F725009DC7B7E70400BC47414681458E
:109DD00028088297255597000000E78040B628089C
:109DE0009305F00F97000000E78040D3134524004F
:109DF0001DB793F7150081CB97000000E780209FE7
:109E00001345140009BF93F78500014589D71797BB
:109E1000FF1F0347975F9797FF1F9387A75E0DC3A9
:109E2000D84F584B11CF37E70400384F904785453E
:109E300017C5FF1F0345C5F7029713458400E1BD11
:109E400097F0FFFFE780407FCDBF5C4D411106C614
:109E500088C317C7FF1F232BF7F4B7E7040083A7B6
:109E60000708170500001305C5DF8297B24097C7A2
:109E7000FF1F238FA7F20145410182800111333575
:109E8000A000A307A100B7E7040083A7471706CEE9
:109E90001306F1008545130550308297F2400561A5
:109EA0008280B7E7040003A387051306000A9145E3
:109EB0001795FF1F0345055802838280411106C68E
:109EC00022C497A7FF1F83C7373581EF97B7FF1FBE
:109ED00083C7C774014481EF97A7FF1F83C7C733A8
:109EE00099E7014597000000E78080F90544228545
:109EF00097000000E780C0F8178501001305854E24
:109F000009E4178501001305E54E2244B2404101E2
:109F10001763010067002396797122D4A30F010013
:109F200037E404008327841726D24AD006D6AA84B1
:109F30002E89130550309305F10132C682973246BF
:109F40008347F10193150601C18185CB01452EC6DA
:109F500097000000E780C0F283274417B2454A8685
:109F600026858297054597000000E78060F1B25092
:109F700022549254025945618280832744174A86AD
:109F800026858297EDB741119397050122C406C635
:109F900026C2C1872E8463D40702B7E40400FC54B0
:109FA0001795FF1F03450549829719C1BC54829735
:109FB0002165218DB240224492444101828093F771
:109FC00015008DC7B7E7040083A7471A1796FF1F30
:109FD0001306464597C5FF1F938545DE1795FF1F5E
:109FE00003454545829713451400E9B793F72500CB
:109FF00085CF97C7FF1F83C7E7DD85E7B7E7040075
:10A0000003A8871A1307401F9797FF1F83C787422C
:10A01000814613064006994517C5FF1F035505DB0A
:10A0200002981345240079B793F745000145D9D329
:10A0300097000000E780C0E813454400A5BF97C71C
:10A04000FF1F83D7A7D86398A70217C7FF1F231046
:10A05000B7D817C7FF1F231DC7D617C7FF1F231A5F
:10A06000D7D62E86178501001305453FBE85176399
:10A07000010067004380178501001305A53F1763A2
:10A080000100670023970357450097C7FF1F83D739
:10A09000E7D36319F704C167F91717C7FF1F232711
:10A0A000F7D297C7FF1F238707D297C7FF1F23A1A8
:10A0B00007D297C7FF1F238907D097A7FF1F238DBC
:10A0C0000714B7E70400FC4F411106C689451795F0
:10A0D000FF1F034525368297B24041011703000058
:10A0E000670063DC178501001305C538176301009D
:10A0F000670043907D15954763E5A71E178701000C
:10A100001307C72C0A053A951C41011122CC06CE33
:10A11000BA972E848287178501001305253697602C
:10A120000100E780208DF24062440561828003C710
:10A1300025009947631AF7022E8597A7FF1F238DE5
:10A14000070C97000000E78040F483456400178502
:10A1500001001305A53397500100E780C0711785F2
:10A1600001001305653465BF97A7FF1F2386070A03
:10A17000FDB703C7250095476319F702C16717C7E5
:10A18000FF1F0357A7C4F91703D5A5006309F702FA
:10A19000B7E7040083A7C717829717850100130547
:10A1A000A53197600100E780E084854717A7FF1F6E
:10A1B0002304F70617850100130585328DB797C76D
:10A1C000FF1F2395A7C083D7E50097C6FF1F2390E5
:10A1D000F6C083D7050197C6FF1F239BF6BE83D722
:10A1E000250197C6FF1F2396F6BE97C7FF1F238D35
:10A1F00007BC631FE5000356E4008355A4001785E0
:10A2000001001305A52C97500100E780C06671BFBF
:10A210009307700F2316F100B7E7040083A7870D9B
:10A220001796FF1F034606216C00829769F5854744
:10A2300017C7FF1F230AF7B87DBF17850100130555
:10A24000E52AF1BD83C5250091476393F502178583
:10A2500001001305252B97500100E780A07997A7EF
:10A26000FF1F238B07FA97000000E780C0C365BD7E
:10A2700099476396F502228597A7FF1F238E07F85B
:10A2800097000000E78060E08345640017850100C7
:10A290001305C51F97500100E780E05D69B595473C
:10A2A000639AF50083471400DDFB17850100130551
:10A2B000A527B5B51785010013058527E1BF1785CB
:10A2C00001001305652697500100E780A07297A74B
:10A2D000FF1F238307F4F95717C7FF1F2318F7AE93
:10A2E00059B782803757315F9797FF1F9387C715FC
:10A2F000130777D598C39356C50017870100130736
:10A30000A712BA9683C5060093568500BD8ABA96F1
:10A3100003C6060093564500BD8A3D89BA962A9722
:10A3200083C6060003470700238407002383D70062
:10A33000A383E7002382B700A382C7009797FF1F7C
:10A34000938787112383B700A383C7002384D70093
:10A35000A384E7008280411106C697000000E780D1
:10A36000A0F8B7E7040083A787141796FF1F13060A
:10A37000A60DD54501458297B2404D469795FF1FE2
:10A380009385850D130570304101170300006700A8
:10A39000E3B861712324811A37E404008327040899
:10A3A0002326111A2322911A2320211B232E31192F
:10A3B00017050000130565BD82971799FF1F130944
:10A3C0006907994785442300A900231CF10097855C
:10A3D0000100938565049307400617750100130576
:10A3E000E5A9231CF1082308910097B9FF1F938961
:10A3F000493397500100E780004883D5090017854D
:10A4000001001305650097500100E780C04629450B
:10A4100097500100E780004B03D50900970000002A
:10A42000E78080EC832744171008854513055030DA
:10A430008297832744171796FF1F1306E601CD4521
:10A44000130570308297832744171796FF1F130652
:10A45000A6FEB54513056030829783274417300860
:10A4600089451305103182978327441730098945A0
:10A47000130520318297832744159305000A0D4563
:10A480008297832744159305000A11458297A305F7
:10A4900091002306910002CD23080100230C010046
:10A4A00083278416300991451305704082978327CE
:10A4B00084161306B1008545130500408297832753
:10A4C00084167000854513051040829783278416F3
:10A4D000300885451305204082978327841610088D
:10A4E0008545130550408297832704157D55829733
:10A4F000832744137D5582977D559790FFFFE78012
:10A50000C0188327440C82979790FFFFE78020F4C0
:10A51000832784141796FF1F130606F3D5450145BC
:10A52000829789471306700F814528092306F10099
:10A530009780FFFFE780A0BD8D4713060008814587
:10A540002808230CF1089780FFFFE78040BC914763
:10A55000230CF100977701009387C783984383C743
:10A5600047003AC8230AF10097C0FFFFE780000EBA
:10A570007000854505459790FFFFE780201830095A
:10A580009305700F09459790FFFFE780201730086B
:10A59000930500080D459790FFFFE78020161008EF
:10A5A000954511459790FFFFE7804015C16717C794
:10A5B000FF1F1307A781F9171CC323220700179554
:10A5C000FF1F1305E5E69790FFFFE7800012832742
:10A5D000C41D17B5FF1F1305E57D82973C48034551
:10A5E0000900854582978320C11A0324811A832498
:10A5F000411A0329011A8329C1195D618280C1674B
:10A6000017B8FF1F0358887CF9176301F8083DCD80
:10A61000B5CD011126CAB7E4040083A7841222CC69
:10A620002E862315B10006CE2A8401478146ED45CA
:10A63000428582972AC611ED17850100130505E0B2
:10A6400097500100E780003BF2406244D24405612C
:10A650008280FC440356A100A28582972C0017B586
:10A66000FF1F0355A5769790FFFFE780C01469DDB3
:10A67000178501001305C5DD97500100E78080377D
:10A6800083A7C412ED45280082977DBF82800DC547
:10A6900085471797FF1FA306F7DA9797FF1F2383B6
:10A6A00007DA35469795FF1F938505D91305603066
:10A6B00017030000670083869797FF1FA38307D8BF
:10A6C000E9BF97B7FF1F83C7E770A9EFC16717B747
:10A6D000FF1F0357A76FF9176306F704411185475A
:10A6E00022C417B7FF1F2307F76E37E404007C4C22
:10A6F00006C689451795FF1F0345C5D382970323D7
:10A70000841A2244B2409797FF1F83C7A7D217B578
:10A71000FF1F0355A56B1307401F8146314699451E
:10A720004101028382806D71232481102326111040
:10A7300023229110328401CD8947630AF5028320D8
:10A74000C110032481108324411051618280178538
:10A7500001001305A5DEAE8497500100E780802933
:10A76000A285268597A0FFFFE780E05BC9BFB7E71A
:10A770000400FC4728008297178501001305C5DCFB
:10A7800097500100E78000278347810039C41307F1
:10A79000000B6380E7021387A7051377F70F8D4639
:10A7A00063EDE602A285280097B0FFFFE7806067AF
:10A7B00079B78547E3F587F8834591001775010060
:10A7C0001305C59FB335B00097A7FF1F238EB78C25
:10A7D00097500100E780200A9DB703479100A20728
:10A7E000B966D98F1387E6556384E70C636DF70468
:10A7F0002D671307B755638FE708636AF70029676A
:10A800001307A755638FE708A2852800A1BF31670A
:10A810001307C7556388E70635671307D755E395D0
:10A82000E7FE8947E3FD87F097000000E780A0E995
:10A830009305E4FFC205C1811305A1009790FFFFB6
:10A84000E780009AEDBD3D671306F7556389C7069B
:10A85000636DF6009386E665E398D7FAA285280033
:10A8600097C0FFFFE780E0A2D9BD9306F766638D2E
:10A87000D7041307F777E399E7F897C0FFFFE7805E
:10A8800080CE75BD0146A285280097C0FFFFE780F6
:10A89000E08475B5A285280097C0FFFFE78000908F
:10A8A00079BDA285280097C0FFFFE780609341BD76
:10A8B000A285280097C0FFFFE780A09449B597C004
:10A8C000FFFFE78020A6A5BD97C0FFFFE780C0ABD4
:10A8D000BDB5C16717B5FF1F0355454FF91763078E
:10A8E000F500B7E7040003A3C7170283828017F3BC
:10A8F000FFFF6700E35C1773FFFFE702A37C2A8476
:10A9000008452E89B28919C900C1971500009385A1
:10A91000A586610597300100E780000981447D5AD2
:10A9200097100000E780E03963C7A40481449710C2
:10A930000000E780003A63C8A40497B7FF1F93871D
:10A94000A7499C43DC47B307F94091872302F400F1
:10A95000638309048327C900B307F4409587A302E2
:10A96000F4001C4C89C79C4799C3228582971773B2
:10A97000FFFF670063785C44139714008504BA975F
:10A980002390470171BF1C48139714008504BA97A0
:10A990002390070069BF832789000547B307F44068
:10A9A0009587A302F40083570400638EE7028DC3EA
:10A9B00009476384E7040D47E395E7FA97870100A9
:10A9C0009387470B1CCC978701009387A70B11A88F
:10A9D00097870100938787D11CCC978701009387C5
:10A9E000E7D15CC8BDBF97870100938727BD1CCC0A
:10A9F00097870100938787BDEDB7978701009387FD
:10AA0000270C1CCC978701009387870CD9BF95E54D
:10AA10001773FFFFE702A36C0046184483479400B6
:10AA200075839D8B6317F70097100000E78060B473
:10AA300048C41773FFFF6700C36C82801773FFFF62
:10AA4000E702436813893500C16442094111AA89AC
:10AA50000144F11413590901054A2EC6971000004C
:10AA6000E7802026B2456348A400014541011773E1
:10AA7000FFFF6700636883A7090013171400BA97E4
:10AA800083D707006388B7006394970063742A0133
:10AA90000504E1B70545D9BF1773FFFFE702A361BE
:10AAA000AA892E89328BB6843A8ABE8A97A0000082
:10AAB000E780A00271C9268597200000E780A010DA
:10AAC0008D4763E7A7007D551773FFFF670023627B
:10AAD00083DB440097100000E780A0242A849710AD
:10AAE0000000E78040259307740031443305850258
:10AAF00063CDA70297100000E780A0229710000006
:10AB0000E78020222A8497100000E780C022930764
:10AB1000740031443305850263C3A7049710000015
:10AB2000E78020209307450029A897100000E780C0
:10AB30008020330585021307F0179307C017E35FE2
:10AB4000A7FA2D55E3C277F963040B02D686528625
:10AB5000A6854A8597200100E780A0C1B5B7971068
:10AB60000000E780401D330585029307C5FFD1BF74
:10AB7000832749001385C90083D52700970000006B
:10AB8000E78000EC61F581B769553DBF97B7FF1FBE
:10AB90002396A72497B7FF1F9387072490438147E5
:10ABA0000C463307F500420741836393B700828068
:10ABB0005446139847008507C2962390E600D5B700
:10ABC00097B7FF1F938747219C4303C58700828067
:10ABD00017B5FF1F0355852082801773FFFFE7021B
:10ABE0000350C1671387D7FF630BE502636AA700B1
:10ABF000F1176300F50201451773FFFF670063500B
:10AC00001387E7FF6302E502FD171D8D133515005D
:10AC1000E5B797500000E780402E7D15C5BF9750DF
:10AC20000000E780C002D5BF97500000E780E00039
:10AC3000EDB71773FFFFE702834A4111AA8401446D
:10AC40002EC697100000E780C008B2456348A400F4
:10AC5000014541011773FFFF6700A34A9C48131584
:10AC600014003E9583570500E385B7FE0504C9BF70
:10AC700003485500814693F7F60F63E507018147C6
:10AC80003E858280584593975600BA9703D7270090
:10AC90006316B70003D70700E304C7FE8506E1BFCC
:10ACA0008346450001479377F70F63E4D700814758
:10ACB00011A81C45131657000507B29703D60700C5
:10ACC000E313B6FE3E8582801773FFFFE702833FE2
:10ACD00093170501C18797BAFF1F938AEA0F635B39
:10ACE000F00883A70A00C0479C4703570400198D4A
:10ACF000420541816368F500014422851773FFFF17
:10AD00006700833F12052A94CDBFDC4713944900A6
:10AD1000014A3E94834744006341FA02014A834753
:10AD200054006349FA028509C20993D9090183A72E
:10AD30000A009847E3EBE9FCC1B71C4413195A0019
:10AD4000A6853E994A8597000000E780C0EE05E1A0
:10AD5000050AC9B75C4413195A00A6853E994A856D
:10AD600097000000E78020ED19E1050A4DBFE30CD4
:10AD700009FA61B7AA8481495DBF1773FFFFE70233
:10AD800003361C452A8481E79307C5001CC51C4473
:10AD9000231204001CC09307F00F63EDB70093F576
:10ADA000F50F228597200000E780A0E91773FFFFC9
:10ADB0006700233593940501C167C18063F9F500ED
:10ADC000A685228597200000E780C0ECC5B7C18129
:10ADD00093F5F50F228597200000E78080E6A68591
:10ADE000228597200000E780C0E7C9B797B7FF1F0B
:10ADF000938787FE884382801C4599C797B7FF1FBA
:10AE000023ACA7FC014582807D55828097B7FF1F48
:10AE1000938787FC984383474500484792073E95B0
:10AE200082801773FFFFE702832B617100451C18B6
:10AE30003EC6B70780013EC81C183ECA835744006F
:10AE400002CE02D002CC231EF100834784002A895F
:10AE500002D22301F1023C083ED402D69700000042
:10AE6000E78000FB835705002316F102975000008E
:10AE7000E780E0CB2307A1025C4003556400F18327
:10AE800013F717008347F10252055181F99BD98FBF
:10AE9000A307F10297100100E780007D39CDAA8455
:10AEA0000355050097A00000E78000C483D7040085
:10AEB0002AD26800231CF10083D72400231DF1004F
:10AEC0001C4803D647008C4397200000E78080D4BD
:10AED0008347B400CA86177601001306A667811758
:10AEE000A305F4006C00481097200100E7806088FB
:10AEF0005D611773FFFF6700C3202155D5BF1C4557
:10AF0000B1CF03C5A700894613576500630BD7026D
:10AF10008D46630ED70285466300D70213074006AD
:10AF20003305E50203C7B700418B15CB83C7B700D4
:10AF3000BD8B3355F54082801375F5031307803EB2
:10AF4000C5B709671375F50313070771D1BF372715
:10AF500009001375F5031307077CD9B701458280F3
:10AF60001773FFFFE702A31703A98500630C090409
:10AF70008347B900AE8493F7070E85C30345990054
:10AF8000930520030D810505B305B50288446105CD
:10AF900097300100E78060B135A02E859700000052
:10AFA000E78020F62A8419CD97000000E780605CD6
:10AFB0008325C900B307B54063FA87002E94B30513
:10AFC000A440E9F51773FFFF6700A31385457DBF14
:10AFD0001773FFFFE702A3102A8403D505000111B0
:10AFE00032C636C43AC22EC002CA02CC02CE97A0E4
:10AFF0000000E78060AF82452ACA22852ECC9700E8
:10B000000000E780E0E003570500231EE1009750B1
:10B010000000E780C0B1A24632469247230FA1004C
:10B0200036874C08B2862285014697000000E780EB
:10B03000E0A605611773FFFF6700A30C1773FFFFFE
:10B04000E702E30961711C183EC6B70780013EC8DC
:10B050001C183ECA3C0800453ED4AA8402CC02CE4D
:10B0600002D002D202D697000000E78060DA835750
:10B07000050035592316F10297500000E78020ABF8
:10B080002307A10209C48357440081EB21594A8553
:10B090005D611773FFFF6700C30603556400520527
:10B0A000518197100100E780205C2A8965D1834790
:10B0B000B40093F7070E99C7130584019730010078
:10B0C000E780E0A083574400231EF10083478400FB
:10B0D0002301F1025C4003550900D98313F70708E7
:10B0E00083471102231CA10093F7F707D98FA30010
:10B0F000F10283572900231DF1005C40F18313F70F
:10B1000017008347F102F99BD98FA307F10297A09B
:10B110000000E780609D2AD235D9834794006800FB
:10B12000139757008347B400FD8BD98FA305F40014
:10B130001C4803D647008C4397200000E78080AD71
:10B14000A687177701001307E740740005464C10E7
:10B15000268597000000E78060942A890DD98347EF
:10B16000B400A685FD8BA305F40097000000E780DE
:10B1700060DF31BF1773FFFFE70263F6832485FEAC
:10B180002A844111268597000000E78080D78347F5
:10B1900034FF93F7070E8DCB2AC626859700000053
:10B1A000E78060C809CD834734FFB245FD8BA30912
:10B1B000F4FE91C5228597300100E780008F4101A0
:10B1C0001773FFFF6700E3F37DD98327C4FF26854C
:10B1D000829775F5834734FF93F7070E91C7228551
:10B1E00097300100E780A08E032584FE97000000C1
:10B1F000E78000E5E9B71773FFFFE70243EB9C41E7
:10B2000041112A8903C7070089472E849356670096
:10B210006380F6040D466388C6049307F007630451
:10B22000F7022E8597200000E78040AFAA8481496D
:10B23000C16B130C490097B7FF1F9387E7B99C4375
:10B24000984763E4E90441011773FFFF6700E3E9EE
:10B2500003D745008547E3F8E7FE2E8597200000D9
:10B26000E78020B1E1B703D74500E3FEE7FC2E8578
:10B2700097200000E78080AAAA84228597200000FA
:10B28000E780E0ABC204C98C5DB7DC470355A90079
:10B29000139A49003E9A93170501C187635DF00038
:10B2A00083570A006397A70263E774038327CA00E2
:10B2B000034D5A002DA0A1672167A98F1307F7EF4F
:10B2C000E374F7FE6397090097000000E780209180
:10B2D00061FD85098DB783278A00034D4A00835D90
:10B2E000A90003576900216A138BC7003AC6814A37
:10B2F00033CA4D01631E5D0197B7FF1F938747AEA9
:10B300009C43E1DBA2866286814526858297D1B780
:10B31000A1679387F7EF930C4BFF63F24703B245A6
:10B320005A8597F0FFFFE780A0710DC103278B00BE
:10B33000104709CE10436382C4023107D5BFEE85A2
:10B34000668597000000E780008F71F993861A00E8
:10B3500093FAF60F130B0B0271BF835644005C4344
:10B36000E3E9F6F622853AC697200000E7800085DB
:10B37000A1679387D7042A8A035D4400324763E8B4
:10B3800097008347D90093E707F8A306F9001C4705
:10B3900066852286E2858297C1670844FD17337A65
:10B3A000FA00529508C02312A40125B797B7FF1FD2
:10B3B000938787A29843814715C31447814763FF4A
:10B3C000D500939745004C47BE9519C903C7550052
:10B3D00081476375E600DC451606B2973E8582809C
:10B3E00003C745008147E37BE6FE16069C45F5B79B
:10B3F0001773FFFFE70203CDAA892E8A814497BA0B
:10B40000FF1F938A6A9D83A70A00984763E6E400BA
:10B410001773FFFF670043CEDC47139444000149D4
:10B420003E9413BB140083474400634BF900014969
:10B4300013BB140083475400634FF9008504E1B740
:10B440000844931759005287DA860146A2853E9533
:10B4500082990509C9BF4844931759005287DA8673
:10B460000546A2853E9582990509E9B71773FFFF46
:10B47000E702E3C6814517F5FFFF1305054897B7B7
:10B48000FF1F239D079497000000E780A0F6177325
:10B49000FFFF670003C797B7FF1F9387E7939C439E
:10B4A00095C31773FFFFE70283C3814517F5FFFFBD
:10B4B0001305A54497000000E780C0F31773FFFF52
:10B4C000670023C482801773FFFFE702A3BF37E43E
:10B4D00004008327841241112315E100AE893289CB
:10B4E000368A3A8681460147ED45AA8482972AC664
:10B4F00021C90356A100D28597400100E780402C66
:10B500008327C413CE8526858297058905C983279D
:10B51000440D2314210101462C00268582972A849C
:10B5200001C9B7E7040083A7C712ED452800829739
:10B53000228541011773FFFF670003BC4944D5B75B
:10B540006554FDB75C41FD175CC182801773FFFF36
:10B55000E702E3B8B7E70400FC5F8297954733053D
:10B56000F50281450D811773FFFF670083B91773DB
:10B57000FFFFE702C3B6B7E70400FC5F8297954779
:10B580003305F5020D811773FFFF670083B717734B
:10B59000FFFFE702C3B4B7E7040083A7870B035597
:10B5A000050082971773FFFF6700A3B51773FFFFAE
:10B5B000E702E3B2035505003287AE861786FF1F08
:10B5C0000356A6EF97B5FF1F9385C581970000002E
:10B5D000E780A0EF1773FFFF6700A3B21773FFFFA9
:10B5E000E702E3AFB7E7040083A7C7178297177393
:10B5F000FFFF670003B11773FFFFE70243AEB7E732
:10B60000040083A7871397A5FF1F9385A57D8297C5
:10B6100001451773FFFF6700C3AE1773FFFFE70213
:10B6200003ACB7E7040083A7C71F81451785FF1F39
:10B630000355A5E482971773FFFF670083AC177368
:10B64000FFFFE702C3A9B7E7040083A7871397A505
:10B65000FF1F9385257A829701451773FFFF6700C7
:10B6600043AA1773FFFFE70283A7B7E7040083A786
:10B67000C71F81451785FF1F035525E6829717735E
:10B68000FFFF670003A81773FFFFE70243A52E859E
:10B6900097800000E78060B797800000E78060F443
:10B6A0001773FFFF6700E3A51773FFFFE70223A3EC
:10B6B00097800000E78060FE1773FFFF670063A4B8
:10B6C0005C49E1175CC95CC583572501A1072319B3
:10B6D000F50083570501A1072318F5008280F14783
:10B6E0003305F50297A7FF1F9387C7729C433E95CA
:10B6F00082808D476315F60803D74600854763F0BF
:10B70000E7081773FFFFE702839D368536842E898D
:10B7100097100000E780806029C983574400931484
:10B720000501C18063E39704228597100000E7803C
:10B73000E05EFD14231294009307A0026300F5025B
:10B740009307B0026307F50293079002631FF500A9
:10B75000228597000100E780408D01A80146CA8537
:10B76000228597A00000E780E0B71773FFFF67000E
:10B770004399228597100000E780400BFDB7828037
:10B7800097A6FF1F938646699C42014599CF98432F
:10B79000D44217A6FF1F2321E6686396D70097A619
:10B7A000FF1F23ADE6661385C7FE82801773FFFF78
:10B7B000E702E39297000000E780A04B7144330555
:10B7C0008502914597900000E780A0F011E565554E
:10B7D0001773FFFF6700E39297A7FF1F23AAA762D3
:10B7E00097000000E780E048330585029145979077
:10B7F0000000E78000EE61DD97A7FF1F23ACA76084
:10B8000097000000E780E04697A7FF1F239CA75EF4
:10B8100097000000E780E04597A7FF1F2395A75EEC
:10B8200097770100938747D817A7FF1F2320F75E5C
:10B8300097070000938707E917A7FF1F2326F75CE8
:10B84000014579B71773FFFFE7026389AA8517A53A
:10B85000FF1F1305255B97100000E78040631773F7
:10B86000FFFF6700038A1773FFFFE7024387970014
:10B870000000E78060FD97100000E780C06297A796
:10B88000FF1F938767599C4391CF1387C7FE19CB3E
:10B8900083D5C7FF17A5FF1F130585589720010003
:10B8A000E780A0201773FFFF6700A3851773FFFFD2
:10B8B000E702E38297000000E780C0EC09CD8347F0
:10B8C00085002A8493F7070499EB0355E500970058
:10B8D0000000E78080F91773FFFF670083828347CA
:10B8E000C5009304450117A9FF1F1309E95285E319
:10B8F000832709005CC997A7FF1F23AF97508327B1
:10B900004900F1FB97A7FF1F23AA9750E9B7FD173E
:10B910002306F500610597800000E78040DE83077D
:10B92000840063CB07048347840093E707F823046C
:10B93000F400B7E704009C5F82974205A947418164
:10B940003375F5028347840093F707FCC98F2304FE
:10B95000F4008347D4003E951C402318A40089CFEF
:10B96000984319CB8347C400504081458507330570
:10B97000F502420541810297832709005CC897A719
:10B98000FF1F23AB97488327490089E797A7FF1F2D
:10B9900023A697488347C4009DDF8355040117A55C
:10B9A000FF1F1305E54797200100E780001025B72A
:10B9B0001763FFFFE702A37297A7FF1F9387876BA9
:10B9C0009C4701448583858B85E3AE84B2853A86A6
:10B9D00097100000E78000532A8419C597100000D3
:10B9E000E7804049829408CC22851763FFFF6700F7
:10B9F00043711763FFFFE702E36C41112E8932C6E2
:10BA0000AA8997000000E780C0313247130605027B
:10BA1000CA86970500009385C5CC17A5FF1F13059F
:10BA2000653E97000000E780E0F82A8425C993046A
:10BA3000C50097000000E780E0411946AA852685E9
:10BA400097100000E780001D8545268597100000AF
:10BA5000E780E018177501001305C5B24E958345C0
:10BA60000500268597100000E780A01D5C48314640
:10BA70008145A1075CC85CC483572401E1172319E1
:10BA8000F40083570401E1172318F4001C4C3E8591
:10BA90009760FFFFE780A067A3042501228541018D
:10BAA0001763FFFF670043651763FFFFE702236328
:10BAB0004111AA842EC632C497100000E780E03DF1
:10BAC000004DB2452246834784000CC050C093F716
:10BAD000F70393E707042304F400231804002685E2
:10BAE00097100000E780003983479400A946231788
:10BAF000A40013D7370005073307D7029D8B8507AE
:10BB00002306F400A306E40083C70401D848850790
:10BB1000230FF7FE17A7FF1F130707305843232AE9
:10BB200004009307440129E317A7FF1F2328F72EDA
:10BB300017A7FF1F2322F72E17A4FF1F1304442E5D
:10BB4000228597200100E78080E81C44858B5D8D6D
:10BB500019E58145228597200100E78000F5410124
:10BB60001763FFFF6700E3591CC317A7FF1F2327B5
:10BB7000F72AD9B71763FFFFE7026356970500005E
:10BB8000938565B7014597000000E78000B0014547
:10BB90001763FFFF6700E3561763FFFFE7022354B5
:10BBA00097000000E78080B01763FFFF67006355D0
:10BBB0008347C500A5E31763FFFFE70243522A84CA
:10BBC0000355E50097000000E78000C821C18347C6
:10BBD000840093F7F7FB2304F4001C4091C7DC4377
:10BBE00081C74C400145829797000000E78080B9EB
:10BBF00017A5FF1F1305C52297200100E78020ED40
:10BC00000355E40097000000E78020C61763FFFF9C
:10BC10006700234F82801763FFFFE702434C97A71B
:10BC2000FF1F9387671F97050000938565C817A5B9
:10BC3000FF1F1305E51E23A0070023A2070097207E
:10BC40000100E78060D61763FFFF6700834B1C4D40
:10BC500091CFDC4381CF1763FFFFE7024348834561
:10BC6000070082971763FFFF6700A349828097A7A9
:10BC7000FF1F9387271D9C4303C50700828097A75A
:10BC8000FF1F9387271C9C4303C51700828097A73B
:10BC9000FF1F9387271B9C4303C52700828097A71C
:10BCA000FF1F9387271A9C4303C54700828097A7ED
:10BCB000FF1F938727199C4303C53700828097A7EE
:10BCC000FF1F938727189C4303C55700828097A7BF
:10BCD000FF1F938727179C4303C56700828097A7A0
:10BCE000FF1F938727169C4303C57700828097A781
:10BCF000FF1F938727159C4303C58700828097A762
:10BD0000FF1F938727149C4303C59700828097A742
:10BD1000FF1F938727139C4303C5A700828097A723
:10BD2000FF1F938727129C4303C5B70011E11D45F0
:10BD3000828097A7FF1F9387E7109C4303C5C70026
:10BD4000828097A7FF1F9387E70F9C4303C5D70007
:10BD5000828097A7FF1F9387E70E9C4303C5E700E8
:10BD6000828097A7FF1F9387E70D9C4303D50701A8
:10BD7000828097A7FF1F9387E70C9C4303C5270189
:10BD8000828097A7FF1F9387E70B9C4303D547014A
:10BD9000828097A7FF1F9387E70A9C4303D567011B
:10BDA000828097A7FF1F9387E7099C4303D58701EC
:10BDB000828097A7FF1F9387E7089C4303C5A701CD
:10BDC000828097A7FF1F9387E7079C4303C5B701AE
:10BDD000828097A7FF1F9387E7069C4303C5C7018F
:10BDE000828097A7FF1F9387E7059C4303C5D70170
:10BDF000828097A7FF1F9387E7049C438857828020
:10BE000097A7FF1F938707049C4303D5C70282802F
:10BE100097A7FF1F938707039C4303D5E70219E108
:10BE20001305800C828097A7FF1F9387A7019C436F
:10BE300003C50703828097A7FF1F9387A7009C4332
:10BE4000C85B828097A7FF1F938747FF8843828044
:10BE500097A7FF1F9387C7FE8843828019E17D550E
:10BE60008280F5DE984265DFFDD917A7FF1F130713
:10BE700067201847AA877155058B631D072403C5E2
:10BE800007001547E37DA7FC03C737001305F0053E
:10BE90007D171377F70FE364E5FC03C35700E30056
:10BEA00003FC83C86700E38C08FA03C777004945A1
:10BEB00079171377F70FE364E5FA03C7A700114872
:10BEC0001305F7FF1375F50FE36BA8F803CE970082
:10BED0000D481305FEFF1375F50FE362A8F803C8BC
:10BEE000B7006309080065181378F80F1305600D93
:10BEF000E36705F703C5C700794879151375F50F92
:10BF0000E36FA8F403C8D7000D457D181378F80F28
:10BF1000E36705F503D80701930E4017511842084F
:10BF200013580801E3ED0EF303C8E7007D181378FA
:10BF3000F80FE36605F303C827017D181378F80F9F
:10BF4000E36F05F103C88700C54E75181378F80F25
:10BF5000E3E70EF103D86701856E938EBEE06D189E
:10BF6000420813580801E3EC0EEF03D847016D189F
:10BF7000420813580801E3E40EEF03D8870179184B
:10BF8000420813580801E36C05ED03C8A7017D18AA
:10BF90001378F80FE36505ED03C5B7011D487D155E
:10BFA0001375F50FE36DA8EA03C5D701714879153C
:10BFB0001375F50FE365A8EA03D5E7011308E00F51
:10BFC0007D1542054181E36CA8E803C50702494895
:10BFD00079151375F50FE364A8E8C85301C937C88C
:10BFE00034005915130858BFE36BA8E603A887026D
:10BFF00037C53400130555BF5918E36205E717A587
:10C00000FF1F232FC5E203C6050117A5FF1F232B22
:10C01000F5E20545E375C5E403D82501D04933763B
:10C020000603E31E06E203C61501E30A06E217A6AD
:10C03000FF1F2325B6E083C5270001466387A500BF
:10C0400003C61700F1453306B60283C707039305FD
:10C05000C00272971A071307C70516031A979608A6
:10C060004697B387B70241553E97329742074183BF
:10C070006362E8061763FFFFE70263063685978071
:10C080000000E780207097000100E780A04F2A841D
:10C0900097A00000E78000622A9497F00000E780F4
:10C0A000E02D2A9497900000E78020892A9497F049
:10C0B000FFFFE780E06F2A9497400000E780E09A56
:10C0C0002A9497700000E78020A422951763FFFF51
:10C0D0006700230382801763FFFFE70243004111DB
:10C0E000A307A10097A00000E78020CD9305F100F1
:10C0F000170500001305E5B597F0FFFFE780802FD7
:10C10000014541011763FFFF6700A3FF1763FFFFAE
:10C11000E70263FA17A4FF1F1304C4F50328840081
:10C1200079599368180097A4FF1F23A914F5137871
:10C13000180063100802BA84BE89368B328A2E89B1
:10C14000AA8A97F0FFFFE780E0A77D15269519E5FD
:10C1500031594A851763FFFF670063F997F0FFFFC6
:10C16000E78040A67D152695A167E353F5FE97A7C6
:10C17000FF1F9387272798433E8C814B01CB0145B6
:10C1800097F00000E780A04B933B15004A85DA86C4
:10C190005686D28597900000E78040552A8911CDB8
:10C1A0001C44F99B17A7FF1F232AF7EC83270C00D9
:10C1B000CDD3E3800BFA829769BF268597A7FF1F2F
:10C1C00023AC07EA97F0FFFFE780809C4146CE85CD
:10C1D00017A5FF1F130585F397300100E780405E28
:10C1E00097D00000E780C0A00325040B97D0000083
:10C1F000E78080A4054597D00000E78080AB054527
:10C2000097000000E78060EDA9B797A7FF1F93870D
:10C2100067E69C47858BEDC71763FFFFE70223ECBA
:10C2200017A5FF1F1305C5EC97A7FF1F23A407E45D
:10C2300097A7FF1F23A207E497A7FF1F23A007E4E8
:10C2400097200100E780A08897500000E78060FDFC
:10C2500097100100E780205497100100E780205AD2
:10C2600097A7FF1F938787DF9C4391C7054597805A
:10C270000000E780C02797A7FF1F9387E7C79C436D
:10C2800099C741657D1597700000E780C0A997F0B8
:10C290000000E780604597D00000E780009797A7EF
:10C2A000FF1F938727F29C431397170163560700DC
:10C2B00097F00000E78080B497A7FF1F23A807E44A
:10C2C00097A7FF1F23A607E497A7FF1F23A407E450
:10C2D00097A7FF1F23A207E497000000E780008CC8
:10C2E00097000000E780807997F0FFFFE780401813
:10C2F00097F00000E780C0DD1763FFFF670063E091
:10C30000828097A7FF1F9387E7D68843828097A7ED
:10C31000FF1F938727D6C8438280B7E7B000938773
:10C32000075063E1A70297A7FF1F9387A7D4D843BD
:10C33000FD576367E50097A7FF1F23AFA7D281478B
:10C340003E858280B957EDBF1763FFFFE70223D90F
:10C3500097800000E780407997800000E780A07B0D
:10C360001763FFFF6700E3D917A7FF1F130787D0E5
:10C370008325470B1DC51763FFFFE70243D697A729
:10C38000FF1F938727AC9C432A8403C61700B7E797
:10C390000400FC470E06829722851763FFFF6700A3
:10C3A00043D62E8582801763FFFFE702A3D12A843C
:10C3B0009304140201112E85B289A685214636C642
:10C3C0003A8997300100E780403D0DE9B2463808D0
:10C3D0002686CE851305940497500000E7806041BF
:10C3E00021462C084A8597300100E780003B133531
:10C3F000150005611763FFFF670003D00145D5BF36
:10C400001763FFFFE702A3CD9305450617A5FF1F9E
:10C41000130585A397100100E78020691763FFFFCC
:10C42000670023CE1763FFFFE70263CB41112EC6DF
:10C4300097F0FFFFE780E013B24588C14101176321
:10C44000FFFF670003CC1763FFFFE702A3C7AA84BF
:10C450002E8497800000E780006CAA89854522859C
:10C4600097000000E780E07D83C7E401138994080A
:10C4700099E313890403CE85228597000000E780A5
:10C48000407C214693051902228597000000E78031
:10C49000607897A7FF1F9387E7BD8C43228597108D
:10C4A0000000E780C08221469385840222859700A0
:10C4B0000000E78020761763FFFF6700E3C3176380
:10C4C000FFFFE70243BF397197F00000E780E0B457
:10C4D0009305400661E997800000E78000606302F1
:10C4E000051497A7FF1F83C7E79713B7170097A6F1
:10C4F000FF1F2389E696014499CFC16417A9FF1F46
:10C50000130949B79309400EFD1497F0FFFFE78028
:10C51000407F6342A40A97F0FFFFE78080054169EE
:10C52000B7290900096AFD7A2A8B81447D1993890C
:10C53000F97B130A0A71938A8AC797F0FFFFE78095
:10C54000407C63D7A4041304400EB387840217A76A
:10C55000FF1F130727B20324070B3E948357C40120
:10C560006382270B18403307EB4063EAE9008347F7
:10C5700044008507B3874703D6976365F7080146EC
:10C580008145094597F0FFFFE780E046AA8B29E542
:10C5900097400000E780808385476317F50689652B
:10C5A0009385057117A5FF1F1305058A97100100D4
:10C5B000E780A04F95A0B30734030327090BBA9770
:10C5C00003D7C7016308970003C75700A38207007A
:10C5D0002382E700050415BF9305C5002285970057
:10C5E0000000E78080E65E852286976501009385DE
:10C5F000A5FA97F0FFFFE780604B5E85971000007B
:10C60000E780608A850415BF97A7FF1F938787A6D9
:10C610009C478D83858BC1F721611763FFFF6700FE
:10C6200003AD01468545094502D002D202D402D6A7
:10C6300097F0FFFFE780203CAA8479DD97F00000A7
:10C64000E780E09C1389C4002A8481454A859700CD
:10C650000000E780005F0C4041464A8597000000DB
:10C66000E780405B832944006385090C4E8502D82E
:10C6700002DA02DC02DE97300100E780E0382ACEE1
:10C68000141005462C0808184ECC97500000E7807F
:10C69000E00A1375F50F51ED8355840093E52500ED
:10C6A0004A8597000000E780E05E11460C104A853D
:10C6B00097000000E78000560146976501009385CA
:10C6C00025EE268597F0FFFFE780403E2685970000
:10C6D0000000E780407D5C40A1D3014685450D45C3
:10C6E00097F0FFFFE7802031AA841DD548401389C9
:10C6F000C40097300100E78020312AC64A859700A0
:10C700000000E780404C3246636FC5004C404A85CC
:10C7100097000000E780005001468145268597F08C
:10C72000FFFFE780A038268597000000E780A0770C
:10C73000E5B583558400ADB71763FFFFE702239A81
:10C7400097A7FF1F938707939C471DC193E7870017
:10C750001795FF1F1305456F17A7FF1F2320F7929B
:10C7600097100100E78040321763FFFF670063996D
:10C77000DD9B17A7FF1F2323F79097300000E7806A
:10C78000E0647DF11795FF1F1305056C97100100FC
:10C79000E780E033D1BF1763FFFFE702C391416930
:10C7A000AA892E8AB28A368BBA8B814417ACFF1FB6
:10C7B000130C4C8C930C400E7D1997F0FFFFE78013
:10C7C000405463C4A40001443DA0338494038327F0
:10C7D0000C0B3E948357C401638627055A87D6867F
:10C7E0005286CE851305040397000000E780E0BB66
:10C7F00001C923800B0022851763FFFF6700238F89
:10C800008347F40185C35A87D6865286CE851305A1
:10C81000940897000000E78040B909C58547238048
:10C82000FB00D1BF850451BF835745006380071EBD
:10C830001763FFFFE702038901112A8497000000B4
:10C84000E780C04D09C985476309F506056117638F
:10C85000FFFF6700638A97E00000E780007C7DF5BA
:10C86000835744004947ED9BE392E7FEC14522858B
:10C8700097000000E7804033AA84228597000000DB
:10C88000E780204F0357440002CE91472A89631A5C
:10C89000F700228597000000E780A0513C082ACCD1
:10C8A0003ECE97E00000E78080765C55C5D37408E3
:10C8B0004A86A6850545829751BF03574400D14754
:10C8C000E3F6E7F8032A0400C1690149979AFF1FBC
:10C8D000938A4A7A130B400EFD1997F0FFFFE78009
:10C8E0004042634FA90E2285032A040097000000EE
:10C8F000E780C042A1452A89228597000000E78091
:10C90000A02AAA84228597000000E780804A14406C
:10C910002A86AA8978082685CA8597000000E780BC
:10C92000C0E7AA8405D503C7F40189476315F7005A
:10C930008347C10181DF5546D28513856400973056
:10C940000100E780E0E7014597800000E780C0191B
:10C9500001C583D7C401A5E79797FF1F9387877108
:10C960009C4793551900858913D73700058B01CF54
:10C970008983858B6399B70001452EC69700000017
:10C98000E780C0DBB2454E8597800000E780601FDE
:10C990000346C1012A8493751900268597900000EB
:10C9A000E780E03935C1268597800000E780E018F0
:10C9B000268511C0014597800000E780004C973024
:10C9C0000000E780A0408547E312F5E883C75400E4
:10C9D0001307F00FE38CE7E68507A382F400BDB5EB
:10C9E000B304690383A70A0BBE9483D7C401638B86
:10C9F00037015546D2851385640097300100E780E2
:10CA0000C0D955DD0509D1BD5DD86DB782801753FA
:10CA1000FFFFE702236B97800000E780000C05C151
:10CA2000C16401441799FF1F1309C9649309400E9B
:10CA3000FD1497F0FFFFE780C02C634EA40017950C
:10CA4000FF1F1305654097100100E780E0031753AF
:10CA5000FFFF6700636A330534038327090B3E95A4
:10CA60008357C50163889700231205009780000053
:10CA7000E780A00C050475BF9797FF1F9387875F1A
:10CA80009C478D83858B8DE31753FFFFE70223655A
:10CA90001795FF1F1305453B97100100E780200302
:10CAA0001753FFFF6700E36582801753FFFFE7021C
:10CAB0000363970500009385C5A01795FF1F130515
:10CAC000A53897100100E78020EE1753FFFF67009D
:10CAD00043631753FFFFE70283608841B7E7040011
:10CAE000BC5B050542054181829709C58547230046
:10CAF000F50005051753FFFF6700A36083C7F5FF27
:10CB00002E858507A38FF5FE828083C7F5FFFD176D
:10CB100093F7F70FA38FF5FE99EF1753FFFFE70287
:10CB2000035CB7E70400BC571385F5FF82971753E2
:10CB3000FFFF6700035D82801C41035745008D8F16
:10CB4000BA951CC12312B5003E85828093D785001B
:10CB5000A2051441DD8D835745001387E6FF18C1F8
:10CB600089072312F50013D685004111238FB6FEE5
:10CB7000A38FC6FE4101828018419307F7FF1CC1B5
:10CB80008357450085072312F500A30FB7FE828067
:10CB9000835745008D8F2312F5001C41BE950CC1B3
:10CBA0002E858280AA8703D7470008410D8FAA955A
:10CBB0002392E7008CC38280184108453305A740C3
:10CBC000828083574500035765001D8F1C4108452F
:10CBD0003385A7403305A74082801753FFFFE70244
:10CBE000035041112EC62A8497000000E780A0FD63
:10CBF000B2456373B50001A0835744000840BE9559
:10CC00002312B4003E9541011753FFFF6700634FA5
:10CC10001753FFFFE702A34C41112E84B28532C6A1
:10CC200097000000E780A0FB3246A2859730010004
:10CC3000E78000B941011753FFFF6700834C17538A
:10CC4000FFFFE702C3492E84854597000000E78077
:10CC500000F9230085001753FFFF6700834A17532D
:10CC6000FFFFE702C34741112317B1008945970031
:10CC70000000E780C0F68347E1002300F50083470A
:10CC8000F100A300F50041011753FFFF6700634760
:10CC90001753FFFFE702A34493D78500A205411174
:10CCA000DD8D2317B100894597000000E78020F350
:10CCB0008347E1002300F5008347F100A300F5005E
:10CCC00041011753FFFF6700C3431753FFFFE702FC
:10CCD00003411397850193D78501C166938606F0BA
:10CCE000D98F13D78500758FD98FA2053707FF001D
:10CCF000F98D4111DD8D2EC6914597000000E7802A
:10CD000000EE6C00114697300100E78060AB4101F6
:10CD10001753FFFF6700E33E1753FFFFE702233C73
:10CD20001C41854503C4070097000000E78080E6AA
:10CD300022851753FFFF6700C33C1753FFFFE7022D
:10CD4000033A1C414111894503C7070083C71700F7
:10CD50002307E100A307F10097000000E78080E3CC
:10CD60000355E10041011753FFFF67008339175353
:10CD7000FFFFE702C3361C414111894503C7070085
:10CD800083C717002307E100A307F1009700000005
:10CD9000E78040E08357E100410113D58700A207F7
:10CDA0005D8D420541811753FFFF6700833517539F
:10CDB000FFFFE702C3320C4141112A84114668008B
:10CDC00097300100E780C09F9145228597000000C1
:10CDD000E78040DCB247C166938606F0139787016F
:10CDE00013D58701598D13D78700758F598DA207E9
:10CDF0003707FF00F98F5D8D41011753FFFF670073
:10CE000043301C45BE950CC18280AE87944391E6A9
:10CE1000584101EF0CC15CC1828003C75700136702
:10CE20001700A382E700B687D5B70CC3EDB7AA8772
:10CE3000084119CD1841D44398C36313D500D8C312
:10CE40002A87034657009376160081E623200700C1
:10CE50008280944381CA8C4203A847008CC36393A9
:10CE60000601CCC3799A14C3A302C7003687D1BF89
:10CE70001C45DC471D8DB777DBB6938777DB0985CB
:10CE80003305F502420541818280F147B385F50201
:10CE900048452E9582808347450085072302F5008B
:10CEA00082801753FFFFE70283232A8409E4175384
:10CEB000FFFF6700032583474400F5DBFD1793F769
:10CEC000F70F2302F400E5F71C4403D727000507FA
:10CED0002391E700DC4399C3228582974C4889CD92
:10CEE00083475400898B99E71C4422859C479C43C7
:10CEF0009C478297232A04000040232004007DB72A
:10CF00001753FFFFE702A31D8357250041112EC6CB
:10CF100081EB0144228541011753FFFF6700631E27
:10CF2000035705008147F146E305F7FEB385D702B5
:10CF3000404585072E948345440008C4F5F5B24763
:10CF4000AA8481E7232A040009A81C456C002285D5
:10CF50009C439C43829748C84DDD85472312F400CB
:10CF6000B24723200400231804002319F4005C486E
:10CF70005CC483D72400FD172391F40061BF1753CD
:10CF8000FFFFE702C3159797FF1F9387E7ED8843DD
:10CF90002326050023240500410597100100E780A2
:10CFA00000B31753FFFF6700C3151753FFFFE702D6
:10CFB00003131794FF1F130424EB1C40411199CF56
:10CFC0009C472300B5002AC65CC197000000E7809B
:10CFD00040FB1C40DC4399C3324582974101175303
:10CFE000FFFF670003120347450029E3584DAA8756
:10CFF0007D551DCF1753FFFFE702630E1CC3DC47AF
:10D000009796FF1F23A2E6E6F1561305070123902A
:10D01000D700970500009385050297100100E7806F
:10D02000A09801451753FFFF6700A30D7D5582802F
:10D0300082801753FFFFE702830A01116146814591
:10D0400028009750FFFFE780800C9797FF1F93877A
:10D05000A7E19C4328009305F00FDC473EC69700EC
:10D060000000E780C0F405611753FFFF6700630904
:10D070009797FF1F938747DF9C43D847A167938704
:10D08000C702631EF70A397106DE22DC26DA800049
:10D090004AD84ED652D456D23285B2849700000078
:10D0A000E780C0C7AA89268597000000E78020C9CD
:10D0B0002318A4FC268597000000E78040C82319A8
:10D0C000A4FC268597000000E78060C783D7440052
:10D0D0000A8A231AA4FC858393F7F70F230EF4FC26
:10D0E0008607BD0793F7073F3301F1408A8A01495C
:10D0F0008347C4FD6367F902CE85130584FC232CA6
:10D1000054FD97000000E78080EA5281130104FC7F
:10D11000F2506254D2544259B259225A925A216161
:10D120008280268597000000E78060C19317190070
:10D13000D69705092390A7001379F90F55BF828070
:10D140009797FF1F938747D29C43D847A167938740
:10D15000A702631AF70A397106DE22DC26DA80009C
:10D160004AD84ED652D456D23285B28497000000A7
:10D17000E780C0BAAA89268597000000E78020BC16
:10D18000FD572318A4FC26852319F4FC9700000002
:10D19000E780E0BA83D744000A8A231AA4FC858377
:10D1A00093F7F70F230EF4FC8607BD0793F7073FAD
:10D1B0003301F1408A8A01498347C4FD6367F9025C
:10D1C000CE85130584FC232C54FD97000000E780D6
:10D1D00000DE5281130104FCF2506254D2544259D1
:10D1E000B259225A925A2161828026859700000006
:10D1F000E780E0B493171900D69705092390A7009C
:10D200001379F90F55BF82809797FF1F9387C7C582
:10D210009C43D847A16789076310F70A397106DE76
:10D2200022DC26DA80004AD84ED652D456D2328535
:10D23000328997000000E78060AEAA894A8597008E
:10D240000000E780C0AF835749000A8A2318A4FC76
:10D25000858393F7F70F230CF4FC8607BD0793F73C
:10D26000073F3301F1408A8A8144834784FD63E7A5
:10D27000F402CE85130584FC232A54FD9700000098
:10D28000E780E0D25281130104FCF2506254D25480
:10D290004259B259225A925A216182804A85970096
:10D2A0000000E780C0A993971400D69785042390C7
:10D2B000A70093F4F40F55BF82809797FF1F9387C1
:10D2C000A7BA9C43D847A1679387E704631EF70A70
:10D2D000397106DE22DC26DA80004AD84ED652D4D6
:10D2E00056D23285B28497000000E78020A3AA8935
:10D2F000268597000000E78080A42318A4FC2685DB
:10D3000097000000E780A0A3231AA4FC26859700BD
:10D310000000E780C0A283D744000A8A2319A4FC36
:10D32000858393F7F70F230EF4FC8607BD0793F769
:10D33000073F3301F1408A8A01498347C4FD63678F
:10D34000F902CE85130584FC232C54FD97000000C0
:10D35000E780E0C55281130104FCF2506254D254BC
:10D360004259B259225A925A2161828026859700E9
:10D370000000E780C09C93171900D69705092390F9
:10D38000A7001379F90F55BF82809797FF1F9387E6
:10D39000A7AD9C43D847A1679387C704631AF70AD0
:10D3A000397106DE22DC26DA80004AD84ED652D405
:10D3B00056D23285B28497000000E7802096AA8971
:10D3C000268597000000E7808097FD572318A4FC6E
:10D3D0002685231AF4FC97000000E780409683D747
:10D3E00044000A8A2319A4FC858393F7F70F230EC0
:10D3F000F4FC8607BD0793F7073F3301F1408A8AA3
:10D4000001498347C4FD6367F902CE85130584FC97
:10D41000232C54FD97000000E78060B9528113016E
:10D4200004FCF2506254D2544259B259225A925AD0
:10D4300021618280268597000000E7804090931745
:10D440001900D69705092390A7001379F90F55BF46
:10D4500082809797FF1F938727A19C43D847A16796
:10D46000DD076317F7041753FFFFE70243C779711E
:10D470003285328497000000E780408A2AC62285E0
:10D4800097000000E780A08B2311A102228597005E
:10D490000000E780A088B2452300A1022808970079
:10D4A0000000E780C0B045611753FFFF670063C508
:10D4B00082809797FF1F9387279B9C43D847A1673C
:10D4C000938787046317F7041753FFFFE70223C10D
:10D4D00079713285328497000000E78020842AC663
:10D4E000228597000000E78080852311A102228514
:10D4F00097000000E7808082B2452300A10228083F
:10D5000097000000E780A0AA45611753FFFF67005E
:10D5100043BF82809797FF1F938707959C43D84707
:10D52000A1679387A7046312F7021753FFFFE7026F
:10D5300003BB01112800814597000000E78020A768
:10D5400005611753FFFF6700C3BB82809797FF1FDA
:10D55000938787919C43D847A167938757026319A4
:10D56000F7021753FFFFE70283B70111328597F0E7
:10D57000FFFFE780A07A2308A100814528009700DB
:10D580000000E780C0A205611753FFFF670063B783
:10D5900082809797FF1F9387278D9C43D847A16769
:10D5A0009387E702631BF7041753FFFFE70223B3D8
:10D5B00001113285328497F0FFFFE7804078AA841A
:10D5C000228597F0FFFFE7808077854709E922856C
:10D5D00097F0FFFFE78080744205B337A000280072
:10D5E0008145231891003ECA97000000E780209CE7
:10D5F00005611753FFFF6700C3B082809797FF1F35
:10D60000938787869C43D84799476313F708175336
:10D61000FFFFE702C3AC79713285328497F0FFFFD8
:10D62000E780C06F2AC6228597F0FFFFE780207150
:10D630002310A102228597F0FFFFE780206E2301CF
:10D64000A102228597F0FFFFE780406DA301A102B0
:10D65000228597F0FFFFE780606C2302A1022285FC
:10D6600097F0FFFFE780806B2313A102228597F0DC
:10D67000FFFFE780A06AB2452314A10228089700A3
:10D680000000E780C09245611753FFFF670063A762
:10D6900082809787FF1F9387277D9C43D847A16788
:10D6A0009387C7036313F7081753FFFFE70223A30A
:10D6B00079713285328497F0FFFFE78020662AC6B1
:10D6C000228597F0FFFFE78080672310A102228563
:10D6D00097F0FFFFE780A0662311A102228597F053
:10D6E000FFFFE780A0632302A102228597F0FFFFDE
:10D6F000E780C062A302A102228597F0FFFFE780C6
:10D70000E0612303A102228597F0FFFFE78000611B
:10D71000B245A303A102280897000000E7802089F2
:10D7200045611753FFFF6700C39D82801753FFFFBA
:10D73000E702E39A01112A8497F0FFFFE780005E79
:10D74000AA84228597F0FFFFE780605F228597F02B
:10D75000FFFFE780C05E035744008D4763F7E70093
:10D76000228597F0FFFFE780805D228597F0FFFF1D
:10D77000E780E05C2800A68597000000E780208312
:10D7800005611753FFFF6700C3979787FF1F9387B4
:10D79000A76D9C43D847A167FD07631FF700175388
:10D7A000FFFFE702C393328597000000E78040F84F
:10D7B0001753FFFF6700E39482809787FF1F9387CB
:10D7C000A76A9C43D847A167E5076315F708175375
:10D7D000FFFFE702C39079713285328497F0FFFF33
:10D7E000E780C0532AC6228597F0FFFFE7802055C7
:10D7F000228597F0FFFFE78080542310A102228545
:10D8000097F0FFFFE780A053520551812311A10239
:10D8100022852302010297F0FFFFE7802050A30238
:10D82000A102228597F0FFFFE780404F2303A1026A
:10D83000228597F0FFFFE780604EB245A303A10267
:10D84000280897F0FFFFE780807645611753FFFFB8
:10D850006700238B82809787FF1F9387E7609C4335
:10D86000D847A1679387E703631FF7001753FFFFAC
:10D87000E702E386328597000000E78060EB1753EC
:10D88000FFFF6700038882809787FF1F9387C75D2C
:10D890009C43D847A16793874704631EF702175339
:10D8A000FFFFE702C38379713285328497F0FFFF6F
:10D8B000E780C0462AC6228597F0FFFFE780204810
:10D8C000B245280897F0FFFFE780606E4561175367
:10D8D000FFFF6700038382809787FF1F9387C758E6
:10D8E0009C43D847A167938787026310F7041743C7
:10D8F000FFFFE702C37E79713285328497F0FFFF24
:10D90000E780C0412AC6228597F0FFFFE7800041EB
:10D91000B2452300A102280897F0FFFFE7802069A5
:10D9200045611743FFFF6700C37D82801743FFFFF8
:10D93000E702E37A011197F0FFFFE780203EAA8516
:10D94000280097F0FFFFE780806605611743FFFF1F
:10D950006700237B9787FF1F938707519C43D84716
:10D96000A167D107631FF7001743FFFFE702237783
:10D97000328597000000E780A0FB1743FFFF670098
:10D98000437882809787FF1F9387074E9C43D84731
:10D99000A167C507631FF7001743FFFFE702237462
:10D9A000328597000000E780A0F81743FFFF67006B
:10D9B000437582809787FF1F9387074B9C43D84707
:10D9C000A167B907631FF7001743FFFFE702237141
:10D9D000328597000000E780A0F51743FFFF67003E
:10D9E000437282809787FF1F938707489C43D847DD
:10D9F000A167AD07631FF7001743FFFFE702236E20
:10DA0000328597000000E780A0F21743FFFF670010
:10DA1000436F82809787FF1F938707459C43D847B2
:10DA200089476318F7021743FFFFE702436B0111B1
:10DA3000328532C897F0FFFFE780402EAA85280084
:10DA400097F0FFFFE780A05605611743FFFF6700CF
:10DA5000436B82809787FF1F938707419C43D8477A
:10DA6000A1678D076311F7041743FFFFE7022367E0
:10DA700001113285328497F0FFFFE780202A1306D8
:10DA80006100AA844C00228597300000E780C02303
:10DA90002800A68597F0FFFFE780605105611743D6
:10DAA000FFFF6700036682809787FF1F9387073C0D
:10DAB0009C4381CFDC4391CB1743FFFFE7022362F6
:10DAC00082971743FFFF6700C36382801743FFFFFE
:10DAD000E702E36079713C08AE843ED2A165B707E6
:10DAE0000A002A843ED448103C08DD053ED636C4E0
:10DAF00032C63AC297D0FFFFE7806028124748102D
:10DB0000BA8597F0FFFFE780C01332464810B28510
:10DB100097F0FFFFE780E014A2464810B68597F023
:10DB2000FFFFE7800012501001478146A68522853D
:10DB300097D0FFFFE780004A45611743FFFF67006A
:10DB4000435C1743FFFFE702835901117C0003295F
:10DB5000C501AE843ECAA165B70707002A843ECC42
:10DB600048087C00C5053ECE97D0FFFFE780202106
:10DB70008345D900480897F0FFFFE780800C5008E4
:10DB800001478146A685228597D0FFFFE780804424
:10DB900005611743FFFF6700C3561743FFFFE70206
:10DBA000035483C7950093F7F707A384F500970004
:10DBB0000000E78040F91743FFFF670083541743D5
:10DBC000FFFFE702C35179713C08AE843ED2A165E4
:10DBD000B70709002A843ED448103C0893854504C1
:10DBE0003ED632C636C497D0FFFFE7804019A24622
:10DBF0004810B68597F0FFFFE780A0043246481032
:10DC0000B28597F0FFFFE780C005501001478146BD
:10DC1000A685228597D0FFFFE780C03B456117436B
:10DC2000FFFF6700034E1743FFFFE702434B83C725
:10DC3000950041112A8493F7F707A384F5003285F4
:10DC40002EC697F0FFFFE780800F85672AC46370B8
:10DC5000F50297700000E78020E92246B24509ED01
:10DC600011478146228597000000E78060E6410168
:10DC70001743FFFF6700E34801478346F501DDB71F
:10DC80001743FFFFE702034401113C003ECAB707F8
:10DC90000A003ECC3C003ECE83C79500AA8932855F
:10DCA00093F7F707A384F5002E8497F0FFFFE78032
:10DCB00000098567637DF504A165AA8493858504C1
:10DCC000480897D0FFFFE780800B268597700000FB
:10DCD000E78080E12A8929E19145480897F0FFFF14
:10DCE000E78020F6A685480897F0FFFFE78060F7F9
:10DCF000CA85480897F0FFFFE780A0F401478146F6
:10DD00005008A2854E8597D0FFFFE780A02C0561C3
:10DD10001743FFFF6700433E8145480897F0FFFF28
:10DD2000E78020F20349090275BF1743FFFFE702AE
:10DD3000633979711C103ECAB7070F003ECC404DC5
:10DD40001C10AA84AE894808994532C636893ECE51
:10DD500097D0FFFFE780A00232464808B28597F0CF
:10DD6000FFFFE78000EE630C0902A545480897F025
:10DD7000FFFFE780C0E62546CA8597200100E780BF
:10DD800020A4500801478146CE85268597D0FFFF05
:10DD9000E780402445611743FFFF6700E335835563
:10DDA000C402480897F0FFFFE780A0EB0355E402A8
:10DDB000814505C5854785456301F502C167FD17A6
:10DDC0009305F00F630BF5007D1597700000E78059
:10DDD000208E9305150093F5F50F480897F0FFFF87
:10DDE000E78020E683450403480897F0FFFFE780BB
:10DDF00040E583451403480897F0FFFFE78060E49F
:10DE000083552403480897F0FFFFE78080E583559A
:10DE10004403480897F0FFFFE780A0E49DB717434D
:10DE2000FFFFE702C32B83C795008146014693F7A6
:10DE3000F707A384F50097000000E78040EF174341
:10DE4000FFFF6700032C1743FFFFE70243297971A7
:10DE50003E841C103ECA2E89B7070F00A1653ECC38
:10DE6000FD051C10AA84480842C03AC23ECE36C402
:10DE700032C697D0FFFFE78080F032464808B2856F
:10DE800097F0FFFFE780E0DBA2464808B68597F0F1
:10DE9000FFFFE78000DD12474808BA8597F0FFFFD3
:10DEA000E78020DC0248630C08029145480897F09F
:10DEB000FFFFE780C0D21146A28597200100E780CE
:10DEC0002090500801478146CA85268597D0FFFFDC
:10DED000E780401045611743FFFF670083228945B3
:10DEE000480897F0FFFFE78080CF834704002300B6
:10DEF000F50083471400A300F500E1B71743FFFFC7
:10DF0000E702431C83C7950001112A8A93F7F7079C
:10DF1000A384F5003285AE8432C697F0FFFFE78018
:10DF200000E232462A89328597F0FFFFE78000DF62
:10DF300085676373F902AA894A8597700000E780B4
:10DF4000A0BA2A8419ED114781464A86A6855285D2
:10DF500097000000E780C0B705611743FFFF670027
:10DF6000A3199387E9FF93F7F70F0547E366F7FED9
:10DF70008347F50195EB8947E380F9FE8346F40179
:10DF8000528501474A86A68597000000E78040B485
:10DF9000A167D90748083ECC230A010002CE9700AA
:10DFA0000000E780A0B04DBF639EE7008947639EF5
:10DFB000F90093071020231FF50097700000E780F9
:10DFC000C0B76DBF0947E39BE7FA8D47E398F9FABD
:10DFD000228597700000E78080DF9787FF1F938777
:10DFE000E7079C4399E79787FF1F9387E7F09C43D8
:10DFF00099C703D5040097800000E780A0CE231FB7
:10E00000040022855DBF1743FFFFE702430D0111A6
:10E010003C003ECAB7070B003ECC3C003ECE83C757
:10E0200095002A89328593F7F707A384F500AE841B
:10E0300097F0FFFFE780A0D093170501C187635ACF
:10E04000F006A1652A849385E502480897D0FFFF72
:10E05000E780E0D2A285480897F0FFFFE78060C024
:10E060009787FF1F938747E99C43A9EB014493756A
:10E07000F40F480897F0FFFFE780A0BC9355844059
:10E0800093F5F50F480897F0FFFFE78080BB9355A5
:10E09000044193F5F50F480897F0FFFFE78060BA59
:10E0A000014781465008A6854A8597D0FFFFE78043
:10E0B00060F205611743FFFF6700A30441658546D1
:10E0C0000546A2857D1597500000E78060BD59DDAB
:10E0D000510597000100E780808F13044006334408
:10E0E000850271B71743FFFFE70263FF0111B7070E
:10E0F00006003EC683C7950021642A8993F7F70777
:10E10000A384F500AE8428009305A4040AC40AC8B9
:10E1100097D0FFFFE780A0C6300001478146A68563
:10E120004A8597D0FFFFE780E0EA97E0FFFFE780AE
:10E13000000E13049404480822CC230A010002CEE6
:10E1400097000000E780809605611743FFFF670096
:10E1500043FB1743FFFFE702E3F6C1642A8901444A
:10E160009789FF1F938909F1130A8002FD1497E034
:10E17000FFFFE78000BA6347A40001451743FFFF94
:10E18000670083F7B307440303A7C90ABA9703D705
:10E1900007006306970083D72700638427010504DF
:10E1A000F9B70545E1BF1743FFFFE702A3F12A8A4C
:10E1B0002E8999C123A0050081498144978AFF1FB8
:10E1C000938A0ACB614B97E0FFFFE780C0BA63C731
:10E1D000A4004E851743FFFF670003F233846403F6
:10E1E00083A70A003E948357040099E7630409005B
:10E1F000232089008504C1BF4146D2851305440010
:10E2000097100100E780605975F5A289E5B71743BB
:10E21000FFFFE70223EB39717C083ED4B7070A0001
:10E220003ED67C083ED883C795002A8A328593F76C
:10E23000F707A384F5002E8932C697F0FFFFE78029
:10E2400000B085676373F5083246AA84328597F07B
:10E25000FFFFE780A0AC8547AA8963E8A706A16510
:10E2600093858504281097D0FFFFE78040B126856D
:10E2700097700000E78040872A8429ED9145281097
:10E2800097F0FFFFE780E09BA685281097F0FFFF3F
:10E29000E780209DCE85281097F0FFFFE780609AE9
:10E2A000014781463010CA85528597D0FFFFE7802D
:10E2B00060D2A1679387770448183EDC230A0102E5
:10E2C00002DE97F0FFFFE780607E21611743FFFFCA
:10E2D000670083E28145281097F0FFFFE780609692
:10E2E000A685281097F0FFFFE780A0979787FF1F6C
:10E2F0009387070F9C4381CB22856389090097D0C0
:10E300000000E78040248345040271B797D00000E5
:10E31000E780C022CDBF1743FFFFE702A3DA83C720
:10E3200095004111AA8993F7F707A384F500328578
:10E33000AE84328A97F0FFFFE78060A08567637F35
:10E34000F5022A8997600000E780007A2A849146C6
:10E3500031C58347F50105476387E70291C70D473C
:10E360006366F704AD461DA89305050303250A005F
:10E37000414697100100E78040420DE941011743F3
:10E38000FFFF670063D79305950803250A00414600
:10E3900097100100E7806040814669F54A86A685AE
:10E3A0004E8597000000E780C081C9BF83250A0021
:10E3B0001305940897700000E780A02919C1C14691
:10E3C000F1BF9787FF1F938767C99C4399E797879A
:10E3D000FF1F938767B29C4399C7228597800000EF
:10E3E000E780208A69FD8547A30FF400228597B056
:10E3F0000000E7806084228597600000E780E0737A
:10E400004E8581464A86A68597F0FFFFE780607BB0
:10E41000A1679387570448003EC42302010002C647
:10E4200097F0FFFFE780806891BF1743FFFFE70287
:10E4300083C883C795004111AA8993F7F707A3847E
:10E44000F50032852E89B28A97F0FFFFE780208F92
:10E4500085676374F50EAA8497600000E780C06842
:10E460002A840DED416B014A978BFF1F938B8BC064
:10E47000130C400E7D1B19A833048A0383A70B0BD2
:10E480003E948357C40163836705050A97E0FFFF45
:10E49000E7802087E342AAFE95460DA08357C50179
:10E4A000639697029305050303A50A00414697105A
:10E4B0000100E780802E994611E181462686CA85B3
:10E4C0004E8597F0FFFFE780C06F85A883A50A00FF
:10E4D0001305040397700000E780A017C14679FD7B
:10E4E0002285231E940097A00000E780E074228517
:10E4F00097600000E78060649787FF1F938747EE6F
:10E500009C43A9C323000402228597D00000E78022
:10E5100040F04E8581462686CA8597F0FFFFE7804A
:10E52000406AA1679387070448003EC423020100A4
:10E5300002C697F0FFFFE780605741011743FFFFD6
:10E540006700E3BA89472300F402E1B7397106DEB8
:10E5500022DC4AD8800052D456D25AD026DA4ED67F
:10E560005ECE2E8A32892A8B97D0FFFFE7806076B5
:10E570000605710541998A8A3301A140232224FCB2
:10E58000231404FC97D0FFFFE780A07483479A0010
:10E590000605350593F7F7072315A4FCA304FA0035
:10E5A0004A85232624FC97E0FFFFE78040799317F4
:10E5B0000501C1876340F0025681130104FCF2504B
:10E5C0006254D2544259B259225A925A025BF24BC7
:10E5D00021618280AA844A8597E0FFFFE780207648
:10E5E000AA894A8597E0FFFFE7806075A16593855A
:10E5F000C5022A89130544FC97C0FFFFE7802078F5
:10E60000268597C0FFFFE780606C854511C94A8663
:10E61000CE8597C0FFFFE780E065AA8B21E9894599
:10E62000130544FC97E0FFFFE780A061A685130572
:10E6300044FC97E0FFFFE780C062CE85130544FCF1
:10E6400097E0FFFFE780E061CA85130544FC97E08F
:10E65000FFFFE780006101478146130644FCD28535
:10E660005A8597D0FFFFE780E096B9B7814513053B
:10E6700044FC97E0FFFFE780C05CA685130544FCDF
:10E6800097E0FFFFE780E05DCE85130544FC97E04F
:10E69000FFFFE780005DCA85130544FC97E0FFFF9C
:10E6A000E780205C814497D0FFFFE7808062E3D45D
:10E6B000A4FA83A70B0113971400BA9783D5070018
:10E6C00099C5130544FC97E0FFFFE7808059850456
:10E6D000D9BF797106D622D44AD000184ECE52CC7A
:10E6E00056CA26D25AC8AE893289AA8A97D0FFFF65
:10E6F000E780205E0605690541990A8A3301A14039
:10E70000232A24FC231C04FC97D0FFFFE780605CD5
:10E7100083C7990006052D0593F7F707231DA4FC71
:10E72000A384F9004A85232E24FC97E0FFFFE780AD
:10E73000006193170501C187634FF00052811301F7
:10E7400004FDB250225492540259F249624AD24A0C
:10E75000424B45618280AA844A8597E0FFFFE780AB
:10E76000005EA1659385A5022A89130544FD97C023
:10E77000FFFFE780C060268597C0FFFFE780005558
:10E78000854509C9CA8597C0FFFFE780A0512A8B3C
:10E7900029E18945130544FD97E0FFFFE780604AC2
:10E7A000A685130544FD97E0FFFFE780804BCA85EF
:10E7B000130544FD97E0FFFFE780A04A014781462B
:10E7C000130644FDCE85568597D0FFFFE7808080F5
:10E7D000B5B78145130544FD97E0FFFFE78060462C
:10E7E000A685130544FD97E0FFFFE7808047CA85B3
:10E7F000130544FD97E0FFFFE780A046814497D0D2
:10E80000FFFFE780004DE3DBA4FA83270B0113979A
:10E810001400BA9783D5070099C5130544FD97E006
:10E82000FFFFE78000448504D9BF1743FFFFE702DD
:10E83000038B83474500404DD5EFFD575DC48346AC
:10E84000940009476363D70A0346B400854663EE24
:10E85000C6088306E40063CA06085C45F95623909F
:10E86000D7009777FF1F83C7E76099E3A304E4000D
:10E870009777FF1F938747689C4381E78947A306E3
:10E88000F4009787FF1F9387A7B59C4381E78947CB
:10E890002306F4009705000093854506AA84130516
:10E8A000040197F00000E7802010FD57231AF402BE
:10E8B00081471CDC01489777FF1F23A9875A977768
:10E8C000FF1F9387E75A232E040304C0804397D089
:10E8D000FFFFE780404A61463306C5028145228535
:10E8E0009740FFFFE780A08281473E851743FFFFE7
:10E8F00067002381FD57D5BF1733FFFFE702237E53
:10E900002A840355450297600000E780E01D19E561
:10E91000231E04001733FFFF6700A37E8357E40123
:10E92000F5DB930504FF174501001305250197E06A
:10E930000000E780E014F9BF1733FFFFE702237AF6
:10E940002E89A16541119385E5032A8436C432C618
:10E95000BE843AC297C0FFFFE7806042124722851B
:10E96000BA8597E0FFFFE780C02D32462285B28549
:10E9700097E0FFFFE780E02EA2462285B68597E06C
:10E98000FFFFE780002E630309029145228597E08F
:10E99000FFFFE780C0241146A68597100100E7809D
:10E9A00020E241011733FFFF6700A37589452285E7
:10E9B00097E0FFFFE780A02283C704002300F50053
:10E9C00083C71400A300F500E9BF1733FFFFE70278
:10E9D000037183C79500444D054793F7F707A38458
:10E9E000F5001C42411183C707006367F7062E84B8
:10E9F0002A89B1C003C7D400630FF7021777FF1F3E
:10EA00001307874F184305C3A386F40097A000009F
:10EA1000E780404A83C7D40099E741657D15974058
:10EA20000000E780403083D72403918B89C797E0AB
:10EA30000000E780C0134A85A28597F0FFFFE780BA
:10EA40008010A167C10748003EC42302010002C62E
:10EA500097F0FFFFE780800541011733FFFF670054
:10EA6000436A1733FFFFE702836703D745008D47EB
:10EA7000AA8441112E8432892E8563E3E70297E050
:10EA8000FFFFE780C02BAA8523000900268597C0D9
:10EA9000FFFFE780202141011733FFFF6700636616
:10EAA00097E0FFFFE780A0292AC6228597E0FFFFB5
:10EAB000E780E028B24585472A862300F9002685AD
:10EAC00097C0FFFFE780001BF9B7397106DE22DC33
:10EAD00026DA80004ED652D456D24AD85AD05ECECC
:10EAE000AE89B284AA8A97D0FFFFE780801D060511
:10EAF0001305250241990A8A3301A140232224FCEF
:10EB0000231404FC97D0FFFFE780A01B83C7990064
:10EB100006054D0593F7F7072315A4FCA384F90018
:10EB20002685232624FC97E0FFFFE78040219317EA
:10EB30000501C1876340F0025281130104FCF250C9
:10EB40006254D2544259B259225A925A025BF24B41
:10EB500021618280AA8B03AB040097C0FFFFE7808E
:10EB6000E01651E583D7440001498544F11793B776
:10EB70001700A301F4FC834734FCA165C9C7938542
:10EB8000E504130544FC97C0FFFFE780401FA685FE
:10EB9000130544FC97E0FFFFE780A00ADE8513051C
:10EBA00044FC97E0FFFFE780C00B834734FC11462D
:10EBB00091E30946DA85130544FC97E0FFFFE780FF
:10EBC00060058144630A0900416B7D1B97D0FFFFFC
:10EBD000E780200F63CCA40201478146130644FC62
:10EBE000CE85568597C0FFFFE780C03EB1B7A685AA
:10EBF000130634FC97000000E780E0E6933415002C
:10EC00002A8986048DBF9385C504A5BF8327C900C3
:10EC100013971400BA9783D507006388650113051D
:10EC200044FC97E0FFFFE780C003850445B7173336
:10EC3000FFFFE702434879711C103EC4B7070F007D
:10EC40003EC61C103EC883C79500AA8A328593F73A
:10EC5000F707A384F500AE89328497E0FFFFE780D1
:10EC6000000E93170501C187635AF0062A8A228590
:10EC700097E0FFFFE780A00C2A895285032B040050
:10EC800097C0FFFFE780800439ED8357440081443B
:10EC90000544F11793B71700A303F10083457100F2
:10ECA000DA872287CA865286280097000000E7800C
:10ECB000E0C8014781463000CE85568597C0FFFFEA
:10ECC000E7804031A1679387D70348083ECC230AE9
:10ECD000810026CE97F0FFFFE78040DD45611733C6
:10ECE000FFFF6700C340A285130671009700000074
:10ECF000E78060D7AA84094455D13544E30055FB29
:10ED00004A8597F0FFFFE78000450D4441D9014453
:10ED100097D0FFFFE780E0FA634DA400C16B014488
:10ED2000FD1B97D0FFFFE780C0F9634EA400154498
:10ED3000B5B7DC4413171400BA9783D70700638371
:10ED400027030504F1B7D84493171400BA9703D7E3
:10ED50000700631B770123902701268597A00000F9
:10ED6000E78080DB01441DBF050465BF1733FFFF4B
:10ED7000E702433583C7950041112A8A93F7F707C5
:10ED8000A384F50032852E89328497E0FFFFE78067
:10ED900000FB93170501C1876353F006AA892285FA
:10EDA00097E0FFFFE780A0F92311A1004E85832A99
:10EDB000040097C0FFFFE78060F139E58357440006
:10EDC00085440144F11793B71700A300F1000348ED
:10EDD000110003572100D6875285CE862686CA8524
:10EDE00097F0FFFFE7806006A167F10748003EC487
:10EDF0002302910022C697F0FFFFE78020CB41015C
:10EE00001733FFFF6700432FA285130611009700F9
:10EE10000000E78040C52A84894455D983572100E2
:10EE200011678544BA97C2071167C1831307F7EFCB
:10EE3000E36FF7F89777FF1F938747229C4381CBB7
:10EE400085451305210097500000E7802075835504
:10EE500021002285814497C0FFFFE780C0DD25D9CE
:10EE600023100500228597A00000E78040CD85B7DC
:10EE70001733FFFFE702232483C7950041112A8B34
:10EE800093F7F707A384F50032852E8A328497E042
:10EE9000FFFFE780C0EA93170501C1876351F006C1
:10EEA000AA8A228597E0FFFFE78060E92A895685D4
:10EEB000832B040097C0FFFFE78040E131E58357D3
:10EEC000440081440544F11793B71700A301F100F2
:10EED00003483100DE875A854A87D6862286D28546
:10EEE00097F0FFFFE78060F6A167ED0748003EC49A
:10EEF0002302810026C697F0FFFFE78020BB410177
:10EF00001733FFFF6700A31EA28513063100970089
:10EF10000000E78040B5AA8409445DD99167CA978B
:10EF2000C2071167C1831307F7EF0544E362F7FADD
:10EF3000CA8597C0FFFFE78000D0014451F981499D
:10EF400097D0FFFFE780E0D863DBA900984893974C
:10EF50001900BA9703D7070005EF2390270197D030
:10EF6000FFFFE78000D71544E384A9F6268597A024
:10EF70000000E780C0BC9777FF1F9387270E9C4354
:10EF80000144B9D74A8597500000E780C05889B737
:10EF900085097DB71733FFFFE702C31279713E84FD
:10EFA0007C083EC82E8AB7071400A1653ECAE50555
:10EFB0007C08AA89080836C4428932C6BA8AC6843F
:10EFC0003ECC97C0FFFFE78080DBCA85080897E04A
:10EFD000FFFFE78000C732460808B28597E0FFFFD1
:10EFE000E78020C8A246630A09049D45080897E007
:10EFF000FFFFE780C0BE1D4681459730FFFFE780D9
:10F00000001163890A089145080897E0FFFFE7802F
:10F0100000BD1146A68597000100E780607A1008C0
:10F0200001478146D2854E8597C0FFFFE78080FA71
:10F0300045611733FFFF6700230CB685080897E08A
:10F04000FFFFE78000C21C400808D8439355C70162
:10F05000858912075183B205D98D97E0FFFFE780BC
:10F0600040C01C40080883C5870097E0FFFFE78089
:10F0700040BD1C40080883C5A70097E0FFFFE7805C
:10F0800040BC1C40080883C5970097E0FFFFE7805D
:10F0900040BB85BF8945080897E0FFFFE78020B4A3
:10F0A00083C704002300F50083C71400A300F50004
:10F0B000BDB71733FFFFE702E30083C79500411197
:10F0C000AA8993F7F707A384F5003285AE843284CA
:10F0D00097E0FFFFE780A0C693170501C187635D36
:10F0E000F0042A89032A040097C0FFFFE78000BECE
:10F0F00019E9835744000548F11793B71700A30790
:10F10000F100814631A81306F100A28597000000A6
:10F11000E78060951DC51C459DC783D64700014803
:10F120000347F10093078500D2884A86A6854E855D
:10F1300097000000E78040E641011733FFFF6700BA
:10F14000A3FB09487DBF1D486DBF1733FFFFE702D2
:10F1500063F765715C083EC4B7077B013EC65C0877
:10F160003EC883C795002A8A328593F7F707A384A0
:10F17000F500AE8997E0FFFFE78040BA8357E100D2
:10F18000E1C78945280097C0FFFFE78040BF814560
:10F19000280097E0FFFFE780C0AA97C0FFFFE78045
:10F1A00020C59777FF1F9387A7239C431774FF1FE2
:10F1B000034444CCAA843334800099C313642400EC
:10F1C0009777FF1F938747D39C4399C313644400E9
:10F1D0009777FF1F938787E89C4399C31364840044
:10F1E00083D504002800014997E0FFFFE78060A76E
:10F1F00083D52400280097E0FFFFE78080A683D511
:10F200004400280097E0FFFFE780A0A597D0FFFF0C
:10F21000E78020A793150501C181280097E0FFFF33
:10F22000E78020A4A285280097E0FFFFE78060A385
:10F230009C446360F902014781463000CE855285C7
:10F2400097C0FFFFE78000D959611733FFFF6700C0
:10F25000A3EADC441314490028003E9497E0FFFF22
:10F26000E7806096834744000347540089070607F8
:10F27000BA978607E36AF5FC835524002800814A83
:10F2800097E0FFFFE780E09D83454400280097E07A
:10F29000FFFFE780009B83455400280097E0FFFFB5
:10F2A000E780209A8347440063C9FA00814A834774
:10F2B000540063C1FA020509A5BF1C4413975A0004
:10F2C0002800BA9783D50700850A97E0FFFFE780FB
:10F2D0004099C9BF032BC40093975A0028003E9B56
:10F2E00083552B00850A97E0FFFFE78080978355C1
:10F2F0000B00280097E0FFFFE780A0964DBF173373
:10F30000FFFFE702C3DD5C4993E717005CC997A0E4
:10F310000000E78020B61733FFFF670083DE173356
:10F32000FFFFE702C3DB2E84814597F0FFFFE780F4
:10F33000C0E705C583570500FD172310F50009C474
:10F34000835725002310F40097000000E78060FB3E
:10F3500001451733FFFF6700C3DA31457DD823101D
:10F360000400C5BF1733FFFFE702C3D583C795006D
:10F3700041112A8A93F7F707A384F50032852E8975
:10F38000328497E0FFFFE780809B93170501C187D8
:10F390006356F006AA89C145228597E0FFFFE78002
:10F3A000A0802A8B4E85832A040097C0FFFFE78048
:10F3B000E09131E983574400231101000544F1171E
:10F3C00093B71700A300F1008144034811000357CD
:10F3D0002100D6875285CE862286CA8597F0FFFF08
:10F3E000E780A0A6A1679387170248003EC42302C6
:10F3F000810026C697E0FFFFE780406B410117338D
:10F40000FFFF670063CF13061100A28597F0FFFF8F
:10F41000E7806065AA8409E523110100094475B7F6
:10F42000930521005A8597000000E78080EF8357FD
:10F4300021002A84D9DB9777FF1F938727C29C433B
:10F4400081CB85451305210097500000E78000150A
:10F45000835521002685314497B0FFFFE780A07DCA
:10F460002DD523100500268597900000E780206D9C
:10F470000144A1BF1733FFFFE70263C641112E8984
:10F480006C00AA8402C697F0FFFFE78000D20DC18E
:10F490000357050005072310E50097000000E780EB
:10F4A00040E681473E8541011733FFFF670063C592
:10F4B0003247954765DBCA85268597300000E7808F
:10F4C000400DC147E34005FE3244854741462310C5
:10F4D000F40083570900A685130544002311F400A6
:10F4E00097000100E780C02D228545BF1733FFFF3D
:10F4F000E70243BD83C795004111AA8A93F7F70736
:10F50000A384F5003285AE89328497E0FFFFE7805F
:10F51000008393170501C1876356F0062A8AC14507
:10F52000228597D0FFFFE7802068AA845285032BAD
:10F53000040097B0FFFFE780607931E9835744000A
:10F54000231101008544F11793B71700A300F100C0
:10F5500001440348110003572100DA875685D286FB
:10F560002686CE8597F0FFFFE780208EA1679387E0
:10F57000070248003EC42302910022C697E0FFFF25
:10F58000E780C05241011733FFFF6700E3B6A28551
:10F590001306110097F0FFFFE780E04C2A8409E58D
:10F5A00023110100894475B7268593052100970032
:10F5B0000000E78060ECAA8449FD83552100228584
:10F5C00097B0FFFFE780206749F5014997C0FFFF2B
:10F5D000E7802070635DA900184893171900BA9757
:10F5E00003D707000DEF035721002390E70097C0D2
:10F5F000FFFFE780006E630625039777FF1F938761
:10F60000E7A59C4399C70355210097500000E78068
:10F6100080F0228597900000E78060521DBF0509A9
:10F6200075B795443DB705C19307F00F630FF5001B
:10F63000C547630CF5009307F5FF05453315F50045
:10F640004205418182800145828041657D1582802D
:10F65000B9E91733FFFFE70283A8034506033284A5
:10F6600097000000E78060FC9305803EB305B5027B
:10F67000C205C18181CD0357E402854763F8E700E5
:10F680001305040197E00000E78020428357E4025D
:10F6900041677D176385E700FD172317F4021733D1
:10F6A000FFFF670003A682801733FFFFE702A3A0D6
:10F6B000004283C79500444D0349140093F7F707B0
:10F6C000A384F50083470400220911673369F90018
:10F6D000A167B347F90041112A8BAE8A63ECE70EAC
:10F6E000834724001307C00EB91793F7F70F63730E
:10F6F000F71003473400C14763EEE70E8347440029
:10F700001307E00793C707086371F70C8349840068
:10F7100083477400A209B3E9F900856763F7F90A22
:10F72000034A6400834754004E85220A336AFA0074
:10F7300097500000E780403B61C123962403834B30
:10F740003400137AFA00239A34032388740323992C
:10F75000440393890401631C090023A6040223982F
:10F7600004024E8597E00000E78060363DA0034923
:10F7700024004A8597000000E78020EB2397A4022D
:10F78000834744004E85A388F402E38D0BFCE30B12
:10F7900009FC97E00000E780202F97900000E780A9
:10F7A000007381460146D6855A8597E0FFFFE780C2
:10F7B0000058A167938797033EC4230201004800C5
:10F7C00002C697E0FFFFE780602E41011733FFFF7D
:10F7D0006700E3918544A2862686D6855A8597E000
:10F7E000FFFFE780C054A167938797033EC42302BD
:10F7F0009100F1B7BD44C5B79144F1BF1733FFFF86
:10F80000E702438C01111C08404D3EC2B7070F00B0
:10F810003EC41C083EC62A89AE8997C0FFFFE78018
:10F8200020D3585C1C5C6346B70E6394E50063E22A
:10F83000A70E3385A740B3B7A700B305B74013069B
:10F84000803E81469D8D97000100E78080B793142C
:10F850000501C180A1659385C503480097B0FFFFEE
:10F86000E780E0518145480097D0FFFFE780603D89
:10F8700083550404480097D0FFFFE780803E8355FE
:10F880002404480097D0FFFFE780A03D814589CC44
:10F89000C167FD179305F00F6388F4002685975024
:10F8A0000000E780E0E0AA85480097D0FFFFE780EE
:10F8B000403903554404814501CDC167FD179305C7
:10F8C000F00F6307F50097500000E78060DEAA851F
:10F8D000480097D0FFFFE780C036834564044800A6
:10F8E00097D0FFFFE780E03583457404480097D048
:10F8F000FFFFE7800035500001478146CE854A85ED
:10F9000097B0FFFFE780006D05611723FFFF6700D9
:10F91000A37E814481B71723FFFFE702437C83C79F
:10F92000950093F7F707A384F50097000000E780A0
:10F9300020ED1723FFFF6700C37C1723FFFFE702BB
:10F94000637883C795004111404D93F7F707A3846F
:10F95000F5002A8A3285B284AE8997D0FFFFE7800E
:10F96000003E2A8B268597D0FFFFE780403D2A89FD
:10F97000268597D0FFFFE780603A93170B0163CA93
:10F980000702E177CA97C207C183116763E3E70201
:10F9900093070910C207C1831307B00F637BF700F9
:10F9A00093170901C187AA8A634AF000C54763FE1D
:10F9B000570141011723FFFF6700037497B0FFFF52
:10F9C000E7804021E31725FFD5B763080B026306E4
:10F9D0000902814463890A02B7077F002310640586
:10F9E000231124057CC0568597000000E780E0C302
:10F9F0009304803EB304950239A0B7077F0023200B
:10FA000004047CC081440355240497E00000E7808F
:10FA1000A0A3A1C497C0FFFFE78080B3269593D72A
:10FA2000F44133379500AE97BA9708DC5CDCCE859D
:10FA3000528597000000E780A0DC99E023220404AF
:10FA4000A1679387B70348003EC42302010002C6A2
:10FA500097E0FFFFE7808005A9BF814701481CDCD4
:10FA6000232E0403E9B71723FFFFE702436797C07C
:10FA7000FFFFE7804030E1473305F502914597509D
:10FA80000000E78000C5E55711C59767FF1F23A158
:10FA9000A73E81473E851723FFFF670083668547A2
:10FAA0001767FF1F2308F73C82801723FFFFE70239
:10FAB00003639767FF1F9387673B80433DC083576E
:10FAC00004046390A70683572404639CB704368913
:10FAD000B28497C0FFFFE780A0A75C5C63C3B70454
:10FAE0006395B7001C5C63EEA7028347640463F36D
:10FAF000F400A6872303F4048347740463F3970098
:10FB0000A687A303F4048357440441677D176385E4
:10FB1000E70085072312F4043C4481C7CA85268583
:10FB200082971723FFFF6700C35D9767FF1F9387C7
:10FB3000E7339C43014599C303C58700828017239F
:10FB4000FFFFE702C3590111B70707003EC683C78D
:10FB50009500584D0AC493F7F7070AC8A384F50027
:10FB60002A89AE8411CB1C4283C707002304F70007
:10FB700097900000E7800034216493055402280028
:10FB800097B0FFFFE780A01F97000000E78020FAF2
:10FB9000AA85280097D0FFFFE780A00A3000014720
:10FBA0008146A6854A8597B0FFFFE780A0421304EF
:10FBB0004402480822CC230A010002CE97E0FFFF4E
:10FBC000E780C0EE05611723FFFF6700835317230B
:10FBD000FFFFE702C35001117C003ECAB7070700D0
:10FBE0003ECC7C003ECE83C795002E84AA8493F73A
:10FBF000F707A384F500A16593855502480897B0DF
:10FC0000FFFFE780C01797000000E78040F2AA8559
:10FC1000480897D0FFFFE780C0025008014781469F
:10FC2000A285268597B0FFFFE780C03A05611723BC
:10FC3000FFFF6700034D9767FF1F938727239C43B0
:10FC4000094599C303C5970082809767FF1F938773
:10FC5000E7219C43094599C303C5D7008280976774
:10FC6000FF1F9387A7209C43014599C303C5A700A5
:10FC700082801723FFFFE702E3440111B707080062
:10FC80003EC683C79500404D0AC493F7F7070AC8DC
:10FC9000A384F5002A89AE8429C41442854703C78A
:10FCA000060063E0E70A83479400094681496380C0
:10FCB000C702B307F740A304E400B339F00083C7D9
:10FCC00016002305F40097900000E780A01E03575C
:10FCD0002403058B19C76386090097D00000E780CD
:10FCE00000E9216493058402280097B0FFFFE780B4
:10FCF000000997000000E78040F4AA85280097D00B
:10FD0000FFFFE78000F497000000E78080F5AA85F8
:10FD1000280097D0FFFFE780C0F2014781463000FE
:10FD2000A6854A8597B0FFFFE780C02A13047402B6
:10FD3000480822CC230A010002CE97E0FFFFE780AB
:10FD4000E0D605611723FFFF6700033B1723FFFF82
:10FD5000E702E33801117C003ECAB70708003ECC39
:10FD60007C003ECE83C795002E84AA8493F7F707C4
:10FD7000A384F500A16593858502480897B0FFFF2D
:10FD8000E780E0FF97000000E78020EBAA854808A5
:10FD900097D0FFFFE780E0EA97000000E78060EC83
:10FDA000AA85480897D0FFFFE780A0E950080147DF
:10FDB0008146A285268597B0FFFFE780A0210561D7
:10FDC0001723FFFF6700E3339767FF1F9387070A37
:10FDD0009C43014599C303C5B70082801723FFFFE9
:10FDE000E702E32F0111B70707003EC683C795005E
:10FDF000404D0AC493F7F7070AC8A384F5002A897F
:10FE0000AE8405C81C42054783C707006368F70630
:10FE10000347B400630FF700A305F40097900000B8
:10FE2000E78040098347B400B9CF97D0FFFFE78050
:10FE300040BE21649305B400280097B0FFFFE7801F
:10FE400000F497000000E78060F8AA85280097D0AA
:10FE5000FFFFE78000DF014781463000A6854A8525
:10FE600097B0FFFFE78000172904480822CC230A37
:10FE7000010002CE97E0FFFFE78040C30561172332
:10FE8000FFFF6700032897D0FFFFE78020BF55B72B
:10FE90001723FFFFE702A32401117C003ECAB70726
:10FEA00007003ECC7C003ECE83C795002E84AA84FA
:10FEB00093F7F707A384F500A165AD05480897B04F
:10FEC000FFFFE780C0EB97000000E78020F0AA85E5
:10FED000480897D0FFFFE780C0D650080147814609
:10FEE000A285268597B0FFFFE780C00E0561172326
:10FEF000FFFF670003219767FF1F938727F79C4346
:10FF0000094599C303C5C70082801723FFFFE70295
:10FF1000031D01117C00AE843ECAA165B70707002E
:10FF20002A843ECCD1057C0048083ECE97B0FFFF26
:10FF3000E780E0E497000000E78020FCAA854808FD
:10FF400097D0FFFFE780E0CF500801478146A685A4
:10FF5000228597B0FFFFE780E00705611723FFFFC9
:10FF60006700231A1723FFFFE702631783C7950073
:10FF700093F7F707A384F50097000000E78020F9C6
:10FF80001723FFFF6700E3171723FFFFE702831321
:10FF900083C795000329C501411193F7F707A3848F
:10FFA000F5001C4283C90700854763E6370797675A
:10FFB000FF1F9387E7429C432E84AA8485CF970036
:10FFC0000000E78080F389476306F50263040902B5
:10FFD0008347C900638037032306390197900000E7
:10FFE000E78040ED83572903898B89C797D00000AC
:10FFF000E780E0B72685A28597000000E78020F122
:020000040001F9
:10000000A167CD0748003EC42302010002C697E065
:10001000FFFFE780A0A941011723FFFF6700C30D81
:100020009767FF1F938787E49C431D4599C303C5CA
:10003000E70082801723FFFFE702630A0111B70779
:1000400007003EC683C79500584D0AC493F7F707CB
:100050000AC8A384F5002A89AE8415C71C4283C749
:10006000070093968701E18663C40606854663818F
:10007000D7068346E7006388F6002307F7009790CA
:100080000000E78020E321649305E400280097B096
:10009000FFFFE780C0CE97000000E780A0F8AA85A8
:1000A000280097D0FFFFE780C0B9014781463000A4
:1000B000A6854A8597B0FFFFE780C0F13504480860
:1000C00022CC230A010002CE97E0FFFFE780009ECA
:1000D00005611723FFFF6700C3021723FFFFE70235
:1000E000030001117C003ECAB70707003ECC7C002C
:1000F0003ECE83C795002E84AA8493F7F707A38486
:10010000F500A165B905480897B0FFFFE78020C753
:1001100097000000E78000F1AA85480897D0FFFF0C
:10012000E78020B2500801478146A285268597B016
:10013000FFFFE78020EA05611723FFFF670063FCEC
:100140001723FFFFE70203F8AA8401441769FF1F82
:10015000130909D2E14997C0FFFFE780C0C163449A
:10016000A400014519A833053403832709003E95EF
:10017000835725006397970011051723FFFF67003A
:10018000A3F70504C9BF032E8500630A0E12176387
:10019000FF1F1303A3EC032303006315030029438C
:1001A0006390061203234E01631503001D436399F8
:1001B00007101723FFFFE70203F0C689428A3E8932
:1001C000BA8AB684328BAE8B2A84B5E103554E00D1
:1001D00019E501431A851723FFFF670043F1A16763
:1001E000A98F116763FBE70097000000E78080F5A7
:1001F000814597F0FFFFE780C0120844B70700E091
:100200005841F98F18455CC1B707001FF98F1CC50D
:100210005C4991C7610597E00000E780408BE38A65
:1002200009FA228597900000E78060C65DB73285A5
:1002300097C00000E78040430D4349DD1C4411672F
:1002400003D54700A167A98F63FBE7009700000073
:10025000E78040EF814597F0FFFFE780800C0323A4
:10026000840093164B01D1828347B3000356630089
:100270008588FD8BA305F300FD777D8E558EFD7679
:10028000FD16B204F18E83274301C58E231273013C
:100290002313D3002304530123052301A3044301A3
:1002A000BDDF228597B0FFFFE780A0C5AA8508447F
:1002B000B5D1610597D00000E780207F8DB71D4341
:1002C0001A8582801723FFFFE702C3DF0569AA842E
:1002D000AE89328A0144FD5A7D1997C0FFFFE7803D
:1002E000409E6347A40001451723FFFF6700C3E05A
:1002F000D84493171400BA9703D70700631F370336
:100300002390570163070A00268597900000E78035
:10031000A0809C449DC383D76700B3F72701639EE9
:100320003701D2880148814701478146014681450E
:10033000268597000000E78040E5050479BF172374
:10034000FFFFE70223D879711C103EC4B7070F00E6
:100350003EC61C103EC883C79500AA8A328593F713
:10036000F707A384F5002E89328497D0FFFFE7803A
:10037000009D93170501C187635AF006AA8922855B
:1003800097D0FFFFE780A09B2A8A4E85032B0400AD
:1003900097B0FFFFE780809339ED83574400814495
:1003A0000544F11793B71700A303F10083457100CB
:1003B000DA872287D2864E86280097E0FFFFE78003
:1003C000E057014781463000CA85568597B0FFFF48
:1003D000E78040C0A1679387F70348083ECC230A13
:1003E000810026CE97D0FFFFE780406C4561172340
:1003F000FFFF670063D0A2851306710097E0FFFF3F
:10040000E7806066AA84094455D1528597E0FFFFD2
:10041000E78060D40D4459D90546D28526859700DA
:100420000000E78060EA2A8451B71723FFFFE70244
:1004300003CB835507000346270041112A842E85EC
:1004400032C62EC497E0FFFFE780E0D001C93246F4
:10045000A245228597000000E78000E741011723AD
:10046000FFFF670003CA1723FFFFE702C3C483C768
:1004700095004111AA8A93F7F707A384F500328506
:10048000AE89328497D0FFFFE780608B9317050118
:10049000C1876357F00AC1452A8A228597C0FFFFAA
:1004A000E78080702A8D228597D0FFFFE780208922
:1004B0002A89228597D0FFFFE7804086930705F8B9
:1004C00093F7F70F1307E007AA8B637BF7062285E4
:1004D00097D0FFFFE78080842A8C228597D0FFFF8A
:1004E000E780C083AA8C5285032B040097A0FFFFEE
:1004F000E780C07D39E9835744002311010081441E
:10050000F11793B71700A300F1000544034711004A
:1005100083562100938784005685DA882288528684
:10052000CE8597F0FFFFE78020A7A167E907480085
:100530003EC42302810026C697D0FFFFE780005704
:1005400041011723FFFF670083BA13061100A2853C
:1005500097E0FFFFE7802051AA8409E523110100FD
:1005600009446DB7930521006A8597F0FFFFE78086
:10057000A0F02A8441FD835521009356C90013162B
:10058000490185486688E2875E87858A518226858B
:1005900097000000E78060BF2A848DBF1723FFFF0C
:1005A000E70263B183C7950041112A8B93F7F707E0
:1005B000A384F5003285AE89328497C0FFFFE780BF
:1005C000007893170501C1876352F00A2A8A2285B1
:1005D00097C0FFFFE780A076AA8A228597C0FFFF19
:1005E000E780E0752A89228597C0FFFFE7800073C6
:1005F000930705F893F7F70F1307E0072A8C637743
:10060000F706228597C0FFFFE7804071AA8C2285FC
:1006100097C0FFFFE78080702A8D5285832B0400EE
:1006200097A0FFFFE780806A39E58357440085443F
:100630000144F11793B71700A301F10003473100FC
:10064000930784005A85DE882688D6865286CE8512
:1006500097F0FFFFE78040948D4748003EC4230297
:10066000910022C697D0FFFFE78040444101172345
:10067000FFFF6700C3A7A2851306310097E0FFFFC5
:10068000E780603E2A84894455D99356C9001316E1
:10069000490185486A88E6876287858A5182D685BE
:1006A00097000000E78060AEAA8449BF1723FFFFD0
:1006B000E70243A12A8981440144617A916A176B58
:1006C000FF1F130BAB9997B0FFFFE780806063C7F4
:1006D000A40022851723FFFF670003A283270900D8
:1006E00093991400CE9703D50700330745014207BD
:1006F00041836364570305C103270B0019C7854570
:100700003E8597400000E78060E9832709000504E3
:10071000CE972390070085047DB797000000E780FF
:1007200060A2832709000504CE972390070065D5B2
:10073000814597F0FFFFE780C0BEF1BF1723FFFFA1
:10074000E702439883C7950041112A8A93F7F70778
:10075000A384F50032852E89328497C0FFFFE7809D
:10076000005E93170501C187635AF004AA89832AA2
:10077000040097A0FFFFE780605531E583574400F0
:1007800085440144F11793B71700A301F100034812
:100790003100D68752850147CE862686CA8597D0F6
:1007A000FFFFE780806AA167F50748003EC4230287
:1007B000910022C697D0FFFFE780402F4101172309
:1007C000FFFF67006393A2851306310097E0FFFFE8
:1007D000E78060292A8489445DD99767FF1F938742
:1007E000E7879C4381CF044997B0FFFFE780604EC5
:1007F000AA85268597400000E78040DA13050401AA
:1008000097000000E780C0EA228597800000E7801B
:1008100000338144ADBF1723FFFFE702C38983C7BD
:1008200095004111AA8A93F7F707A384F500328552
:10083000AE8932842311010097C0FFFFE78020506A
:1008400093170501C1876354F0062A8AC1452285A2
:1008500097C0FFFFE7804035AA8B5285032B040029
:1008600097A0FFFFE780804621E983574400854435
:100870000144F11793B71700A300F10003481100DA
:1008800003572100DA875685D2862686CE8597D0F3
:10089000FFFFE780805BA1679387270248003EC483
:1008A0002302910022C697D0FFFFE780202041015C
:1008B0001723FFFF6700A383A2851306110097E0AB
:1008C000FFFFE780401A2A8489444DD99757FF1FBC
:1008D0009387C77898433E8901CF044997B0FFFFBB
:1008E000E780203FAA85268597400000E78000CB5F
:1008F0001305040197000000E78080DB97B0FFFF3D
:10090000E780203D95443DD9930521005E8597F011
:10091000FFFFE78060B6AA8435F11C480357210029
:1009200022852390E70097800000E78040218327FD
:100930000900A9D70355210097400000E780A0BD1A
:1009400035BF1713FFFFE702037783C795004111F7
:10095000AA8A93F7F707A384F5003285AE8932841B
:1009600097C0FFFFE780A03D93170501C187635142
:10097000F0062A8A228597C0FFFFE780403C2A893B
:100980005285032B040097A0FFFFE780203431E558
:100990008357440085440144F11793B71700A3011E
:1009A000F10003483100DA8756854A87D2862686C9
:1009B000CE8597D0FFFFE7804049A167F90748003F
:1009C0003EC42302910022C697D0FFFFE780000EAD
:1009D00041011713FFFF67008371A28513063100E1
:1009E00097E0FFFFE78020082A8489445DD991675A
:1009F000CA97C2071167C1831307F7EF8544E36203
:100A0000F7FA9757FF1F938767659843BE8B01CF0F
:100A1000044997B0FFFFE780C02BAA852685974041
:100A20000000E780A0B71305040197000000E780ED
:100A300020C897B0FFFFE780C02995443DD11C48EE
:100A4000228581442390270197800000E780200FB2
:100A500083A70B00B9D74A8597400000E780A0AB79
:100A600089B71713FFFFE70283672A844105B28421
:100A700097000000E780C0C311C522859780000061
:100A8000E780E00B81460146A6852285978000001D
:100A9000E780C04E1C4C89C7DC4799C322858297EA
:100AA0001713FFFF6700E3659757FF1F9387073C06
:100AB0009C43014599C31385070182809757FF1F07
:100AC0009387C73A884382801713FFFFE7022361A9
:100AD0009317C600DD8DC2054111C1812A8432C63B
:100AE00097C0FFFFE780E017324622851182937599
:100AF000F60F97C0FFFFE780C01441011713FFFFF7
:100B0000670023601713FFFFE702C35B79713C089E
:100B10003ED2B7070C003ED43C083ED683C79500B2
:100B2000AE842A8993F7F707A384F500A16593851E
:100B30003504481097A0FFFFE7806024C165FD15CC
:100B40000144175AFF1F130AEA52930A400EAE8956
:100B50002E8B2EC697B0FFFFE780A01A4205931791
:100B600004014181C183B24563E9A702C167FD1752
:100B70006387F500481097C0FFFFE780800E501094
:100B800001478146A6854A8597A0FFFFE7808044FC
:100B900045611713FFFF670023563307540383276C
:100BA0000A0BBA9703D6C701630A3601638A350177
:100BB000481097000000E78060F1DA85050451BF16
:100BC000B285EDBF1713FFFFE702E34E79717C0892
:100BD0003EC8B70711003ECA7C083ECC83C79500CB
:100BE000AA89328593F7F707A384F5002E8997C069
:100BF000FFFFE780C01485676378F504A165AA84C8
:100C00008905080897A0FFFFE780601726859740B1
:100C10000000E78060ED133415000A04A28508087F
:100C200097C0FFFFE780E001A685080897C0FFFF97
:100C3000E780200325CC014781461008CA854E85F0
:100C400097A0FFFFE780003945611713FFFF67009A
:100C5000034AB30754030327CA0ABA9703D7070006
:100C6000631C970003D6270063806505080897007A
:100C70000000E780A0E5DE8505042EC697B0FFFFE3
:100C8000E78020094205931704014181C183B245E1
:100C9000E3E1A7FCC167FD17E38FF5F8080897C0EB
:100CA000FFFFE78000FC41BFB285F9B7C165FD15C4
:100CB0000144175AFF1F130AEA3B930A80022E8B46
:100CC000AE8B65BF1713FFFFE702634118418347EF
:100CD000170083460700A207D58FD207D183239040
:100CE000F50083472700034717008D45A207D98FDA
:100CF00091832310F60097C0FFFFE780A0E9171348
:100D0000FFFF670003401713FFFFE702A33BC16427
:100D100001441759FF1F1309E93593098002FD1497
:100D200097B0FFFFE780E0FE6347A400014517137B
:100D3000FFFF6700633C330534038327C90A3E95F0
:100D400083570500E38597FE0504D9BF1713FFFFFE
:100D5000E70243372A8AAE89B284B68A97400000F8
:100D6000E78080D819E591473E851713FFFF67009C
:100D7000A3382A894E8597C00000E780E08E2A8438
:100D8000638E0A048D476DD103570500C547E31DE7
:100D900047FD0347F9018546AD47E317D7FC834775
:100DA000450081CF4146A6855D0597F00000E780AC
:100DB000C09E814755D9AD4745BF13096501230240
:100DC000E500CA85268597100000E780606231C182
:100DD000A547E38B0AF82302040079B705C18357BE
:100DE0000500E39247F94146A685190597F00000F2
:100DF000E780A09A81472DD99947BDB74E859700C6
:100E00000000E78080F02A84954739DD13095500FA
:100E10004DBF4146A685231044012311340113051B
:100E2000190097F00000E780A099228597800000C4
:100E3000E780A0EA81470DBF1713FFFFE702232ACF
:100E400079717C003ECCB7070A003ECE7C003ED0D4
:100E500083C79500B2842E8493F7F707A384F50027
:100E60001306A1002A892C00268597000000E78040
:100E7000A0E5A16528088D0597A0FFFFE78020F079
:100E800090408355A10003558100854697000000DE
:100E9000E78000ECAA84AA85280897C0FFFFE780B6
:100EA00040DA0356A100835581002808970000000E
:100EB000E780C0C1300801478146A2854A8597A0D6
:100EC000FFFFE7802011854748103ED4230291029E
:100ED00002D697D0FFFFE78060BD45611713FFFF83
:100EE000670023221713FFFFE702631F79717C005D
:100EF0003ECCB7070A003ECE7C003ED083C79500AB
:100F0000B2842E8493F7F707A384F5001306A1009B
:100F10002A892C00268597000000E780E0DAA16589
:100F200028088D0597A0FFFFE78060E59040835576
:100F3000A10003558100814697000000E78040E151
:100F4000AA84AA85280897C0FFFFE78080CF0356B0
:100F5000A10083558100280897000000E78000B7B2
:100F6000300801478146A2854A8597A0FFFFE780A8
:100F7000600648102302910202D402D697D0FFFFE8
:100F8000E780C0B245611713FFFF6700831717138F
:100F9000FFFFE702C31497000000E78060DB171330
:100FA000FFFF670003169757FF1F938767EC88437F
:100FB00082801713FFFFE702831283572500411138
:100FC000AE842A842307B10017F5FFFF13052546D9
:100FD0006C002316F10097A0FFFFE780A04191C4A9
:100FE000228597800000E780E0D6FD572310F400AB
:100FF000130620028145130554009710FFFFE78078
:10100000001141011713FFFF6700A30F1713FFFF24
:10101000E702430B79717C003ECCB7070A003ECE55
:101020007C003ED083C79500AA89AE8493F7F7076A
:101030003285A384F5001306A1002C009700000060
:10104000E78080C803558100114497400000E78085
:10105000A0A915C50355A100014497B00000E78081
:10106000A06011CD035705008357810045446318E4
:10107000F700854597000000E780E0F3014421690F
:1010800093053900280897A0FFFFE78040CFA2858D
:10109000280897C0FFFFE780C0BA0356A100835518
:1010A0008100280897000000E78040A2300801472F
:1010B0008146A6854E8597A0FFFFE780A0F14810E6
:1010C0004AD42302810202D697D0FFFFE780009E18
:1010D00045611713FFFF670023021713FFFFE702A5
:1010E00063FE9757FF1F938767D82A8488432E890A
:1010F00015C5035745038357C4016311F70223261F
:10110000050223180502410597D00000E780209CC6
:101110006306090097800000E78060DB81449759EF
:10112000FF1F938929F5130A800297B0FFFFE7801C
:1011300040BE63C4A4049757FF1F9387E7DB9C431B
:1011400099C70355C40197200000E780C0BD63071D
:101150000900228597800000E780C0A01306400E9A
:10116000814522859710FFFFE78060FAFD57231E17
:10117000F4001713FFFF670023F83385440383A7A8
:10118000C90A3E95035705008357C4016317F7004A
:10119000CA8597000000E78000E2850479B717133D
:1011A000FFFFE70223F283C795004111AA8993F755
:1011B000F707A384F5003285AE8497C0FFFFE78070
:1011C00000B885676378F5042A8997400000E780B6
:1011D000A091014401CD83D70400314463882701E5
:1011E000854597000000E78080EF01444E85A28688
:1011F0004A86A68597D0FFFFE780A09CA1679387CA
:10120000170448003EC42302810002C697D0FFFFA6
:10121000E780C08941011713FFFF6700E3ED171353
:10122000FFFFE70223EA9757FF1F938727C48043F6
:1012300029C4014597C00000E7800021814701488B
:10124000C1641CDC232E0403232004041759FF1F50
:10125000130949E201449309400EFD1497B0FFFFC2
:10126000E78020AA634FA400814517F5FFFF13050F
:10127000857F97A0FFFFE780E0171713FFFF670048
:10128000A3E7330534038327090B3E958357C50134
:1012900063879700854597000000E78040E40504D8
:1012A00075BF9357050113D78700A380F5009317E7
:1012B0000501C183A1832380E5002381F500A3817B
:1012C000A50082801713FFFFE70263E123000500FA
:1012D00083C71500A300F50083C725002301F5008F
:1012E00083C73500A301F50083C745002302F5003D
:1012F00083C75500A302F50083C7650093059500D9
:10130000A30305002303F50023040500328597009D
:101310000000E78040F91713FFFF670083DE171313
:10132000FFFFE70223DA4111E9540DCD85CD93F992
:10133000C5FF2E842A89AA84338AA900B7EA04004B
:1013400063189A020D88854411CCB7E704009C5FAE
:1013500082972AC622866C003305390197E0000087
:10136000E7800046268541011713FFFF6700C3D8B9
:1013700083A78A039104829793170501C183A183F0
:10138000A38EF4FE93570501238FF4FEA183238ED1
:10139000A4FEA38FF4FE6DB763E6D5021713FFFF1B
:1013A000E702E3D3B28741113686BE8536C697E0A1
:1013B0000000E780E040B246410136851713FFFF89
:1013C000670023D481463685828083870500138792
:1013D000F5003D05FD8793F77708834607007D15E7
:1013E0008606B58FA300F5006307B7007D17834716
:1013F00017009D83DDB782801713FFFFE70223CE1E
:10140000B7E7040083A7070932872A863A858297BF
:10141000133515001713FFFF6700A3CE15C18147D1
:101420008DC11713FFFFE70283CB414697E0000011
:10143000E780003985473E851713FFFF670063CCBF
:1014400081473E8582801DCD1713FFFFE70223C928
:10145000414681452A849710FFFFE78040CB4146F3
:101460008145130504039710FFFFE78040CA014739
:10147000C1672322040438C87CC805451713FFFF41
:10148000670023C80145828081473DCDB5CD171344
:10149000FFFFE702C3C4B2842E891306800581458D
:1014A0002A849710FFFFE78080C6CA8524C426855A
:1014B00097000000E780C0F64146814522859710DD
:1014C000FFFFE780C0C43044A2852285970000005A
:1014D000E780C0F293040401A285268597000000EE
:1014E000E780E0EEA6851305040297000000E78080
:1014F00000EE228597000000E78020F585473E85B5
:101500001713FFFF6700E3BF3E8582801713FFFFBD
:10151000E70243BB4111E9540DCD85CD93F9C5FFD9
:101520002E842A89AA84338AA900B7EA0400639822
:1015300044030D88814411CCB7E704009C5F829777
:101540002AC622866C003305390197E00000E78047
:101550002027268541011713FFFF6700E3B983A702
:101560008A039104829793170501C183A183A38EF7
:10157000F4FE93570501238FF4FEA183238EA4FE6E
:10158000A38FF4FE6DB765CD1713FFFFE70283B39A
:10159000B28411E605451713FFFF6700E3B52A84FF
:1015A0002E890145EDD93C487848B3E6E700E5D6F9
:1015B0009386F7FFB3B7F6007D17032A4404BA9762
:1015C00034C87CC863050A06C14913050A03B389F8
:1015D00049412295637D3601B2862E86A685970005
:1015E0000000E780A0DB7C40BE9464C065B7CE8677
:1015F0002E86CE8597000000E78040DAC114D29491
:101600004E9923220404A2879306040103C707000E
:1016100003C607038507318FA38FE7FEE398F6FE25
:101620003044A285228597000000E78020DD2699BE
:10163000C1493306994063EC9900A9DCA686A685CA
:101640001305040397000000E78040D579BF814768
:10165000B306F4003307F6000347070083C506000E
:1016600085072D8F2380E600E39437FF3044A28561
:10167000228597000000E78060D8C1145DBF014556
:1016800082800DC11713FFFFE70263A513068005D3
:1016900081459710FFFFE78080A705451713FFFFDF
:1016A000670023A601458280814749C5C1C517133C
:1016B000FFFFE702C3A2FC4141462E84AA8463993E
:1016C000C70413860501A2878146C14503C70700E9
:1016D00003C507038507298F3305D6000345050099
:1016E0008506298FA38FE7FEE392B6FE3044A285DC
:1016F000268597000000E78060D0228597000000D3
:10170000E78060F885473E851713FFFF6700639FFA
:10171000138507031D8E814522959710FFFFE780F3
:10172000009F7C40130700F813060402A297238849
:10173000E70251BF3E8582801713FFFFE702239A1D
:101740006D712E84B284AA85901028003689970086
:101750000000E780A0D309EDD55725A050400C40EC
:10176000280097000000E78040E27DD5FD142104A9
:10177000F5F42C004A8597000000E78020F38147AC
:1017800061DD3E8551611713FFFF670083971713D3
:10179000FFFFE702C39441112EC432C62C00054658
:1017A00097000000E78080F941011713FFFF6700F1
:1017B00043951713FFFFE702839201112A842EC677
:1017C00002C802CA02CC02CE97E00000E780C02324
:1017D000B2462A86A285080897000000E78060FBD1
:1017E0001375F50F05611713FFFF6700839117133A
:1017F000FFFFE702C38E7971B2872A84214623084E
:10180000B10013051101BE853AC436C697E0000049
:10181000E78000FBB24693059101368597000000F2
:10182000E78060A82285141035460C089700000058
:10183000E78020F62A84224701E921460C103A85E8
:1018400097E00000E780C0F7228545611713FFFF8E
:101850006700238B1713FFFFE70263887171AE8463
:10186000AA850A85328497000000E78060BB11C911
:101870000A86A685228597000000E78020B8814768
:1018800011E1C5473E854D611713FFFF6700638770
:101890001713FFFFE702A3811D712A8AB289BE8454
:1018A00035468547130511012E8CB68A3A8BC28CBA
:1018B000468D2308F10097E00000E78060F01010EB
:1018C0000C085285231F010097000000E780C0F834
:1018D0002A843DEDA1476313FD089307900591E02D
:1018E000E5473546E2851305110113990A012308DE
:1018F000F1001359090197E00000E78060EC1357ED
:10190000890093978A00D98F90080C085285231F6D
:10191000F10097000000E78020F42A8415E9A1E493
:101920009387FA0091831379F9003EC66313090087
:101930004149668B8144C14B854DB247639F970CEB
:101940006A868C0033855C0197E00000E78040E701
:10195000228525611703FFFF670023799307900411
:10196000C9F0A547BDBF834701050947C14B2308FF
:10197000F10083471105A58FA308F1009387240088
:10198000814463E1FB04014714083386E6008C08B8
:10199000B386E400BA95DA9683C6060083C50500CF
:1019A0000507AD8E2300D600E390E7FE4147639C18
:1019B000E70490080C08528597000000E780C0E912
:1019C00025D181A0B3069B00BA871008B305F600A5
:1019D00090083E9603C50600034606008507850667
:1019E000298E2380C500E39277FF998F90080C0819
:1019F0005285BE9497000000E78000E689470147C2
:101A000049D12A84B1B790083E96034606001408CF
:101A1000BE962380C600850759BFB24785046387F9
:101A2000971481471808B306F70098083E97338645
:101A3000F90003470700034606008507318F23801E
:101A4000E600E39177FF90080C08528597000000AC
:101A5000E78080E05DF53546E28513051101230836
:101A6000B10197E00000E780A0D5139704014183FE
:101A7000939784002183D98F10180C085285231F57
:101A8000F10097000000E78020DD25FD8147101858
:101A90003387F9003E960347070003460600B30666
:101AA000FB008507318F2380E600E39277FF65A86E
:101AB0001808B306F70098083E973386F9000347E5
:101AC0000700034606008507318F2380E600E3E127
:101AD00027FFCA87639E770990080C0852859700F4
:101AE0000000E78060D711FD81479800B306F7003A
:101AF000900818103E973E960347070003460600DD
:101B00008507318F2380E600E39177FF3546E28534
:101B1000130511012308B10197E00000E78040CAD6
:101B2000139704014183939784002183D98F101860
:101B30000C085285231FF10097000000E780C0D1F8
:101B4000E31105EC814710183387F9003E960347EF
:101B5000070003460600B306FB008507318F23808C
:101B6000E600E3E227FFC109410BC1BB814785B70E
:101B70009408BE9683C6060018083E972300D70037
:101B8000850789BF638006321703FFFFE7022352F0
:101B900059712A84BE89B28B8547354613051102D7
:101BA0002E8B468C4289BA8A368A2300F10297E04E
:101BB0000000E780E0C010180C10228523170102F6
:101BC00097000000E78040C963180512A147631F12
:101BD000FC069307900563930900E5473546DA85CF
:101BE0001305110293140A012300F102C18097E04A
:101BF0000000E780E0BC93178A0013D78400D98FD8
:101C000090080C1022852317F10297000000E7804E
:101C1000A0C47DE1639209049307FA00BD88918313
:101C200091E0C144C207C183DE8C814A3EC6414D6A
:101C3000B24763E2FA0E6286B3854B01881097E0E3
:101C40000000E78080B54DC93D557DA09307900405
:101C5000E39609F8A54759B7834701050947C14CE1
:101C60002300F10283471105B3C7F900A300F10275
:101C700093872900814963E1FC04814618103306EB
:101C8000D7008C083387D900B695569703470700CD
:101C900083C5050085062D8F2300E600E390D7FE5F
:101CA00041476390E70690080C10228597000000DA
:101CB000E78080BA35D189A0B3863A01BA8710107F
:101CC000B305F60090083E9603C5060003460600DD
:101CD00085078506298E2380C500E39297FF338709
:101CE000EC4090080C102285BA9997000000E7801C
:101CF000A0B68947014741D165611703FFFF67001F
:101D0000C33E90083E96034606001410BE962380FC
:101D1000C600850779B7B247850A93990A01939D52
:101D20008A0093D909016391570F85473546DA85B3
:101D3000130511022300F10293D9890097E00000F6
:101D4000E78000A8B3ED3D0190000C102285231719
:101D5000B10397000000E78020B059FD8147A689B4
:101D600063EA970626860C084A8597E00000E7801C
:101D700020A581471810B306F700100898083E9771
:101D80003E9603470700034606008507318F2380F0
:101D9000E600E3E197FE639FA90590080C102285F9
:101DA00097000000E78040AB21F981479810B30607
:101DB000F700900818183E973E9603470700034621
:101DC00006008507318F2380E600E391A7FF4109D4
:101DD000C10CB9BD18089000B306F7003E963387D2
:101DE000FC0003470700034606008507318F238068
:101DF000E600B5B798084E97034707001C10CE972A
:101E00002380E700850941BF85473546DA851305FC
:101E100011022300F10293D9890097E00000E780C6
:101E2000209AB3ED3D0190000C1022852317B103D9
:101E300097000000E78040A2E31005EC81471808F6
:101E40009000B306F7003E963387FC000347070077
:101E5000034606008507318F2380E600E391A7FF44
:101E600041460C084A8597E00000E780609581476D
:101E70001810B306F700100898083E973E960347DF
:101E80000700034606008507318F2380E600E391B3
:101E9000A7FF90080C10228597000000E780C09BE8
:101EA0001DD599BD7D5582801703FFFFE7022323CF
:101EB00001112A842E8593055100328902C002C285
:101EC00002C402C69304740097F0FFFFE780A03DB0
:101ED0001D46A6851305910097E00000E780408E1F
:101EE00010088A854A8597000000E780E09619ED82
:101EF00093071400180883C60700034607008507E8
:101F00000507B18EA38FD7FEE397F4FE0561170393
:101F1000FFFF6700031F1703FFFFE702A31A2E84CA
:101F20008C414111AA89838715003289914463D37A
:101F30000700A1449747FF1F9387874A9C43A1C787
:101F4000C1CA8D472310F10083C725004A852301AC
:101F5000F10083C73500A301F10083C745002302C8
:101F6000F10083C75500A302F10083C76500930504
:101F70009100A30301002303F1002304010097F063
:101F8000FFFFE78040320C404A860A8597F0FFFF4A
:101F9000E78080330328040083564400A6881D0888
:101FA00081470147E51642868A854E8597000000E5
:101FB000E780408E2A8919E5A685228597B0FFFF24
:101FC000E780E0C14A8541011703FFFF6700C312A4
:101FD0004A860A8597F0FFFFE780002F6DB7170349
:101FE000FFFFE702230E2E848C414111AA898387CB
:101FF00015003289914463D30700A1449747FF1F1E
:102000009387073E9C43A1C7C1C68D472310F100AB
:1020100083C725004A852301F10083C73500A3014A
:10202000F10083C745002302F10083C75500A302D6
:10203000F10083C7650093059100A303010023030A
:10204000F1002304010097F0FFFFE780C0250C405A
:102050004A860A8597F0FFFFE780002783564400F1
:10206000032804008A85858EC2061D08C1822312BA
:10207000D400A68881470147E51642864E85970021
:102080000000E78060B041011703FFFF6700C3064F
:102090004A860A8597F0FFFFE78000234DBF1703AC
:1020A000FFFFE702C303B335B000011185052A899C
:1020B0001315F601336515012308B10093051101CD
:1020C00036843AC632C03EC442C297F0FFFFE78072
:1020D000801DA2471248425593D68700230BF1007A
:1020E0009305910193578800A30AD100A30BF10037
:1020F000230C010197F0FFFFE780E01A3247024608
:1021000003280400B337E00083564400920791444B
:1021100011C2A1444A85A68842860C0897F0FFFFA9
:10212000E78040772A8919E5A685228597B0FFFFC9
:10213000E780E0AA4A8505611703FFFF670063FC9B
:102140001703FFFFE70203F801113EC68647B335C8
:10215000B0008505AA891315F6015D8D2308B1002D
:102160009305110136843A89B28442C446C297F07D
:10217000FFFFE78040132248924816459357880096
:10218000A30AF1009305910193D78800230B010165
:10219000A30BF100230C110197F0FFFFE780A010C3
:1021A0003247104083564400B337E00092070328BB
:1021B0000900914891C0A1480C084E859700000085
:1021C000E780809CAA8401E9835544004A8597B042
:1021D000FFFFE780C0A0268505611703FFFF6700AA
:1021E000A3F1AA959307F00F17070100130787784B
:1021F0006317B50013C5F7FF1375F50F828005054A
:102200008346F5FFB58FBA9783C70700D5B7035745
:10221000450014419307F00F170601001306867559
:10222000369742074183139506014181631BE50000
:10223000AD8FB29703C50700130515F313351500CD
:102240008280850603C5F6FFA98FB29783C7070072
:10225000D9BF1703FFFFE70283E8B28736842E86D3
:10226000BA86AA853E85BA8497F0FFFFE780605260
:10227000634F0500228597D00000E780E0782A862A
:10228000A686A285268597F0FFFFE780805017037A
:10229000FFFF670003E71703FFFFE702A3E25D719B
:1022A0002A8BAE8A170501001305456A2C00B284FB
:1022B000368ABA893E8997F0FFFFE780C04F2A84AB
:1022C0005DE134104146DA85280097F0FFFFE78092
:1022D000404C2A8449E98547A303F100A6C293072D
:1022E00071002408BEC4A68685470D462C18281008
:1022F00002DC02DED6C0BEC697F0FFFFE7800044D6
:102300002A8435E183477102A6860D4693F7F707C5
:102310002300FA00C1473EDE2C188947281026DC2E
:10232000A303F10097F0FFFFE78040412A8405ED09
:102330004146A6854E8597D00000E78060488D47CE
:10234000A6860D462C182810A303F10097F0FFFF76
:10235000E780C03E2A8401E94146A6854A8597D098
:102360000000E780E045228561611703FFFF6700F9
:10237000A3D81703FFFFE70283D697F700009387E0
:10238000E7A1984383C7470079712A89AE8417056E
:1023900001001305255C0C083AC42306F10097F0F0
:1023A000FFFFE78040412A8405ED14104146CA85AD
:1023B000080897F0FFFFE780C03D2A8415E1140864
:1023C00015462C00081097F0FFFFE780803C2A8418
:1023D00001E921462C08268597D00000E780403E81
:1023E000228545611703FFFF6700A3D11703FFFF95
:1023F000E702E3CE97F700009387479A9C477971ED
:10240000AA842E8417050100130545550C083EC605
:1024100097F0FFFFE780203A0DE914104146A685AA
:10242000080897F0FFFFE780C03605E11408114661
:102430006C00081097F0FFFFE780A03519E583478F
:10244000F10193F7F7032300F40045611703FFFF41
:10245000670023CB1703FFFFE70263C83688A14854
:1024600081470147E54697F0FFFFE780A042170349
:10247000FFFF670003C91703FFFFE70243C6368863
:10248000A14881470147E54697F0FFFFE780C06F0D
:102490001703FFFF6700E3C61703FFFFE70223C42C
:1024A00001112A842E850C0832C697F0FFFFE780C1
:1024B000803009ED3247970601009386A648100840
:1024C000C145228597000000E780E0D80561170329
:1024D000FFFF670003C31703FFFFE70243C041117B
:1024E000C1472EC032C48A8509463EC23EC697F017
:1024F000FFFFE780A02441011703FFFF670063C0CF
:102500001703FFFFE702A3BD4111AE8613061009B2
:10251000AA850A8502C002C202C402C697F0FFFF64
:10252000E780202741011703FFFF670083BD1703E2
:10253000FFFFE702C3BA32879706010093868642FF
:102540002E869305000297000000E780C0D0170395
:10255000FFFF670003BB1703FFFFE70243B8797172
:10256000C1472ACC2ED032D42C080D4628003ECEAE
:102570003ED23ED602C402C602C802CA97F0FFFF8E
:10258000E780C01B45611703FFFF670083B7170390
:10259000FFFFE702C3B40111AA842E8417050100CE
:1025A0001305C53C8A8597F0FFFFE780C02015E53D
:1025B00014084146A6850A8597F0FFFFE780601D55
:1025C00009ED8347E1010347F101A207D98FCA074B
:1025D000C9836177D98F2310F40005611703FFFFCA
:1025E000670023B215CD1703FFFFE70243AF9747FC
:1025F000FF1F9387678C90439745FF1F9385058C3A
:102600001745FF1F1305458797D00000E78000C5D9
:102610001745FF1F130545861703FFFF670063AECD
:102620001745FF1F1305458582808DCD1703FFFFDA
:10263000E702E3AA9747FF1F938707889443011196
:102640002E840A869745FF1F9385458797D0000003
:10265000E78040C60A850294014505611703FFFF24
:10266000670023AA7D5582801703FFFFE70223A797
:1026700097D00000E78080D19747FF1F23AEA78245
:1026800017F5FFFF1305E5C997B00000E780C07498
:102690001703FFFF6700E3A61747FF1F1307078411
:1026A0009317150008433E95FD572310F5008280CF
:1026B0001703FFFFE702A3A22A84084009E51703D6
:1026C000FFFF670003A41C4158401CC06313E500D2
:1026D0005CC08347550023200500F99BA302F50049
:1026E00097A0FFFFE780207CC9BF1703FFFFE70229
:1026F000639D9747FF1F9387678098432A8411CB78
:102700008347350093F7070289C7035505008945BC
:1027100002971305440197B00000E780403B8355C2
:1027200004000355E40097300000E780A00C4858EF
:1027300019C597A0FFFFE7800077232A040213053D
:10274000840397000000E780E0F68144B149979048
:10275000FFFFE780406663CBA40283473400232059
:10276000040493F727FCA301F40000489790FFFFAF
:10277000E780606513161500814522859700FFFFED
:10278000E780E0981703FFFF67000397B3873403E0
:102790000329040385043E994A8597000000E780D9
:1027A00060F12304090065B78347350093F70702FA
:1027B00099E3014582808357E500E39CB7FEC1673A
:1027C000FD176316F60005458280054599A8170395
:1027D000FFFFE702C39093170601C187B2842A84E2
:1027E00001496359F002835705009DCB014563679A
:1027F000F600034584003E953325A6001375F50FBA
:102800000DA01C4813171900BA9783D70700E38E51
:1028100097FA05099790FFFFE780E05AE343A9FE86
:1028200001451703FFFF6700C38D1703FFFFE70292
:102830006389AE89AA849790FFFFE780804E2A843F
:1028400097D0FFFFE780A02EAA86014713068401D8
:1028500097050000938585E41735FF1F130545682C
:102860009790FFFFE78000152A8925C98C4413043F
:10287000C50022859E0593F5050897A0FFFFE78018
:10288000403CCC4083877400E18163DD070493E51D
:102890000508228597A0FFFFE780A03A0D469385A3
:1028A0004400228597A0FFFFE780C03683D504004F
:1028B000228597A0FFFFE780E03D83D52400228595
:1028C00097A0FFFFE780003D03D6490083A50900DC
:1028D000228597A0FFFFE780E0334A851703FFFFBB
:1028E0006700838193F5F5076DB717F3FEFFE702E5
:1028F000037F01112A84328532C697A0FFFFE7804B
:10290000E0279780FFFFE780E02C8357040017370C
:10291000FF1F130727763246231BF100930700F8A9
:10292000A30DF1001C471843231AA1008983858B4E
:10293000B307F740B28548083ECE231C0100230DA3
:10294000010097000000E78080EE056117F3FEFFAD
:102950006700237B17F3FEFFE702C37600410145C2
:102960003DC49304C40026853289AE8997A0FFFF39
:10297000E780C02495452A8A2685035B040197A039
:10298000FFFFE7802021268597A0FFFFE780603EBC
:102990008D45AA8A268597A0FFFFE780A01F268580
:1029A00097A0FFFFE780E03C5C48420A135A0A0107
:1029B000D2975CC423186401814763983A014605A5
:1029C0004D81330625419337160013F5F70F17F3A2
:1029D000FEFF6700637217F3FEFFE702C36D8969AC
:1029E0002A8BAE8B328AB68A81440144314CFD1960
:1029F0009790FFFFE780203C63CDA4009790FFFFF6
:102A0000E780603E018D33B5AA0017F3FEFF670033
:102A1000036E3389840383270B003E9963170A00F2
:102A20008347890085043E94E1B703560A00DE859A
:102A30004A8533F6C90097000000E780E0F16DD1C8
:102A40000545E1B717F3FEFFE702636901112A8428
:102A50007C000355E5003ECAB70707003ECC7C006A
:102A60003ECE97200000E78020082A898545480847
:102A700097A0FFFFE78020399945480897A0FFFFFE
:102A8000E780E015AA844A8597200000E780A00827
:102A90002380A4009737FF1F9387C75D9C4341663F
:102AA000130606F09396870113D78701558F93D6A7
:102AB0008700F18E558FA207B706FF00F58FD98FDB
:102AC00011462C00138514003EC497D00000E78007
:102AD00020CF5008A382040089452285970000007A
:102AE000E780E0E019C9AA851305840397A0FFFFDA
:102AF000E780E0313C4085073CC0056117F3FEFFED
:102B00006700236017F3FEFFE702635D9790FFFF06
:102B1000E780602D2A8405049790FFFFE780A02BB3
:102B20003305A402F14791453305F50297200000D3
:102B3000E78020BA11E5655517F3FEFF6700635C77
:102B40009737FF1F23A4A73A9790FFFFE780A0299C
:102B50002A8405049790FFFFE780E0273305A4024D
:102B60008945060597200000E780A0B669D597370C
:102B7000FF1F23A5A7369790FFFFE780C0262A8472
:102B800005049790FFFFE78000253304A4029737E0
:102B9000FF1F239787349790FFFFE780C0242A8484
:102BA0009790FFFFE7802023930714003385A70247
:102BB0009737FF1F2397A732970701009387C79E78
:102BC0001737FF1F2322F7320145BDB717F3FEFF6A
:102BD000E702434FAA842E8901449739FF1F938946
:102BE0006949130A80069790FFFFE780C01E63477C
:102BF000A400014517F3FEFF6700035033054403AB
